
IBM(R) Linker for OS/2(R), Version 5.0 
Copyright (C) IBM Corporation 1988, 2003.
Copyright (C) Microsoft Corp. 1988, 1989.
All rights reserved.

Current option settings:
	PDD	CODE:RX	DATA:RWS
	Alignfile:0x00000010	ALIGNAddr:0x00010000	NOBASe
	BRowse	NODBgpack	DEbug:none	NODEFaultlibrarysearch
	NOEXEPACK	NOEXTdictionary	NOFIxed	FReeformat	NOIGnorecase
	Linenumbers	NOLOgo	MAP:bin\Debug.ACP\uniaud32.map
	OCache:0x1cb4cc00	OLDcpp	NOOPTFunc	PACKCode:0xffffffff
	PACKData:0xffffffff	PMTYPE:VIO	SEGMENTS:256 	NOSEGOrder
	NOSTRictwarnings	NONOSTRictwarnings	NOSTUB	NOVERBose
	VERSION:00.00


ILink : warning LNK4019: device driver can not have a stack

 UNIAUD32

 Start         Length     Name                   Class
 0001:00000000 00000048BH DATA16                 DATA16 16-bit
	at offset 00000000 0048BH bytes from F:\src\os2\uniaud32\drv32\bin\Debug.ACP\startup.obj (startup.asm)

 0002:00000000 0000006DBH CODE16                 CODE 16-bit
	at offset 00000000 006DBH bytes from F:\src\os2\uniaud32\drv32\bin\Debug.ACP\startup.obj (startup.asm)

 0003:00000000 000000000H FIRSTCODE32            CODE 32-bit

 0003:00000000 0000E6756H CODE32                 CODE 32-bit
	at offset 00000000 004DDH bytes from F:\src\os2\uniaud32\drv32\bin\Debug.ACP\startup.obj (startup.asm)
	at offset 000004DD 001FBH bytes from F:\src\os2\uniaud32\drv32\bin\Debug.ACP\strategy.obj (F:\src\os2\uniaud32\drv32\strategy.c)
	at offset 000006D8 00176H bytes from F:\src\os2\uniaud32\drv32\bin\Debug.ACP\read.obj (F:\src\os2\uniaud32\drv32\read.cpp)
	at offset 0000084E 005CFH bytes from F:\src\os2\uniaud32\drv32\bin\Debug.ACP\init.obj (F:\src\os2\uniaud32\drv32\init.c)
	at offset 00000E1D 00807H bytes from F:\src\os2\uniaud32\drv32\bin\Debug.ACP\parse.obj (F:\src\os2\uniaud32\drv32\parse.c)
	at offset 00001624 0004EH bytes from F:\src\os2\uniaud32\drv32\bin\Debug.ACP\devhlp.obj (devhlp.asm)
	at offset 00001672 00641H bytes from F:\src\os2\uniaud32\drv32\bin\Debug.ACP\idc.obj (F:\src\os2\uniaud32\drv32\idc.c)
	at offset 00001CB3 00C39H bytes from F:\src\os2\uniaud32\drv32\bin\Debug.ACP\dispatch.obj (F:\src\os2\uniaud32\drv32\dispatch.c)
	at offset 000028EC 00A3AH bytes from F:\src\os2\uniaud32\drv32\bin\Debug.ACP\rmhelp.obj (F:\src\os2\uniaud32\drv32\rmhelp.cpp)
	at offset 00003326 0018EH bytes from F:\src\os2\uniaud32\drv32\bin\Debug.ACP\irq.obj (F:\src\os2\uniaud32\drv32\irq.cpp)
	at offset 000034B4 00194H bytes from F:\src\os2\uniaud32\drv32\bin\Debug.ACP\util.obj (F:\src\os2\uniaud32\drv32\util.cpp)
	at offset 00003648 00724H bytes from F:\src\os2\uniaud32\lib\Debug.ACP\linuxlib.lib (F:\src\os2\uniaud32\lib32\vsprintf.c)
	at offset 00003D6C 00204H bytes from F:\src\os2\uniaud32\lib\Debug.ACP\linuxlib.lib (F:\src\os2\uniaud32\lib32\timer.c)
	at offset 00003F70 000CCH bytes from F:\src\os2\uniaud32\lib\Debug.ACP\linuxlib.lib (F:\src\os2\uniaud32\lib32\strncmp.c)
	at offset 0000403C 000AEH bytes from F:\src\os2\uniaud32\lib\Debug.ACP\linuxlib.lib (F:\src\os2\uniaud32\lib32\task.c)
	at offset 000040EA 00B31H bytes from F:\src\os2\uniaud32\lib\Debug.ACP\linuxlib.lib (F:\src\os2\uniaud32\lib32\misc.c)
	at offset 00004C1B 004DBH bytes from F:\src\os2\uniaud32\lib\Debug.ACP\linuxlib.lib (F:\src\os2\uniaud32\lib32\ossidc.cpp)
	at offset 000050F6 00966H bytes from F:\src\os2\uniaud32\lib\Debug.ACP\linuxlib.lib (F:\src\os2\uniaud32\lib32\soundmidi.c)
	at offset 00005A5C 017B1H bytes from F:\src\os2\uniaud32\lib\Debug.ACP\linuxlib.lib (F:\src\os2\uniaud32\lib32\soundmixer.c)
	at offset 0000720D 02654H bytes from F:\src\os2\uniaud32\lib\Debug.ACP\linuxlib.lib (F:\src\os2\uniaud32\lib32\sound.c)
	at offset 00009861 00806H bytes from F:\src\os2\uniaud32\lib\Debug.ACP\linuxlib.lib (F:\src\os2\uniaud32\lib32\debug.c)
	at offset 0000A067 00B85H bytes from F:\src\os2\uniaud32\lib\Debug.ACP\linuxlib.lib (F:\src\os2\uniaud32\lib32\memory.cpp)
	at offset 0000ABEC 01C82H bytes from F:\src\os2\uniaud32\lib\Debug.ACP\linuxlib.lib (F:\src\os2\uniaud32\lib32\ioctl.c)
	at offset 0000C86E 0050DH bytes from F:\src\os2\uniaud32\lib\Debug.ACP\linuxlib.lib (F:\src\os2\uniaud32\lib32\irq.c)
	at offset 0000CD7B 02C25H bytes from F:\src\os2\uniaud32\lib\Debug.ACP\linuxlib.lib (F:\src\os2\uniaud32\lib32\pci.c)
	at offset 0000F9A0 0092FH bytes from F:\src\os2\uniaud32\lib\Debug.ACP\linuxlib.lib (F:\src\os2\uniaud32\lib32\malloc.cpp)
	at offset 000102CF 00067H bytes from F:\src\os2\uniaud32\lib\Debug.ACP\linuxlib.lib (F:\src\os2\uniaud32\lib32\strncpy.c)
	at offset 00010336 0013FH bytes from F:\src\os2\uniaud32\lib\Debug.ACP\linuxlib.lib (F:\src\os2\uniaud32\lib32\waitqueue.c)
	at offset 00010475 000B6H bytes from F:\src\os2\uniaud32\lib\Debug.ACP\linuxlib.lib (F:\src\os2\uniaud32\lib32\spinlock.c)
	at offset 0001052B 01019H bytes from F:\src\os2\uniaud32\lib\Debug.ACP\core.lib (F:\src\os2\uniaud32\alsa-kernel\core\hwdep.c)
	at offset 00011544 03FB7H bytes from F:\src\os2\uniaud32\lib\Debug.ACP\core.lib (F:\src\os2\uniaud32\alsa-kernel\core\timer.c)
	at offset 000154FB 031F3H bytes from F:\src\os2\uniaud32\lib\Debug.ACP\core.lib (F:\src\os2\uniaud32\alsa-kernel\core\rawmidi.c)
	at offset 000186EE 005BCH bytes from F:\src\os2\uniaud32\lib\Debug.ACP\core.lib (F:\src\os2\uniaud32\alsa-kernel\core\pcm_misc.c)
	at offset 00018CAA 04BB2H bytes from F:\src\os2\uniaud32\lib\Debug.ACP\core.lib (F:\src\os2\uniaud32\alsa-kernel\core\pcm_lib.c)
	at offset 0001D85C 016D5H bytes from F:\src\os2\uniaud32\lib\Debug.ACP\core.lib (F:\src\os2\uniaud32\alsa-kernel\core\pcm.c)
	at offset 0001EF31 007D9H bytes from F:\src\os2\uniaud32\lib\Debug.ACP\core.lib (F:\src\os2\uniaud32\alsa-kernel\core\sound.c)
	at offset 0001F70A 0191FH bytes from F:\src\os2\uniaud32\lib\Debug.ACP\core.lib (F:\src\os2\uniaud32\alsa-kernel\core\info.c)
	at offset 00021029 00784H bytes from F:\src\os2\uniaud32\lib\Debug.ACP\core.lib (F:\src\os2\uniaud32\alsa-kernel\core\pcm_memory.c)
	at offset 000217AD 00372H bytes from F:\src\os2\uniaud32\lib\Debug.ACP\core.lib (F:\src\os2\uniaud32\alsa-kernel\core\pcm_timer.c)
	at offset 00021B1F 06C49H bytes from F:\src\os2\uniaud32\lib\Debug.ACP\core.lib (F:\src\os2\uniaud32\alsa-kernel\core\pcm_native.c)
	at offset 00028768 0034DH bytes from F:\src\os2\uniaud32\lib\Debug.ACP\core.lib (F:\src\os2\uniaud32\alsa-kernel\core\info_oss.c)
	at offset 00028AB5 00692H bytes from F:\src\os2\uniaud32\lib\Debug.ACP\core.lib (F:\src\os2\uniaud32\alsa-kernel\core\sound_oss.c)
	at offset 00029147 005C9H bytes from F:\src\os2\uniaud32\lib\Debug.ACP\core.lib (F:\src\os2\uniaud32\alsa-kernel\core\device.c)
	at offset 00029710 02F49H bytes from F:\src\os2\uniaud32\lib\Debug.ACP\core.lib (F:\src\os2\uniaud32\alsa-kernel\core\control.c)
	at offset 0002C659 00714H bytes from F:\src\os2\uniaud32\lib\Debug.ACP\core.lib (F:\src\os2\uniaud32\alsa-kernel\core\memalloc.c)
	at offset 0002CD6D 01530H bytes from F:\src\os2\uniaud32\lib\Debug.ACP\core.lib (F:\src\os2\uniaud32\alsa-kernel\core\init.c)
	at offset 0002E29D 002DEH bytes from F:\src\os2\uniaud32\lib\Debug.ACP\core.lib (F:\src\os2\uniaud32\alsa-kernel\core\sgbuf.c)
	at offset 0002E57B 019B9H bytes from F:\src\os2\uniaud32\lib\Debug.ACP\pci.lib (F:\src\os2\uniaud32\alsa-kernel\pci\bt87x.c)
	at offset 0002FF34 0143EH bytes from F:\src\os2\uniaud32\lib\Debug.ACP\pci.lib (F:\src\os2\uniaud32\alsa-kernel\pci\als4000.c)
	at offset 00031372 050E4H bytes from F:\src\os2\uniaud32\lib\Debug.ACP\pci.lib (F:\src\os2\uniaud32\alsa-kernel\pci\cmipci.c)
	at offset 00036456 02745H bytes from F:\src\os2\uniaud32\lib\Debug.ACP\pci.lib (F:\src\os2\uniaud32\alsa-kernel\pci\atiixp.c)
	at offset 00038B9B 020A1H bytes from F:\src\os2\uniaud32\lib\Debug.ACP\pci.lib (F:\src\os2\uniaud32\alsa-kernel\pci\fm801.c)
	at offset 0003AC3C 03D14H bytes from F:\src\os2\uniaud32\lib\Debug.ACP\pci.lib (F:\src\os2\uniaud32\alsa-kernel\pci\via82xx.c)
	at offset 0003E950 0309AH bytes from F:\src\os2\uniaud32\lib\Debug.ACP\pci.lib (F:\src\os2\uniaud32\alsa-kernel\pci\maestro3.c)
	at offset 000419EA 04EA8H bytes from F:\src\os2\uniaud32\lib\Debug.ACP\pci.lib (F:\src\os2\uniaud32\alsa-kernel\pci\intel8x0.c)
	at offset 00046892 0429AH bytes from F:\src\os2\uniaud32\lib\Debug.ACP\pci.lib (F:\src\os2\uniaud32\alsa-kernel\pci\es1968.c)
	at offset 0004AB2C 02C2AH bytes from F:\src\os2\uniaud32\lib\Debug.ACP\pci.lib (F:\src\os2\uniaud32\alsa-kernel\pci\es1938.c)
	at offset 0004D756 03536H bytes from F:\src\os2\uniaud32\lib\Debug.ACP\pci.lib (F:\src\os2\uniaud32\alsa-kernel\pci\cs4281.c)
	at offset 00050C8C 031D8H bytes from F:\src\os2\uniaud32\lib\Debug.ACP\pci.lib (F:\src\os2\uniaud32\alsa-kernel\pci\ens1371.c)
	at offset 00053E64 0046DH bytes from F:\src\os2\uniaud32\lib\Debug.ACP\pci.lib (F:\src\os2\uniaud32\alsa-kernel\pci\pci_iomap_compat.c)
	at offset 000542D1 02958H bytes from F:\src\os2\uniaud32\lib\Debug.ACP\ca0106.lib (F:\src\os2\uniaud32\alsa-kernel\pci\ca0106\ca0106_main.c)
	at offset 00056C29 00899H bytes from F:\src\os2\uniaud32\lib\Debug.ACP\ca0106.lib (F:\src\os2\uniaud32\alsa-kernel\pci\ca0106\ca_midi.c)
	at offset 000574C2 015E3H bytes from F:\src\os2\uniaud32\lib\Debug.ACP\ca0106.lib (F:\src\os2\uniaud32\alsa-kernel\pci\ca0106\ca0106_mixer.c)
	at offset 00058AA5 00DDCH bytes from F:\src\os2\uniaud32\lib\Debug.ACP\ca0106.lib (F:\src\os2\uniaud32\alsa-kernel\pci\ca0106\ca0106_proc.c)
	at offset 00059881 09414H bytes from F:\src\os2\uniaud32\lib\Debug.ACP\hda.lib (F:\src\os2\uniaud32\alsa-kernel\pci\hda\patch_via.c)
	at offset 00062C95 02B72H bytes from F:\src\os2\uniaud32\lib\Debug.ACP\hda.lib (F:\src\os2\uniaud32\alsa-kernel\pci\hda\patch_conexant.c)
	at offset 00065807 003FFH bytes from F:\src\os2\uniaud32\lib\Debug.ACP\hda.lib (F:\src\os2\uniaud32\alsa-kernel\pci\hda\patch_atihdmi.c)
	at offset 00065C06 081EBH bytes from F:\src\os2\uniaud32\lib\Debug.ACP\hda.lib (F:\src\os2\uniaud32\alsa-kernel\pci\hda\patch_sigmatel.c)
	at offset 0006DDF1 03F77H bytes from F:\src\os2\uniaud32\lib\Debug.ACP\hda.lib (F:\src\os2\uniaud32\alsa-kernel\pci\hda\patch_analog.c)
	at offset 00071D68 00D7BH bytes from F:\src\os2\uniaud32\lib\Debug.ACP\hda.lib (F:\src\os2\uniaud32\alsa-kernel\pci\hda\patch_cmedia.c)
	at offset 00072AE3 0CEBAH bytes from F:\src\os2\uniaud32\lib\Debug.ACP\hda.lib (F:\src\os2\uniaud32\alsa-kernel\pci\hda\patch_realtek.c)
	at offset 0007F99D 03DE1H bytes from F:\src\os2\uniaud32\lib\Debug.ACP\hda.lib (F:\src\os2\uniaud32\alsa-kernel\pci\hda\hda_intel.c)
	at offset 0008377E 0704DH bytes from F:\src\os2\uniaud32\lib\Debug.ACP\hda.lib (F:\src\os2\uniaud32\alsa-kernel\pci\hda\hda_codec.c)
	at offset 0008A7CB 00463H bytes from F:\src\os2\uniaud32\lib\Debug.ACP\hda.lib (F:\src\os2\uniaud32\alsa-kernel\pci\hda\hda_hwdep.c)
	at offset 0008AC2E 01F9CH bytes from F:\src\os2\uniaud32\lib\Debug.ACP\hda.lib (F:\src\os2\uniaud32\alsa-kernel\pci\hda\hda_generic.c)
	at offset 0008CBCA 01B1AH bytes from F:\src\os2\uniaud32\lib\Debug.ACP\hda.lib (F:\src\os2\uniaud32\alsa-kernel\pci\hda\hda_proc.c)
	at offset 0008E6E4 000AEH bytes from F:\src\os2\uniaud32\lib\Debug.ACP\sequencer.lib (F:\src\os2\uniaud32\alsa-kernel\core\seq\seq.c)
	at offset 0008E792 00BA2H bytes from F:\src\os2\uniaud32\lib\Debug.ACP\sequencer.lib (F:\src\os2\uniaud32\alsa-kernel\core\seq\seq_device.c)
	at offset 0008F334 00117H bytes from F:\src\os2\uniaud32\lib\Debug.ACP\sequencer.lib (F:\src\os2\uniaud32\alsa-kernel\core\seq\seq_info.c)
	at offset 0008F44B 00317H bytes from F:\src\os2\uniaud32\lib\Debug.ACP\sequencer.lib (F:\src\os2\uniaud32\alsa-kernel\core\seq\seq_system.c)
	at offset 0008F762 01427H bytes from F:\src\os2\uniaud32\lib\Debug.ACP\sequencer.lib (F:\src\os2\uniaud32\alsa-kernel\core\seq\seq_queue.c)
	at offset 00090B89 00CF0H bytes from F:\src\os2\uniaud32\lib\Debug.ACP\sequencer.lib (F:\src\os2\uniaud32\alsa-kernel\core\seq\seq_memory.c)
	at offset 00091879 03ED2H bytes from F:\src\os2\uniaud32\lib\Debug.ACP\sequencer.lib (F:\src\os2\uniaud32\alsa-kernel\core\seq\seq_clientmgr.c)
	at offset 0009574B 01515H bytes from F:\src\os2\uniaud32\lib\Debug.ACP\sequencer.lib (F:\src\os2\uniaud32\alsa-kernel\core\seq\seq_ports.c)
	at offset 00096C60 00CAAH bytes from F:\src\os2\uniaud32\lib\Debug.ACP\sequencer.lib (F:\src\os2\uniaud32\alsa-kernel\core\seq\seq_timer.c)
	at offset 0009790A 00A34H bytes from F:\src\os2\uniaud32\lib\Debug.ACP\sequencer.lib (F:\src\os2\uniaud32\alsa-kernel\core\seq\seq_prioq.c)
	at offset 0009833E 0061FH bytes from F:\src\os2\uniaud32\lib\Debug.ACP\sequencer.lib (F:\src\os2\uniaud32\alsa-kernel\core\seq\seq_fifo.c)
	at offset 0009895D 006F7H bytes from F:\src\os2\uniaud32\lib\Debug.ACP\opl3.lib (F:\src\os2\uniaud32\alsa-kernel\drivers\opl3\opl3_seq.c)
	at offset 00099054 00D69H bytes from F:\src\os2\uniaud32\lib\Debug.ACP\opl3.lib (F:\src\os2\uniaud32\alsa-kernel\drivers\opl3\opl3_lib.c)
	at offset 00099DBD 003D2H bytes from F:\src\os2\uniaud32\lib\Debug.ACP\opl3.lib (F:\src\os2\uniaud32\alsa-kernel\drivers\opl3\opl3_drums.c)
	at offset 0009A18F 0127CH bytes from F:\src\os2\uniaud32\lib\Debug.ACP\opl3.lib (F:\src\os2\uniaud32\alsa-kernel\drivers\opl3\opl3_midi.c)
	at offset 0009B40B 00D57H bytes from F:\src\os2\uniaud32\lib\Debug.ACP\opl3.lib (F:\src\os2\uniaud32\alsa-kernel\drivers\opl3\opl3_synth.c)
	at offset 0009C162 00F18H bytes from F:\src\os2\uniaud32\lib\Debug.ACP\mpu401.lib (F:\src\os2\uniaud32\alsa-kernel\drivers\mpu401\mpu401_uart.c)
	at offset 0009D07A 002D4H bytes from F:\src\os2\uniaud32\lib\Debug.ACP\cs46xx.lib (F:\src\os2\uniaud32\alsa-kernel\pci\cs46xx\cs46xx.c)
	at offset 0009D34E 04673H bytes from F:\src\os2\uniaud32\lib\Debug.ACP\cs46xx.lib (F:\src\os2\uniaud32\alsa-kernel\pci\cs46xx\cs46xx_lib.c)
	at offset 000A19C1 00956H bytes from F:\src\os2\uniaud32\lib\Debug.ACP\cs5535audio.lib (F:\src\os2\uniaud32\alsa-kernel\pci\cs5535audio\cs5535audio.c)
	at offset 000A2317 002B3H bytes from F:\src\os2\uniaud32\lib\Debug.ACP\cs5535audio.lib (F:\src\os2\uniaud32\alsa-kernel\pci\cs5535audio\cs5535audio_pm.c)
	at offset 000A25CA 00B55H bytes from F:\src\os2\uniaud32\lib\Debug.ACP\cs5535audio.lib (F:\src\os2\uniaud32\alsa-kernel\pci\cs5535audio\cs5535audio_pcm.c)
	at offset 000A311F 0068EH bytes from F:\src\os2\uniaud32\lib\Debug.ACP\emu10k1.lib (F:\src\os2\uniaud32\alsa-kernel\pci\emu10k1\emu10k1.c)
	at offset 000A37AD 015ABH bytes from F:\src\os2\uniaud32\lib\Debug.ACP\emu10k1.lib (F:\src\os2\uniaud32\alsa-kernel\pci\emu10k1\p16v.c)
	at offset 000A4D58 001E4H bytes from F:\src\os2\uniaud32\lib\Debug.ACP\emu10k1.lib (F:\src\os2\uniaud32\alsa-kernel\pci\emu10k1\timer.c)
	at offset 000A4F3C 082E8H bytes from F:\src\os2\uniaud32\lib\Debug.ACP\emu10k1.lib (F:\src\os2\uniaud32\alsa-kernel\pci\emu10k1\emufx.c)
	at offset 000AD224 03247H bytes from F:\src\os2\uniaud32\lib\Debug.ACP\emu10k1.lib (F:\src\os2\uniaud32\alsa-kernel\pci\emu10k1\emumixer.c)
	at offset 000B046B 03D70H bytes from F:\src\os2\uniaud32\lib\Debug.ACP\emu10k1.lib (F:\src\os2\uniaud32\alsa-kernel\pci\emu10k1\emupcm.c)
	at offset 000B41DB 00B31H bytes from F:\src\os2\uniaud32\lib\Debug.ACP\emu10k1.lib (F:\src\os2\uniaud32\alsa-kernel\pci\emu10k1\emumpu401.c)
	at offset 000B4D0C 02999H bytes from F:\src\os2\uniaud32\lib\Debug.ACP\emu10k1.lib (F:\src\os2\uniaud32\alsa-kernel\pci\emu10k1\emu10k1_main.c)
	at offset 000B76A5 00FCEH bytes from F:\src\os2\uniaud32\lib\Debug.ACP\emu10k1.lib (F:\src\os2\uniaud32\alsa-kernel\pci\emu10k1\emuproc.c)
	at offset 000B8673 00F59H bytes from F:\src\os2\uniaud32\lib\Debug.ACP\emu10k1.lib (F:\src\os2\uniaud32\alsa-kernel\pci\emu10k1\io.c)
	at offset 000B95CC 00431H bytes from F:\src\os2\uniaud32\lib\Debug.ACP\emu10k1.lib (F:\src\os2\uniaud32\alsa-kernel\pci\emu10k1\voice.c)
	at offset 000B99FD 00F44H bytes from F:\src\os2\uniaud32\lib\Debug.ACP\emu10k1.lib (F:\src\os2\uniaud32\alsa-kernel\pci\emu10k1\memory.c)
	at offset 000BA941 00551H bytes from F:\src\os2\uniaud32\lib\Debug.ACP\emu10k1.lib (F:\src\os2\uniaud32\alsa-kernel\pci\emu10k1\irq.c)
	at offset 000BAE92 0088FH bytes from F:\src\os2\uniaud32\lib\Debug.ACP\ymfpci.lib (F:\src\os2\uniaud32\alsa-kernel\pci\ymfpci\ymfpci.c)
	at offset 000BB721 059D0H bytes from F:\src\os2\uniaud32\lib\Debug.ACP\ymfpci.lib (F:\src\os2\uniaud32\alsa-kernel\pci\ymfpci\ymfpci_main.c)
	at offset 000C10F1 036E1H bytes from F:\src\os2\uniaud32\lib\Debug.ACP\ali5451.lib (F:\src\os2\uniaud32\alsa-kernel\pci\ali5451\ali5451.c)
	at offset 000C47D2 00408H bytes from F:\src\os2\uniaud32\lib\Debug.ACP\trident.lib (F:\src\os2\uniaud32\alsa-kernel\pci\trident\trident.c)
	at offset 000C4BDA 05EE4H bytes from F:\src\os2\uniaud32\lib\Debug.ACP\trident.lib (F:\src\os2\uniaud32\alsa-kernel\pci\trident\trident_main.c)
	at offset 000CAABE 00636H bytes from F:\src\os2\uniaud32\lib\Debug.ACP\trident.lib (F:\src\os2\uniaud32\alsa-kernel\pci\trident\trident_memory.c)
	at offset 000CB0F4 02924H bytes from F:\src\os2\uniaud32\lib\Debug.ACP\nm256.lib (F:\src\os2\uniaud32\alsa-kernel\pci\nm256\nm256.c)
	at offset 000CDA18 014B6H bytes from F:\src\os2\uniaud32\lib\Debug.ACP\sb.lib (F:\src\os2\uniaud32\alsa-kernel\isa\sb\sb_mixer.c)
	at offset 000CEECE 006DCH bytes from F:\src\os2\uniaud32\lib\Debug.ACP\sb.lib (F:\src\os2\uniaud32\alsa-kernel\isa\sb\sb_common.c)
	at offset 000CF5AA 0691CH bytes from F:\src\os2\uniaud32\lib\Debug.ACP\core_oss.lib (F:\src\os2\uniaud32\alsa-kernel\core\oss\pcm_oss.c)
	at offset 000D5EE0 00140H bytes from F:\acpi\lib\acpidrv.lib (acpi)
	at offset 000D6020 002BCH bytes from F:\acpi\lib\acpidrv.lib (FindAddress)
	at offset 000D62DC 0010CH bytes from F:\src\os2\uniaud32\lib\Debug.ACP\linuxlib.lib (F:\src\os2\uniaud32\lib32\semaphore.c)
	at offset 000D63E8 00A77H bytes from F:\src\os2\uniaud32\lib\Debug.ACP\core.lib (F:\src\os2\uniaud32\alsa-kernel\core\vmaster.c)
	at offset 000D6E5F 000F3H bytes from F:\src\os2\uniaud32\lib\Debug.ACP\core.lib (F:\src\os2\uniaud32\alsa-kernel\core\misc.c)
	at offset 000D6F52 00160H bytes from F:\src\os2\uniaud32\lib\Debug.ACP\core.lib (F:\src\os2\uniaud32\alsa-kernel\core\memory.c)
	at offset 000D70B2 0136CH bytes from F:\src\os2\uniaud32\lib\Debug.ACP\ac97.lib (F:\src\os2\uniaud32\alsa-kernel\pci\ac97\ac97_pcm.c)
	at offset 000D841E 0B452H bytes from F:\src\os2\uniaud32\lib\Debug.ACP\ac97.lib (F:\src\os2\uniaud32\alsa-kernel\pci\ac97\ac97_codec.c)
	at offset 000E3870 019D7H bytes from F:\src\os2\uniaud32\lib\Debug.ACP\ac97.lib (F:\src\os2\uniaud32\alsa-kernel\pci\ac97\ac97_proc.c)
	at offset 000E5247 010BDH bytes from F:\src\os2\uniaud32\lib\Debug.ACP\sequencer.lib (F:\src\os2\uniaud32\alsa-kernel\core\seq\seq_midi_emul.c)
	at offset 000E6304 00452H bytes from F:\src\os2\uniaud32\lib\Debug.ACP\synth.lib (F:\src\os2\uniaud32\alsa-kernel\synth\util_mem.c)

 0003:000E6760 0000029A6H _TEXT                  CODE 32-bit
	at offset 00000000 0004FH bytes from E:\watcom\lib386\os2\clib3r.lib (i8s)
	at offset 00000050 0001CH bytes from E:\watcom\lib386\os2\clib3r.lib (i8m)
	at offset 00000070 000ADH bytes from E:\watcom\lib386\os2\clib3r.lib (strstr.c)
	at offset 00000120 00041H bytes from E:\watcom\lib386\os2\clib3r.lib (strlcpy.c)
	at offset 00000170 00091H bytes from E:\watcom\lib386\os2\clib3r.lib (sscanf.c)
	at offset 00000210 000C7H bytes from E:\watcom\lib386\os2\clib3r.lib (snprintf.c)
	at offset 000002E0 00018H bytes from E:\watcom\lib386\os2\clib3r.lib (memset.c)
	at offset 00000300 00053H bytes from E:\watcom\lib386\os2\clib3r.lib (memmove.c)
	at offset 00000360 0023DH bytes from E:\watcom\lib386\os2\clib3r.lib (strtol.c)
	at offset 000005A0 00101H bytes from E:\watcom\lib386\os2\clib3r.lib (istable.c)
	at offset 000006B0 000A3H bytes from E:\watcom\lib386\os2\clib3r.lib (__stos)
	at offset 00000760 00DCBH bytes from E:\watcom\lib386\os2\clib3r.lib (scnf.c)
	at offset 00001530 00CE4H bytes from E:\watcom\lib386\os2\clib3r.lib (prtf.c)
	at offset 00002214 0004BH bytes from E:\watcom\lib386\os2\clib3r.lib (seterrno.c)
	at offset 00002260 0000EH bytes from E:\watcom\lib386\os2\clib3r.lib (tolower.c)
	at offset 00002270 0004CH bytes from E:\watcom\lib386\os2\clib3r.lib (fdfs386)
	at offset 000022C0 00020H bytes from E:\watcom\lib386\os2\clib3r.lib (strupr.c)
	at offset 000022E0 00008H bytes from E:\watcom\lib386\os2\clib3r.lib (bits.c)
	at offset 000022F0 00042H bytes from E:\watcom\lib386\os2\clib3r.lib (noefgfmt.c)
	at offset 00002332 00128H bytes from E:\watcom\lib386\os2\clib3r.lib (maino32.c)
	at offset 00002460 0002EH bytes from E:\watcom\lib386\os2\clib3r.lib (wctomb.c)
	at offset 00002490 000BCH bytes from E:\watcom\lib386\os2\clib3r.lib (mbtowc.c)
	at offset 00002550 00017H bytes from E:\watcom\lib386\os2\clib3r.lib (mbislead.c)
	at offset 00002570 00074H bytes from E:\watcom\lib386\os2\clib3r.lib (ltoa.c)
	at offset 000025F0 00099H bytes from E:\watcom\lib386\os2\clib3r.lib (lltoa.c)
	at offset 00002690 00074H bytes from E:\watcom\lib386\os2\clib3r.lib (itoa.c)
	at offset 00002710 00070H bytes from E:\watcom\lib386\os2\clib3r.lib (xmsgo32.c)
	at offset 00002780 000B3H bytes from E:\watcom\lib386\os2\clib3r.lib (initrtns.c)
	at offset 00002833 00001H bytes from E:\watcom\lib386\os2\clib3r.lib (crwdata)
	at offset 00002840 0000BH bytes from E:\watcom\lib386\os2\clib3r.lib (cinit.c)
	at offset 0000284B 00132H bytes from E:\watcom\lib386\os2\clib3r.lib (mbinit.c)
	at offset 00002980 00026H bytes from E:\watcom\lib386\os2\clib3r.lib (enterdb.c)

 0003:000E9108 000000000H LASTCODE32             CODE 32-bit

 0004:00000000 000000007H BEGTEXT                CODE 32-bit
	at offset 00000000 00007H bytes from E:\watcom\lib386\os2\clib3r.lib (segdefns)

 0005:00000000 000000030H BSS32                  BSS 32-bit
	at offset 00000000 00004H bytes from F:\src\os2\uniaud32\drv32\bin\Debug.ACP\begin.obj (begin.asm)
	at offset 00000004 0002CH bytes from F:\acpi\lib\acpidrv.lib (acpi)

 0005:00000030 000001724H _BSS                   BSS 32-bit
	at offset 00000000 00008H bytes from F:\src\os2\uniaud32\drv32\bin\Debug.ACP\strategy.obj (F:\src\os2\uniaud32\drv32\strategy.c)
	at offset 00000008 0000CH bytes from F:\src\os2\uniaud32\drv32\bin\Debug.ACP\read.obj (F:\src\os2\uniaud32\drv32\read.cpp)
	at offset 00000014 00008H bytes from F:\src\os2\uniaud32\drv32\bin\Debug.ACP\parse.obj (F:\src\os2\uniaud32\drv32\parse.c)
	at offset 0000001C 00006H bytes from F:\src\os2\uniaud32\drv32\bin\Debug.ACP\idc.obj (F:\src\os2\uniaud32\drv32\idc.c)
	at offset 00000024 0005CH bytes from F:\src\os2\uniaud32\drv32\bin\Debug.ACP\rmhelp.obj (F:\src\os2\uniaud32\drv32\rmhelp.cpp)
	at offset 00000080 00028H bytes from F:\src\os2\uniaud32\lib\Debug.ACP\linuxlib.lib (F:\src\os2\uniaud32\lib32\ossidc.cpp)
	at offset 000000A8 00028H bytes from F:\src\os2\uniaud32\lib\Debug.ACP\linuxlib.lib (F:\src\os2\uniaud32\lib32\debug.c)
	at offset 000000D0 00008H bytes from F:\src\os2\uniaud32\lib\Debug.ACP\linuxlib.lib (F:\src\os2\uniaud32\lib32\memory.cpp)
	at offset 000000D8 00440H bytes from F:\src\os2\uniaud32\lib\Debug.ACP\linuxlib.lib (F:\src\os2\uniaud32\lib32\pci.c)
	at offset 00000518 0002CH bytes from F:\src\os2\uniaud32\lib\Debug.ACP\linuxlib.lib (F:\src\os2\uniaud32\lib32\malloc.cpp)
	at offset 00000544 00004H bytes from F:\src\os2\uniaud32\lib\Debug.ACP\core.lib (F:\src\os2\uniaud32\alsa-kernel\core\hwdep.c)
	at offset 00000548 00004H bytes from F:\src\os2\uniaud32\lib\Debug.ACP\core.lib (F:\src\os2\uniaud32\alsa-kernel\core\timer.c)
	at offset 0000054C 00020H bytes from F:\src\os2\uniaud32\lib\Debug.ACP\core.lib (F:\src\os2\uniaud32\alsa-kernel\core\rawmidi.c)
	at offset 0000056C 00104H bytes from F:\src\os2\uniaud32\lib\Debug.ACP\core.lib (F:\src\os2\uniaud32\alsa-kernel\core\pcm.c)
	at offset 00000670 0040CH bytes from F:\src\os2\uniaud32\lib\Debug.ACP\core.lib (F:\src\os2\uniaud32\alsa-kernel\core\sound.c)
	at offset 00000A7C 00010H bytes from F:\src\os2\uniaud32\lib\Debug.ACP\core.lib (F:\src\os2\uniaud32\alsa-kernel\core\info.c)
	at offset 00000A8C 000C4H bytes from F:\src\os2\uniaud32\lib\Debug.ACP\core.lib (F:\src\os2\uniaud32\alsa-kernel\core\info_oss.c)
	at offset 00000B50 00204H bytes from F:\src\os2\uniaud32\lib\Debug.ACP\core.lib (F:\src\os2\uniaud32\alsa-kernel\core\sound_oss.c)
	at offset 00000D54 00004H bytes from F:\src\os2\uniaud32\lib\Debug.ACP\core.lib (F:\src\os2\uniaud32\alsa-kernel\core\memalloc.c)
	at offset 00000D58 0004CH bytes from F:\src\os2\uniaud32\lib\Debug.ACP\core.lib (F:\src\os2\uniaud32\alsa-kernel\core\init.c)
	at offset 00000DA4 00028H bytes from F:\src\os2\uniaud32\lib\Debug.ACP\pci.lib (F:\src\os2\uniaud32\alsa-kernel\pci\bt87x.c)
	at offset 00000DCC 00004H bytes from F:\src\os2\uniaud32\lib\Debug.ACP\pci.lib (F:\src\os2\uniaud32\alsa-kernel\pci\als4000.c)
	at offset 00000DD0 00024H bytes from F:\src\os2\uniaud32\lib\Debug.ACP\pci.lib (F:\src\os2\uniaud32\alsa-kernel\pci\cmipci.c)
	at offset 00000DF4 00008H bytes from F:\src\os2\uniaud32\lib\Debug.ACP\pci.lib (F:\src\os2\uniaud32\alsa-kernel\pci\atiixp.c)
	at offset 00000DFC 00024H bytes from F:\src\os2\uniaud32\lib\Debug.ACP\pci.lib (F:\src\os2\uniaud32\alsa-kernel\pci\fm801.c)
	at offset 00000E20 00014H bytes from F:\src\os2\uniaud32\lib\Debug.ACP\pci.lib (F:\src\os2\uniaud32\alsa-kernel\pci\via82xx.c)
	at offset 00000E34 00004H bytes from F:\src\os2\uniaud32\lib\Debug.ACP\pci.lib (F:\src\os2\uniaud32\alsa-kernel\pci\maestro3.c)
	at offset 00000E38 00018H bytes from F:\src\os2\uniaud32\lib\Debug.ACP\pci.lib (F:\src\os2\uniaud32\alsa-kernel\pci\intel8x0.c)
	at offset 00000E50 00024H bytes from F:\src\os2\uniaud32\lib\Debug.ACP\pci.lib (F:\src\os2\uniaud32\alsa-kernel\pci\es1968.c)
	at offset 00000E74 00004H bytes from F:\src\os2\uniaud32\lib\Debug.ACP\pci.lib (F:\src\os2\uniaud32\alsa-kernel\pci\es1938.c)
	at offset 00000E78 00024H bytes from F:\src\os2\uniaud32\lib\Debug.ACP\pci.lib (F:\src\os2\uniaud32\alsa-kernel\pci\cs4281.c)
	at offset 00000E9C 00044H bytes from F:\src\os2\uniaud32\lib\Debug.ACP\pci.lib (F:\src\os2\uniaud32\alsa-kernel\pci\ens1371.c)
	at offset 00000EE0 00024H bytes from F:\src\os2\uniaud32\lib\Debug.ACP\ca0106.lib (F:\src\os2\uniaud32\alsa-kernel\pci\ca0106\ca0106_main.c)
	at offset 00000F04 00008H bytes from F:\src\os2\uniaud32\lib\Debug.ACP\hda.lib (F:\src\os2\uniaud32\alsa-kernel\pci\hda\patch_sigmatel.c)
	at offset 00000F0C 00068H bytes from F:\src\os2\uniaud32\lib\Debug.ACP\hda.lib (F:\src\os2\uniaud32\alsa-kernel\pci\hda\hda_intel.c)
	at offset 00000F74 00008H bytes from F:\src\os2\uniaud32\lib\Debug.ACP\sequencer.lib (F:\src\os2\uniaud32\alsa-kernel\core\seq\seq_device.c)
	at offset 00000F7C 0000CH bytes from F:\src\os2\uniaud32\lib\Debug.ACP\sequencer.lib (F:\src\os2\uniaud32\alsa-kernel\core\seq\seq_info.c)
	at offset 00000F88 00024H bytes from F:\src\os2\uniaud32\lib\Debug.ACP\sequencer.lib (F:\src\os2\uniaud32\alsa-kernel\core\seq\seq_queue.c)
	at offset 00000FAC 003C8H bytes from F:\src\os2\uniaud32\lib\Debug.ACP\sequencer.lib (F:\src\os2\uniaud32\alsa-kernel\core\seq\seq_clientmgr.c)
	at offset 00001374 00044H bytes from F:\src\os2\uniaud32\lib\Debug.ACP\cs46xx.lib (F:\src\os2\uniaud32\alsa-kernel\pci\cs46xx\cs46xx.c)
	at offset 000013B8 00008H bytes from F:\src\os2\uniaud32\lib\Debug.ACP\cs5535audio.lib (F:\src\os2\uniaud32\alsa-kernel\pci\cs5535audio\cs5535audio.c)
	at offset 000013C0 00084H bytes from F:\src\os2\uniaud32\lib\Debug.ACP\emu10k1.lib (F:\src\os2\uniaud32\alsa-kernel\pci\emu10k1\emu10k1.c)
	at offset 00001444 00064H bytes from F:\src\os2\uniaud32\lib\Debug.ACP\ymfpci.lib (F:\src\os2\uniaud32\alsa-kernel\pci\ymfpci\ymfpci.c)
	at offset 000014A8 00008H bytes from F:\src\os2\uniaud32\lib\Debug.ACP\ali5451.lib (F:\src\os2\uniaud32\alsa-kernel\pci\ali5451\ali5451.c)
	at offset 000014B0 00004H bytes from F:\src\os2\uniaud32\lib\Debug.ACP\trident.lib (F:\src\os2\uniaud32\alsa-kernel\pci\trident\trident.c)
	at offset 000014B4 0001CH bytes from F:\src\os2\uniaud32\lib\Debug.ACP\nm256.lib (F:\src\os2\uniaud32\alsa-kernel\pci\nm256\nm256.c)
	at offset 000014D0 00020H bytes from F:\src\os2\uniaud32\lib\Debug.ACP\core_oss.lib (F:\src\os2\uniaud32\alsa-kernel\core\oss\pcm_oss.c)
	at offset 000014F0 00106H bytes from E:\watcom\lib386\os2\clib3r.lib (maino32.c)
	at offset 000015F8 00101H bytes from E:\watcom\lib386\os2\clib3r.lib (mbislead.c)
	at offset 000016FC 00004H bytes from E:\watcom\lib386\os2\clib3r.lib (mbisdbcs.c)
	at offset 00001700 00004H bytes from E:\watcom\lib386\os2\clib3r.lib (cinit.c)
	at offset 00001704 00020H bytes from F:\src\os2\uniaud32\lib\Debug.ACP\ac97.lib (F:\src\os2\uniaud32\alsa-kernel\pci\ac97\ac97_codec.c)

 0005:00001754 000000000H C_COMMON               DATA 32-bit

 0005:00001754 000000010H c_common               DATA 32-bit
	at offset 00000000 00010H bytes from F:\acpi\lib\acpidrv.lib (acpi)

 0005:00001764 000000098H DATA32                 DATA 32-bit
	at offset 00000000 0008AH bytes from F:\src\os2\uniaud32\drv32\bin\Debug.ACP\startup.obj (startup.asm)
	at offset 0000008C 0000CH bytes from F:\src\os2\uniaud32\drv32\bin\Debug.ACP\devhlp.obj (devhlp.asm)

 0005:00001800 000061BD8H _DATA                  DATA 32-bit
	at offset 00000000 00080H bytes from F:\src\os2\uniaud32\drv32\bin\Debug.ACP\strategy.obj (F:\src\os2\uniaud32\drv32\strategy.c)
	at offset 00000080 00018H bytes from F:\src\os2\uniaud32\drv32\bin\Debug.ACP\parse.obj (F:\src\os2\uniaud32\drv32\parse.c)
	at offset 00000098 00004H bytes from F:\src\os2\uniaud32\drv32\bin\Debug.ACP\rmhelp.obj (F:\src\os2\uniaud32\drv32\rmhelp.cpp)
	at offset 0000009C 00020H bytes from F:\src\os2\uniaud32\drv32\bin\Debug.ACP\irq.obj (F:\src\os2\uniaud32\drv32\irq.cpp)
	at offset 000000BC 0000CH bytes from F:\src\os2\uniaud32\lib\Debug.ACP\linuxlib.lib (F:\src\os2\uniaud32\lib32\timer.c)
	at offset 000000C8 00028H bytes from F:\src\os2\uniaud32\lib\Debug.ACP\linuxlib.lib (F:\src\os2\uniaud32\lib32\task.c)
	at offset 000000F0 00414H bytes from F:\src\os2\uniaud32\lib\Debug.ACP\linuxlib.lib (F:\src\os2\uniaud32\lib32\misc.c)
	at offset 00000504 00108H bytes from F:\src\os2\uniaud32\lib\Debug.ACP\linuxlib.lib (F:\src\os2\uniaud32\lib32\ossidc.cpp)
	at offset 0000060C 00004H bytes from F:\src\os2\uniaud32\lib\Debug.ACP\linuxlib.lib (F:\src\os2\uniaud32\lib32\soundmidi.c)
	at offset 00000610 001F1H bytes from F:\src\os2\uniaud32\lib\Debug.ACP\linuxlib.lib (F:\src\os2\uniaud32\lib32\soundmixer.c)
	at offset 00000804 061D8H bytes from F:\src\os2\uniaud32\lib\Debug.ACP\linuxlib.lib (F:\src\os2\uniaud32\lib32\sound.c)
	at offset 000069DC 00013H bytes from F:\src\os2\uniaud32\lib\Debug.ACP\linuxlib.lib (F:\src\os2\uniaud32\lib32\debug.c)
	at offset 000069F0 0202CH bytes from F:\src\os2\uniaud32\lib\Debug.ACP\linuxlib.lib (F:\src\os2\uniaud32\lib32\ioctl.c)
	at offset 00008A1C 00880H bytes from F:\src\os2\uniaud32\lib\Debug.ACP\linuxlib.lib (F:\src\os2\uniaud32\lib32\irq.c)
	at offset 0000929C 03F44H bytes from F:\src\os2\uniaud32\lib\Debug.ACP\linuxlib.lib (F:\src\os2\uniaud32\lib32\pci.c)
	at offset 0000D1E0 00004H bytes from F:\src\os2\uniaud32\lib\Debug.ACP\linuxlib.lib (F:\src\os2\uniaud32\lib32\malloc.cpp)
	at offset 0000D1E4 00068H bytes from F:\src\os2\uniaud32\lib\Debug.ACP\core.lib (F:\src\os2\uniaud32\alsa-kernel\core\hwdep.c)
	at offset 0000D24C 000ACH bytes from F:\src\os2\uniaud32\lib\Debug.ACP\core.lib (F:\src\os2\uniaud32\alsa-kernel\core\timer.c)
	at offset 0000D2F8 00090H bytes from F:\src\os2\uniaud32\lib\Debug.ACP\core.lib (F:\src\os2\uniaud32\alsa-kernel\core\rawmidi.c)
	at offset 0000D388 00210H bytes from F:\src\os2\uniaud32\lib\Debug.ACP\core.lib (F:\src\os2\uniaud32\alsa-kernel\core\pcm_misc.c)
	at offset 0000D598 000A0H bytes from F:\src\os2\uniaud32\lib\Debug.ACP\core.lib (F:\src\os2\uniaud32\alsa-kernel\core\pcm_lib.c)
	at offset 0000D638 000E0H bytes from F:\src\os2\uniaud32\lib\Debug.ACP\core.lib (F:\src\os2\uniaud32\alsa-kernel\core\pcm.c)
	at offset 0000D718 0005CH bytes from F:\src\os2\uniaud32\lib\Debug.ACP\core.lib (F:\src\os2\uniaud32\alsa-kernel\core\sound.c)
	at offset 0000D774 00048H bytes from F:\src\os2\uniaud32\lib\Debug.ACP\core.lib (F:\src\os2\uniaud32\alsa-kernel\core\info.c)
	at offset 0000D7BC 00008H bytes from F:\src\os2\uniaud32\lib\Debug.ACP\core.lib (F:\src\os2\uniaud32\alsa-kernel\core\pcm_memory.c)
	at offset 0000D7C4 00030H bytes from F:\src\os2\uniaud32\lib\Debug.ACP\core.lib (F:\src\os2\uniaud32\alsa-kernel\core\pcm_timer.c)
	at offset 0000D7F4 00144H bytes from F:\src\os2\uniaud32\lib\Debug.ACP\core.lib (F:\src\os2\uniaud32\alsa-kernel\core\pcm_native.c)
	at offset 0000D938 0000CH bytes from F:\src\os2\uniaud32\lib\Debug.ACP\core.lib (F:\src\os2\uniaud32\alsa-kernel\core\info_oss.c)
	at offset 0000D944 0000CH bytes from F:\src\os2\uniaud32\lib\Debug.ACP\core.lib (F:\src\os2\uniaud32\alsa-kernel\core\sound_oss.c)
	at offset 0000D950 00060H bytes from F:\src\os2\uniaud32\lib\Debug.ACP\core.lib (F:\src\os2\uniaud32\alsa-kernel\core\control.c)
	at offset 0000D9B0 0001CH bytes from F:\src\os2\uniaud32\lib\Debug.ACP\core.lib (F:\src\os2\uniaud32\alsa-kernel\core\memalloc.c)
	at offset 0000D9CC 00058H bytes from F:\src\os2\uniaud32\lib\Debug.ACP\core.lib (F:\src\os2\uniaud32\alsa-kernel\core\init.c)
	at offset 0000DA24 00264H bytes from F:\src\os2\uniaud32\lib\Debug.ACP\pci.lib (F:\src\os2\uniaud32\alsa-kernel\pci\bt87x.c)
	at offset 0000DC88 00164H bytes from F:\src\os2\uniaud32\lib\Debug.ACP\pci.lib (F:\src\os2\uniaud32\alsa-kernel\pci\als4000.c)
	at offset 0000DDEC 00D81H bytes from F:\src\os2\uniaud32\lib\Debug.ACP\pci.lib (F:\src\os2\uniaud32\alsa-kernel\pci\cmipci.c)
	at offset 0000EB70 0032CH bytes from F:\src\os2\uniaud32\lib\Debug.ACP\pci.lib (F:\src\os2\uniaud32\alsa-kernel\pci\atiixp.c)
	at offset 0000EE9C 0046CH bytes from F:\src\os2\uniaud32\lib\Debug.ACP\pci.lib (F:\src\os2\uniaud32\alsa-kernel\pci\fm801.c)
	at offset 0000F308 00678H bytes from F:\src\os2\uniaud32\lib\Debug.ACP\pci.lib (F:\src\os2\uniaud32\alsa-kernel\pci\via82xx.c)
	at offset 0000F980 00648H bytes from F:\src\os2\uniaud32\lib\Debug.ACP\pci.lib (F:\src\os2\uniaud32\alsa-kernel\pci\maestro3.c)
	at offset 0000FFC8 00D30H bytes from F:\src\os2\uniaud32\lib\Debug.ACP\pci.lib (F:\src\os2\uniaud32\alsa-kernel\pci\intel8x0.c)
	at offset 00010CF8 00244H bytes from F:\src\os2\uniaud32\lib\Debug.ACP\pci.lib (F:\src\os2\uniaud32\alsa-kernel\pci\es1968.c)
	at offset 00010F3C 00861H bytes from F:\src\os2\uniaud32\lib\Debug.ACP\pci.lib (F:\src\os2\uniaud32\alsa-kernel\pci\es1938.c)
	at offset 000117A0 00298H bytes from F:\src\os2\uniaud32\lib\Debug.ACP\pci.lib (F:\src\os2\uniaud32\alsa-kernel\pci\cs4281.c)
	at offset 00011A38 0042CH bytes from F:\src\os2\uniaud32\lib\Debug.ACP\pci.lib (F:\src\os2\uniaud32\alsa-kernel\pci\ens1371.c)
	at offset 00011E64 004B4H bytes from F:\src\os2\uniaud32\lib\Debug.ACP\ca0106.lib (F:\src\os2\uniaud32\alsa-kernel\pci\ca0106\ca0106_main.c)
	at offset 00012318 00020H bytes from F:\src\os2\uniaud32\lib\Debug.ACP\ca0106.lib (F:\src\os2\uniaud32\alsa-kernel\pci\ca0106\ca_midi.c)
	at offset 00012338 00634H bytes from F:\src\os2\uniaud32\lib\Debug.ACP\ca0106.lib (F:\src\os2\uniaud32\alsa-kernel\pci\ca0106\ca0106_mixer.c)
	at offset 0001296C 00058H bytes from F:\src\os2\uniaud32\lib\Debug.ACP\ca0106.lib (F:\src\os2\uniaud32\alsa-kernel\pci\ca0106\ca0106_proc.c)
	at offset 000129C4 029D4H bytes from F:\src\os2\uniaud32\lib\Debug.ACP\hda.lib (F:\src\os2\uniaud32\alsa-kernel\pci\hda\patch_via.c)
	at offset 00015398 027ECH bytes from F:\src\os2\uniaud32\lib\Debug.ACP\hda.lib (F:\src\os2\uniaud32\alsa-kernel\pci\hda\patch_conexant.c)
	at offset 00017B84 00160H bytes from F:\src\os2\uniaud32\lib\Debug.ACP\hda.lib (F:\src\os2\uniaud32\alsa-kernel\pci\hda\patch_atihdmi.c)
	at offset 00017CE4 02AF4H bytes from F:\src\os2\uniaud32\lib\Debug.ACP\hda.lib (F:\src\os2\uniaud32\alsa-kernel\pci\hda\patch_sigmatel.c)
	at offset 0001A7D8 07860H bytes from F:\src\os2\uniaud32\lib\Debug.ACP\hda.lib (F:\src\os2\uniaud32\alsa-kernel\pci\hda\patch_analog.c)
	at offset 00022038 007A4H bytes from F:\src\os2\uniaud32\lib\Debug.ACP\hda.lib (F:\src\os2\uniaud32\alsa-kernel\pci\hda\patch_cmedia.c)
	at offset 000227DC 1F38FH bytes from F:\src\os2\uniaud32\lib\Debug.ACP\hda.lib (F:\src\os2\uniaud32\alsa-kernel\pci\hda\patch_realtek.c)
	at offset 00041B6C 00340H bytes from F:\src\os2\uniaud32\lib\Debug.ACP\hda.lib (F:\src\os2\uniaud32\alsa-kernel\pci\hda\hda_intel.c)
	at offset 00041EAC 00477H bytes from F:\src\os2\uniaud32\lib\Debug.ACP\hda.lib (F:\src\os2\uniaud32\alsa-kernel\pci\hda\hda_codec.c)
	at offset 00042324 00090H bytes from F:\src\os2\uniaud32\lib\Debug.ACP\hda.lib (F:\src\os2\uniaud32\alsa-kernel\pci\hda\hda_generic.c)
	at offset 000423B4 000E0H bytes from F:\src\os2\uniaud32\lib\Debug.ACP\hda.lib (F:\src\os2\uniaud32\alsa-kernel\pci\hda\hda_proc.c)
	at offset 00042494 0005CH bytes from F:\src\os2\uniaud32\lib\Debug.ACP\sequencer.lib (F:\src\os2\uniaud32\alsa-kernel\core\seq\seq.c)
	at offset 000424F0 00028H bytes from F:\src\os2\uniaud32\lib\Debug.ACP\sequencer.lib (F:\src\os2\uniaud32\alsa-kernel\core\seq\seq_device.c)
	at offset 00042518 00008H bytes from F:\src\os2\uniaud32\lib\Debug.ACP\sequencer.lib (F:\src\os2\uniaud32\alsa-kernel\core\seq\seq_system.c)
	at offset 00042520 00004H bytes from F:\src\os2\uniaud32\lib\Debug.ACP\sequencer.lib (F:\src\os2\uniaud32\alsa-kernel\core\seq\seq_queue.c)
	at offset 00042524 00140H bytes from F:\src\os2\uniaud32\lib\Debug.ACP\sequencer.lib (F:\src\os2\uniaud32\alsa-kernel\core\seq\seq_clientmgr.c)
	at offset 00042664 00030H bytes from F:\src\os2\uniaud32\lib\Debug.ACP\opl3.lib (F:\src\os2\uniaud32\alsa-kernel\drivers\opl3\opl3_seq.c)
	at offset 00042694 00074H bytes from F:\src\os2\uniaud32\lib\Debug.ACP\opl3.lib (F:\src\os2\uniaud32\alsa-kernel\drivers\opl3\opl3_lib.c)
	at offset 00042708 000A7H bytes from F:\src\os2\uniaud32\lib\Debug.ACP\opl3.lib (F:\src\os2\uniaud32\alsa-kernel\drivers\opl3\opl3_drums.c)
	at offset 000427B0 000E8H bytes from F:\src\os2\uniaud32\lib\Debug.ACP\opl3.lib (F:\src\os2\uniaud32\alsa-kernel\drivers\opl3\opl3_midi.c)
	at offset 00042898 00024H bytes from F:\src\os2\uniaud32\lib\Debug.ACP\opl3.lib (F:\src\os2\uniaud32\alsa-kernel\drivers\opl3\opl3_synth.c)
	at offset 000428BC 00028H bytes from F:\src\os2\uniaud32\lib\Debug.ACP\mpu401.lib (F:\src\os2\uniaud32\alsa-kernel\drivers\mpu401\mpu401_uart.c)
	at offset 000428E4 000ACH bytes from F:\src\os2\uniaud32\lib\Debug.ACP\cs46xx.lib (F:\src\os2\uniaud32\alsa-kernel\pci\cs46xx\cs46xx.c)
	at offset 00042990 0DBC4H bytes from F:\src\os2\uniaud32\lib\Debug.ACP\cs46xx.lib (F:\src\os2\uniaud32\alsa-kernel\pci\cs46xx\cs46xx_lib.c)
	at offset 00050554 000C4H bytes from F:\src\os2\uniaud32\lib\Debug.ACP\cs5535audio.lib (F:\src\os2\uniaud32\alsa-kernel\pci\cs5535audio\cs5535audio.c)
	at offset 00050618 00110H bytes from F:\src\os2\uniaud32\lib\Debug.ACP\cs5535audio.lib (F:\src\os2\uniaud32\alsa-kernel\pci\cs5535audio\cs5535audio_pcm.c)
	at offset 00050728 000ECH bytes from F:\src\os2\uniaud32\lib\Debug.ACP\emu10k1.lib (F:\src\os2\uniaud32\alsa-kernel\pci\emu10k1\emu10k1.c)
	at offset 00050814 002E8H bytes from F:\src\os2\uniaud32\lib\Debug.ACP\emu10k1.lib (F:\src\os2\uniaud32\alsa-kernel\pci\emu10k1\p16v.c)
	at offset 00050AFC 00030H bytes from F:\src\os2\uniaud32\lib\Debug.ACP\emu10k1.lib (F:\src\os2\uniaud32\alsa-kernel\pci\emu10k1\timer.c)
	at offset 00050B2C 001C0H bytes from F:\src\os2\uniaud32\lib\Debug.ACP\emu10k1.lib (F:\src\os2\uniaud32\alsa-kernel\pci\emu10k1\emufx.c)
	at offset 00050CEC 0169CH bytes from F:\src\os2\uniaud32\lib\Debug.ACP\emu10k1.lib (F:\src\os2\uniaud32\alsa-kernel\pci\emu10k1\emumixer.c)
	at offset 00052388 00334H bytes from F:\src\os2\uniaud32\lib\Debug.ACP\emu10k1.lib (F:\src\os2\uniaud32\alsa-kernel\pci\emu10k1\emupcm.c)
	at offset 000526BC 00020H bytes from F:\src\os2\uniaud32\lib\Debug.ACP\emu10k1.lib (F:\src\os2\uniaud32\alsa-kernel\pci\emu10k1\emumpu401.c)
	at offset 000526DC 00894H bytes from F:\src\os2\uniaud32\lib\Debug.ACP\emu10k1.lib (F:\src\os2\uniaud32\alsa-kernel\pci\emu10k1\emu10k1_main.c)
	at offset 00052F70 00270H bytes from F:\src\os2\uniaud32\lib\Debug.ACP\emu10k1.lib (F:\src\os2\uniaud32\alsa-kernel\pci\emu10k1\emuproc.c)
	at offset 000531E0 00280H bytes from F:\src\os2\uniaud32\lib\Debug.ACP\emu10k1.lib (F:\src\os2\uniaud32\alsa-kernel\pci\emu10k1\io.c)
	at offset 00053460 0008CH bytes from F:\src\os2\uniaud32\lib\Debug.ACP\ymfpci.lib (F:\src\os2\uniaud32\alsa-kernel\pci\ymfpci\ymfpci.c)
	at offset 000534EC 006D8H bytes from F:\src\os2\uniaud32\lib\Debug.ACP\ymfpci.lib (F:\src\os2\uniaud32\alsa-kernel\pci\ymfpci\ymfpci_main.c)
	at offset 00053BC4 002B0H bytes from F:\src\os2\uniaud32\lib\Debug.ACP\ali5451.lib (F:\src\os2\uniaud32\alsa-kernel\pci\ali5451\ali5451.c)
	at offset 00053E74 000CCH bytes from F:\src\os2\uniaud32\lib\Debug.ACP\trident.lib (F:\src\os2\uniaud32\alsa-kernel\pci\trident\trident.c)
	at offset 00053F40 004ECH bytes from F:\src\os2\uniaud32\lib\Debug.ACP\trident.lib (F:\src\os2\uniaud32\alsa-kernel\pci\trident\trident_main.c)
	at offset 0005442C 0C7ACH bytes from F:\src\os2\uniaud32\lib\Debug.ACP\nm256.lib (F:\src\os2\uniaud32\alsa-kernel\pci\nm256\nm256.c)
	at offset 00060BD8 004B8H bytes from F:\src\os2\uniaud32\lib\Debug.ACP\sb.lib (F:\src\os2\uniaud32\alsa-kernel\isa\sb\sb_mixer.c)
	at offset 00061090 00014H bytes from F:\src\os2\uniaud32\lib\Debug.ACP\sb.lib (F:\src\os2\uniaud32\alsa-kernel\isa\sb\sb_common.c)
	at offset 000610A4 00080H bytes from F:\src\os2\uniaud32\lib\Debug.ACP\core_oss.lib (F:\src\os2\uniaud32\alsa-kernel\core\oss\pcm_oss.c)
	at offset 00061124 0008CH bytes from E:\watcom\lib386\os2\clib3r.lib (strtol.c)
	at offset 000611B0 00008H bytes from E:\watcom\lib386\os2\clib3r.lib (noefgfmt.c)
	at offset 000611B8 00040H bytes from E:\watcom\lib386\os2\clib3r.lib (maino32.c)
	at offset 000611F8 0004AH bytes from E:\watcom\lib386\os2\clib3r.lib (crwdata)
	at offset 00061244 00004H bytes from E:\watcom\lib386\os2\clib3r.lib (mbinit.c)
	at offset 00061248 00001H bytes from E:\watcom\lib386\os2\clib3r.lib (enterdb.c)
	at offset 0006124C 00004H bytes from E:\watcom\lib386\os2\clib3r.lib (amblksiz.c)
	at offset 00061250 00051H bytes from F:\src\os2\uniaud32\lib\Debug.ACP\ac97.lib (F:\src\os2\uniaud32\alsa-kernel\pci\ac97\ac97_pcm.c)
	at offset 000612A4 00802H bytes from F:\src\os2\uniaud32\lib\Debug.ACP\ac97.lib (F:\src\os2\uniaud32\alsa-kernel\pci\ac97\ac97_codec.c)
	at offset 00061AA8 00110H bytes from F:\src\os2\uniaud32\lib\Debug.ACP\ac97.lib (F:\src\os2\uniaud32\alsa-kernel\pci\ac97\ac97_proc.c)
	at offset 00061BB8 00018H bytes from F:\src\os2\uniaud32\lib\Debug.ACP\sequencer.lib (F:\src\os2\uniaud32\alsa-kernel\core\seq\seq_midi_emul.c)
	at offset 00061BD0 00008H bytes from F:\src\os2\uniaud32\lib\Debug.ACP\synth.lib (F:\src\os2\uniaud32\alsa-kernel\synth\util_mem.c)

 0005:000633D8 0000159E9H CONST                  DATA 32-bit
	at offset 00000000 00013H bytes from F:\src\os2\uniaud32\drv32\bin\Debug.ACP\strategy.obj (F:\src\os2\uniaud32\drv32\strategy.c)
	at offset 00000013 0003EH bytes from F:\src\os2\uniaud32\drv32\bin\Debug.ACP\init.obj (F:\src\os2\uniaud32\drv32\init.c)
	at offset 00000051 00073H bytes from F:\src\os2\uniaud32\drv32\bin\Debug.ACP\parse.obj (F:\src\os2\uniaud32\drv32\parse.c)
	at offset 000000C4 00012H bytes from F:\src\os2\uniaud32\drv32\bin\Debug.ACP\idc.obj (F:\src\os2\uniaud32\drv32\idc.c)
	at offset 000000D6 00096H bytes from F:\src\os2\uniaud32\drv32\bin\Debug.ACP\dispatch.obj (F:\src\os2\uniaud32\drv32\dispatch.c)
	at offset 0000016C 001CCH bytes from F:\src\os2\uniaud32\drv32\bin\Debug.ACP\rmhelp.obj (F:\src\os2\uniaud32\drv32\rmhelp.cpp)
	at offset 00000338 00081H bytes from F:\src\os2\uniaud32\drv32\bin\Debug.ACP\irq.obj (F:\src\os2\uniaud32\drv32\irq.cpp)
	at offset 000003BC 00029H bytes from F:\src\os2\uniaud32\lib\Debug.ACP\linuxlib.lib (F:\src\os2\uniaud32\lib32\vsprintf.c)
	at offset 000003E8 0001FH bytes from F:\src\os2\uniaud32\lib\Debug.ACP\linuxlib.lib (F:\src\os2\uniaud32\lib32\timer.c)
	at offset 00000408 00054H bytes from F:\src\os2\uniaud32\lib\Debug.ACP\linuxlib.lib (F:\src\os2\uniaud32\lib32\misc.c)
	at offset 0000045C 000C2H bytes from F:\src\os2\uniaud32\lib\Debug.ACP\linuxlib.lib (F:\src\os2\uniaud32\lib32\ossidc.cpp)
	at offset 00000520 001C8H bytes from F:\src\os2\uniaud32\lib\Debug.ACP\linuxlib.lib (F:\src\os2\uniaud32\lib32\soundmidi.c)
	at offset 000006E8 0028FH bytes from F:\src\os2\uniaud32\lib\Debug.ACP\linuxlib.lib (F:\src\os2\uniaud32\lib32\soundmixer.c)
	at offset 00000978 00809H bytes from F:\src\os2\uniaud32\lib\Debug.ACP\linuxlib.lib (F:\src\os2\uniaud32\lib32\sound.c)
	at offset 00001184 0002EH bytes from F:\src\os2\uniaud32\lib\Debug.ACP\linuxlib.lib (F:\src\os2\uniaud32\lib32\debug.c)
	at offset 000011B2 000DEH bytes from F:\src\os2\uniaud32\lib\Debug.ACP\linuxlib.lib (F:\src\os2\uniaud32\lib32\memory.cpp)
	at offset 00001290 00195H bytes from F:\src\os2\uniaud32\lib\Debug.ACP\linuxlib.lib (F:\src\os2\uniaud32\lib32\ioctl.c)
	at offset 00001428 0009AH bytes from F:\src\os2\uniaud32\lib\Debug.ACP\linuxlib.lib (F:\src\os2\uniaud32\lib32\irq.c)
	at offset 000014C4 0032EH bytes from F:\src\os2\uniaud32\lib\Debug.ACP\linuxlib.lib (F:\src\os2\uniaud32\lib32\pci.c)
	at offset 000017F2 001FDH bytes from F:\src\os2\uniaud32\lib\Debug.ACP\linuxlib.lib (F:\src\os2\uniaud32\lib32\malloc.cpp)
	at offset 000019F0 0006AH bytes from F:\src\os2\uniaud32\lib\Debug.ACP\linuxlib.lib (F:\src\os2\uniaud32\lib32\waitqueue.c)
	at offset 00001A5C 00109H bytes from F:\src\os2\uniaud32\lib\Debug.ACP\core.lib (F:\src\os2\uniaud32\alsa-kernel\core\hwdep.c)
	at offset 00001B68 00166H bytes from F:\src\os2\uniaud32\lib\Debug.ACP\core.lib (F:\src\os2\uniaud32\alsa-kernel\core\timer.c)
	at offset 00001CD0 00313H bytes from F:\src\os2\uniaud32\lib\Debug.ACP\core.lib (F:\src\os2\uniaud32\alsa-kernel\core\rawmidi.c)
	at offset 00001FE4 000A3H bytes from F:\src\os2\uniaud32\lib\Debug.ACP\core.lib (F:\src\os2\uniaud32\alsa-kernel\core\pcm_lib.c)
	at offset 00002088 001FCH bytes from F:\src\os2\uniaud32\lib\Debug.ACP\core.lib (F:\src\os2\uniaud32\alsa-kernel\core\pcm.c)
	at offset 00002284 000DEH bytes from F:\src\os2\uniaud32\lib\Debug.ACP\core.lib (F:\src\os2\uniaud32\alsa-kernel\core\sound.c)
	at offset 00002364 000B4H bytes from F:\src\os2\uniaud32\lib\Debug.ACP\core.lib (F:\src\os2\uniaud32\alsa-kernel\core\info.c)
	at offset 00002418 0006AH bytes from F:\src\os2\uniaud32\lib\Debug.ACP\core.lib (F:\src\os2\uniaud32\alsa-kernel\core\pcm_timer.c)
	at offset 00002484 000C4H bytes from F:\src\os2\uniaud32\lib\Debug.ACP\core.lib (F:\src\os2\uniaud32\alsa-kernel\core\pcm_native.c)
	at offset 00002548 000F2H bytes from F:\src\os2\uniaud32\lib\Debug.ACP\core.lib (F:\src\os2\uniaud32\alsa-kernel\core\info_oss.c)
	at offset 0000263C 00068H bytes from F:\src\os2\uniaud32\lib\Debug.ACP\core.lib (F:\src\os2\uniaud32\alsa-kernel\core\sound_oss.c)
	at offset 000026A4 000BDH bytes from F:\src\os2\uniaud32\lib\Debug.ACP\core.lib (F:\src\os2\uniaud32\alsa-kernel\core\device.c)
	at offset 00002764 0011DH bytes from F:\src\os2\uniaud32\lib\Debug.ACP\core.lib (F:\src\os2\uniaud32\alsa-kernel\core\control.c)
	at offset 00002884 0007EH bytes from F:\src\os2\uniaud32\lib\Debug.ACP\core.lib (F:\src\os2\uniaud32\alsa-kernel\core\memalloc.c)
	at offset 00002904 0022FH bytes from F:\src\os2\uniaud32\lib\Debug.ACP\core.lib (F:\src\os2\uniaud32\alsa-kernel\core\init.c)
	at offset 00002B34 00020H bytes from F:\src\os2\uniaud32\lib\Debug.ACP\core.lib (F:\src\os2\uniaud32\alsa-kernel\core\sgbuf.c)
	at offset 00002B54 00339H bytes from F:\src\os2\uniaud32\lib\Debug.ACP\pci.lib (F:\src\os2\uniaud32\alsa-kernel\pci\bt87x.c)
	at offset 00002E90 00103H bytes from F:\src\os2\uniaud32\lib\Debug.ACP\pci.lib (F:\src\os2\uniaud32\alsa-kernel\pci\als4000.c)
	at offset 00002F94 00578H bytes from F:\src\os2\uniaud32\lib\Debug.ACP\pci.lib (F:\src\os2\uniaud32\alsa-kernel\pci\cmipci.c)
	at offset 0000350C 00291H bytes from F:\src\os2\uniaud32\lib\Debug.ACP\pci.lib (F:\src\os2\uniaud32\alsa-kernel\pci\atiixp.c)
	at offset 000037A0 0027EH bytes from F:\src\os2\uniaud32\lib\Debug.ACP\pci.lib (F:\src\os2\uniaud32\alsa-kernel\pci\fm801.c)
	at offset 00003A20 00651H bytes from F:\src\os2\uniaud32\lib\Debug.ACP\pci.lib (F:\src\os2\uniaud32\alsa-kernel\pci\via82xx.c)
	at offset 00004074 00267H bytes from F:\src\os2\uniaud32\lib\Debug.ACP\pci.lib (F:\src\os2\uniaud32\alsa-kernel\pci\maestro3.c)
	at offset 000042DC 00A94H bytes from F:\src\os2\uniaud32\lib\Debug.ACP\pci.lib (F:\src\os2\uniaud32\alsa-kernel\pci\intel8x0.c)
	at offset 00004D70 002FBH bytes from F:\src\os2\uniaud32\lib\Debug.ACP\pci.lib (F:\src\os2\uniaud32\alsa-kernel\pci\es1968.c)
	at offset 0000506C 00422H bytes from F:\src\os2\uniaud32\lib\Debug.ACP\pci.lib (F:\src\os2\uniaud32\alsa-kernel\pci\es1938.c)
	at offset 00005490 002CBH bytes from F:\src\os2\uniaud32\lib\Debug.ACP\pci.lib (F:\src\os2\uniaud32\alsa-kernel\pci\cs4281.c)
	at offset 0000575C 00266H bytes from F:\src\os2\uniaud32\lib\Debug.ACP\pci.lib (F:\src\os2\uniaud32\alsa-kernel\pci\ens1371.c)
	at offset 000059C4 00301H bytes from F:\src\os2\uniaud32\lib\Debug.ACP\ca0106.lib (F:\src\os2\uniaud32\alsa-kernel\pci\ca0106\ca0106_main.c)
	at offset 00005CC8 00045H bytes from F:\src\os2\uniaud32\lib\Debug.ACP\ca0106.lib (F:\src\os2\uniaud32\alsa-kernel\pci\ca0106\ca_midi.c)
	at offset 00005D10 0067DH bytes from F:\src\os2\uniaud32\lib\Debug.ACP\ca0106.lib (F:\src\os2\uniaud32\alsa-kernel\pci\ca0106\ca0106_mixer.c)
	at offset 00006390 003C4H bytes from F:\src\os2\uniaud32\lib\Debug.ACP\ca0106.lib (F:\src\os2\uniaud32\alsa-kernel\pci\ca0106\ca0106_proc.c)
	at offset 00006754 00560H bytes from F:\src\os2\uniaud32\lib\Debug.ACP\hda.lib (F:\src\os2\uniaud32\alsa-kernel\pci\hda\patch_via.c)
	at offset 00006CB4 007E0H bytes from F:\src\os2\uniaud32\lib\Debug.ACP\hda.lib (F:\src\os2\uniaud32\alsa-kernel\pci\hda\patch_conexant.c)
	at offset 00007494 00048H bytes from F:\src\os2\uniaud32\lib\Debug.ACP\hda.lib (F:\src\os2\uniaud32\alsa-kernel\pci\hda\patch_atihdmi.c)
	at offset 000074DC 00F6AH bytes from F:\src\os2\uniaud32\lib\Debug.ACP\hda.lib (F:\src\os2\uniaud32\alsa-kernel\pci\hda\patch_sigmatel.c)
	at offset 00008448 00A51H bytes from F:\src\os2\uniaud32\lib\Debug.ACP\hda.lib (F:\src\os2\uniaud32\alsa-kernel\pci\hda\patch_analog.c)
	at offset 00008E9C 001A9H bytes from F:\src\os2\uniaud32\lib\Debug.ACP\hda.lib (F:\src\os2\uniaud32\alsa-kernel\pci\hda\patch_cmedia.c)
	at offset 00009048 021E3H bytes from F:\src\os2\uniaud32\lib\Debug.ACP\hda.lib (F:\src\os2\uniaud32\alsa-kernel\pci\hda\patch_realtek.c)
	at offset 0000B22C 0099BH bytes from F:\src\os2\uniaud32\lib\Debug.ACP\hda.lib (F:\src\os2\uniaud32\alsa-kernel\pci\hda\hda_intel.c)
	at offset 0000BBC8 00995H bytes from F:\src\os2\uniaud32\lib\Debug.ACP\hda.lib (F:\src\os2\uniaud32\alsa-kernel\pci\hda\hda_codec.c)
	at offset 0000C560 0000DH bytes from F:\src\os2\uniaud32\lib\Debug.ACP\hda.lib (F:\src\os2\uniaud32\alsa-kernel\pci\hda\hda_hwdep.c)
	at offset 0000C570 002C1H bytes from F:\src\os2\uniaud32\lib\Debug.ACP\hda.lib (F:\src\os2\uniaud32\alsa-kernel\pci\hda\hda_generic.c)
	at offset 0000C834 00784H bytes from F:\src\os2\uniaud32\lib\Debug.ACP\hda.lib (F:\src\os2\uniaud32\alsa-kernel\pci\hda\hda_proc.c)
	at offset 0000CFB8 00163H bytes from F:\src\os2\uniaud32\lib\Debug.ACP\sequencer.lib (F:\src\os2\uniaud32\alsa-kernel\core\seq\seq_device.c)
	at offset 0000D11C 00015H bytes from F:\src\os2\uniaud32\lib\Debug.ACP\sequencer.lib (F:\src\os2\uniaud32\alsa-kernel\core\seq\seq_info.c)
	at offset 0000D134 00016H bytes from F:\src\os2\uniaud32\lib\Debug.ACP\sequencer.lib (F:\src\os2\uniaud32\alsa-kernel\core\seq\seq_system.c)
	at offset 0000D14C 00156H bytes from F:\src\os2\uniaud32\lib\Debug.ACP\sequencer.lib (F:\src\os2\uniaud32\alsa-kernel\core\seq\seq_queue.c)
	at offset 0000D2A4 0013AH bytes from F:\src\os2\uniaud32\lib\Debug.ACP\sequencer.lib (F:\src\os2\uniaud32\alsa-kernel\core\seq\seq_memory.c)
	at offset 0000D3E0 001FBH bytes from F:\src\os2\uniaud32\lib\Debug.ACP\sequencer.lib (F:\src\os2\uniaud32\alsa-kernel\core\seq\seq_clientmgr.c)
	at offset 0000D5DC 00060H bytes from F:\src\os2\uniaud32\lib\Debug.ACP\sequencer.lib (F:\src\os2\uniaud32\alsa-kernel\core\seq\seq_ports.c)
	at offset 0000D63C 00127H bytes from F:\src\os2\uniaud32\lib\Debug.ACP\sequencer.lib (F:\src\os2\uniaud32\alsa-kernel\core\seq\seq_timer.c)
	at offset 0000D764 000C3H bytes from F:\src\os2\uniaud32\lib\Debug.ACP\sequencer.lib (F:\src\os2\uniaud32\alsa-kernel\core\seq\seq_prioq.c)
	at offset 0000D828 00047H bytes from F:\src\os2\uniaud32\lib\Debug.ACP\sequencer.lib (F:\src\os2\uniaud32\alsa-kernel\core\seq\seq_fifo.c)
	at offset 0000D870 00028H bytes from F:\src\os2\uniaud32\lib\Debug.ACP\opl3.lib (F:\src\os2\uniaud32\alsa-kernel\drivers\opl3\opl3_seq.c)
	at offset 0000D898 0014DH bytes from F:\src\os2\uniaud32\lib\Debug.ACP\opl3.lib (F:\src\os2\uniaud32\alsa-kernel\drivers\opl3\opl3_lib.c)
	at offset 0000D9E8 0000FH bytes from F:\src\os2\uniaud32\lib\Debug.ACP\opl3.lib (F:\src\os2\uniaud32\alsa-kernel\drivers\opl3\opl3_synth.c)
	at offset 0000D9F8 000E6H bytes from F:\src\os2\uniaud32\lib\Debug.ACP\mpu401.lib (F:\src\os2\uniaud32\alsa-kernel\drivers\mpu401\mpu401_uart.c)
	at offset 0000DAE0 00035H bytes from F:\src\os2\uniaud32\lib\Debug.ACP\cs46xx.lib (F:\src\os2\uniaud32\alsa-kernel\pci\cs46xx\cs46xx.c)
	at offset 0000DB18 005A3H bytes from F:\src\os2\uniaud32\lib\Debug.ACP\cs46xx.lib (F:\src\os2\uniaud32\alsa-kernel\pci\cs46xx\cs46xx_lib.c)
	at offset 0000E0BC 00129H bytes from F:\src\os2\uniaud32\lib\Debug.ACP\cs5535audio.lib (F:\src\os2\uniaud32\alsa-kernel\pci\cs5535audio\cs5535audio.c)
	at offset 0000E1E8 000C2H bytes from F:\src\os2\uniaud32\lib\Debug.ACP\cs5535audio.lib (F:\src\os2\uniaud32\alsa-kernel\pci\cs5535audio\cs5535audio_pm.c)
	at offset 0000E2AC 0005CH bytes from F:\src\os2\uniaud32\lib\Debug.ACP\cs5535audio.lib (F:\src\os2\uniaud32\alsa-kernel\pci\cs5535audio\cs5535audio_pcm.c)
	at offset 0000E308 000BBH bytes from F:\src\os2\uniaud32\lib\Debug.ACP\emu10k1.lib (F:\src\os2\uniaud32\alsa-kernel\pci\emu10k1\emu10k1.c)
	at offset 0000E3C4 00189H bytes from F:\src\os2\uniaud32\lib\Debug.ACP\emu10k1.lib (F:\src\os2\uniaud32\alsa-kernel\pci\emu10k1\p16v.c)
	at offset 0000E550 00016H bytes from F:\src\os2\uniaud32\lib\Debug.ACP\emu10k1.lib (F:\src\os2\uniaud32\alsa-kernel\pci\emu10k1\timer.c)
	at offset 0000E568 00B47H bytes from F:\src\os2\uniaud32\lib\Debug.ACP\emu10k1.lib (F:\src\os2\uniaud32\alsa-kernel\pci\emu10k1\emufx.c)
	at offset 0000F0B0 01071H bytes from F:\src\os2\uniaud32\lib\Debug.ACP\emu10k1.lib (F:\src\os2\uniaud32\alsa-kernel\pci\emu10k1\emumixer.c)
	at offset 00010124 000B8H bytes from F:\src\os2\uniaud32\lib\Debug.ACP\emu10k1.lib (F:\src\os2\uniaud32\alsa-kernel\pci\emu10k1\emupcm.c)
	at offset 000101DC 00082H bytes from F:\src\os2\uniaud32\lib\Debug.ACP\emu10k1.lib (F:\src\os2\uniaud32\alsa-kernel\pci\emu10k1\emumpu401.c)
	at offset 00010260 007C9H bytes from F:\src\os2\uniaud32\lib\Debug.ACP\emu10k1.lib (F:\src\os2\uniaud32\alsa-kernel\pci\emu10k1\emu10k1_main.c)
	at offset 00010A2C 00831H bytes from F:\src\os2\uniaud32\lib\Debug.ACP\emu10k1.lib (F:\src\os2\uniaud32\alsa-kernel\pci\emu10k1\emuproc.c)
	at offset 00011260 0009CH bytes from F:\src\os2\uniaud32\lib\Debug.ACP\emu10k1.lib (F:\src\os2\uniaud32\alsa-kernel\pci\emu10k1\io.c)
	at offset 000112FC 0008CH bytes from F:\src\os2\uniaud32\lib\Debug.ACP\emu10k1.lib (F:\src\os2\uniaud32\alsa-kernel\pci\emu10k1\memory.c)
	at offset 00011388 000C9H bytes from F:\src\os2\uniaud32\lib\Debug.ACP\emu10k1.lib (F:\src\os2\uniaud32\alsa-kernel\pci\emu10k1\irq.c)
	at offset 00011454 00128H bytes from F:\src\os2\uniaud32\lib\Debug.ACP\ymfpci.lib (F:\src\os2\uniaud32\alsa-kernel\pci\ymfpci\ymfpci.c)
	at offset 0001157C 00374H bytes from F:\src\os2\uniaud32\lib\Debug.ACP\ymfpci.lib (F:\src\os2\uniaud32\alsa-kernel\pci\ymfpci\ymfpci_main.c)
	at offset 000118F0 0044CH bytes from F:\src\os2\uniaud32\lib\Debug.ACP\ali5451.lib (F:\src\os2\uniaud32\alsa-kernel\pci\ali5451\ali5451.c)
	at offset 00011D3C 00068H bytes from F:\src\os2\uniaud32\lib\Debug.ACP\trident.lib (F:\src\os2\uniaud32\alsa-kernel\pci\trident\trident.c)
	at offset 00011DA4 00442H bytes from F:\src\os2\uniaud32\lib\Debug.ACP\trident.lib (F:\src\os2\uniaud32\alsa-kernel\pci\trident\trident_main.c)
	at offset 000121E8 00035H bytes from F:\src\os2\uniaud32\lib\Debug.ACP\trident.lib (F:\src\os2\uniaud32\alsa-kernel\pci\trident\trident_memory.c)
	at offset 00012220 0043FH bytes from F:\src\os2\uniaud32\lib\Debug.ACP\nm256.lib (F:\src\os2\uniaud32\alsa-kernel\pci\nm256\nm256.c)
	at offset 00012660 0036EH bytes from F:\src\os2\uniaud32\lib\Debug.ACP\sb.lib (F:\src\os2\uniaud32\alsa-kernel\isa\sb\sb_mixer.c)
	at offset 000129D0 00187H bytes from F:\src\os2\uniaud32\lib\Debug.ACP\sb.lib (F:\src\os2\uniaud32\alsa-kernel\isa\sb\sb_common.c)
	at offset 00012B58 00247H bytes from F:\src\os2\uniaud32\lib\Debug.ACP\core_oss.lib (F:\src\os2\uniaud32\alsa-kernel\core\oss\pcm_oss.c)
	at offset 00012DA0 00025H bytes from E:\watcom\lib386\os2\clib3r.lib (alphabet.c)
	at offset 00012DC8 000E3H bytes from F:\src\os2\uniaud32\lib\Debug.ACP\linuxlib.lib (F:\src\os2\uniaud32\lib32\semaphore.c)
	at offset 00012EAC 0001AH bytes from F:\src\os2\uniaud32\lib\Debug.ACP\core.lib (F:\src\os2\uniaud32\alsa-kernel\core\vmaster.c)
	at offset 00012EC8 0008CH bytes from F:\src\os2\uniaud32\lib\Debug.ACP\ac97.lib (F:\src\os2\uniaud32\alsa-kernel\pci\ac97\ac97_pcm.c)
	at offset 00012F54 01E46H bytes from F:\src\os2\uniaud32\lib\Debug.ACP\ac97.lib (F:\src\os2\uniaud32\alsa-kernel\pci\ac97\ac97_codec.c)
	at offset 00014D9C 00BFFH bytes from F:\src\os2\uniaud32\lib\Debug.ACP\ac97.lib (F:\src\os2\uniaud32\alsa-kernel\pci\ac97\ac97_proc.c)
	at offset 0001599C 0004DH bytes from F:\src\os2\uniaud32\lib\Debug.ACP\sequencer.lib (F:\src\os2\uniaud32\alsa-kernel\core\seq\seq_midi_emul.c)

 0005:00078DD0 000006762H CONST2                 DATA 32-bit
	at offset 00000000 00183H bytes from F:\src\os2\uniaud32\drv32\bin\Debug.ACP\init.obj (F:\src\os2\uniaud32\drv32\init.c)
	at offset 00000184 00040H bytes from F:\src\os2\uniaud32\lib\Debug.ACP\core.lib (F:\src\os2\uniaud32\alsa-kernel\core\info.c)
	at offset 000001C4 00004H bytes from F:\src\os2\uniaud32\lib\Debug.ACP\core.lib (F:\src\os2\uniaud32\alsa-kernel\core\pcm_memory.c)
	at offset 000001C8 0000CH bytes from F:\src\os2\uniaud32\lib\Debug.ACP\core.lib (F:\src\os2\uniaud32\alsa-kernel\core\pcm_native.c)
	at offset 000001D4 001C0H bytes from F:\src\os2\uniaud32\lib\Debug.ACP\pci.lib (F:\src\os2\uniaud32\alsa-kernel\pci\bt87x.c)
	at offset 00000394 00060H bytes from F:\src\os2\uniaud32\lib\Debug.ACP\pci.lib (F:\src\os2\uniaud32\alsa-kernel\pci\als4000.c)
	at offset 000003F4 00100H bytes from F:\src\os2\uniaud32\lib\Debug.ACP\pci.lib (F:\src\os2\uniaud32\alsa-kernel\pci\cmipci.c)
	at offset 000004F4 0008CH bytes from F:\src\os2\uniaud32\lib\Debug.ACP\pci.lib (F:\src\os2\uniaud32\alsa-kernel\pci\atiixp.c)
	at offset 00000580 00064H bytes from F:\src\os2\uniaud32\lib\Debug.ACP\pci.lib (F:\src\os2\uniaud32\alsa-kernel\pci\fm801.c)
	at offset 000005E4 00064H bytes from F:\src\os2\uniaud32\lib\Debug.ACP\pci.lib (F:\src\os2\uniaud32\alsa-kernel\pci\via82xx.c)
	at offset 00000648 001B8H bytes from F:\src\os2\uniaud32\lib\Debug.ACP\pci.lib (F:\src\os2\uniaud32\alsa-kernel\pci\maestro3.c)
	at offset 00000800 002A0H bytes from F:\src\os2\uniaud32\lib\Debug.ACP\pci.lib (F:\src\os2\uniaud32\alsa-kernel\pci\intel8x0.c)
	at offset 00000AA0 00070H bytes from F:\src\os2\uniaud32\lib\Debug.ACP\pci.lib (F:\src\os2\uniaud32\alsa-kernel\pci\es1968.c)
	at offset 00000B10 00048H bytes from F:\src\os2\uniaud32\lib\Debug.ACP\pci.lib (F:\src\os2\uniaud32\alsa-kernel\pci\es1938.c)
	at offset 00000B58 00048H bytes from F:\src\os2\uniaud32\lib\Debug.ACP\pci.lib (F:\src\os2\uniaud32\alsa-kernel\pci\cs4281.c)
	at offset 00000BA0 00080H bytes from F:\src\os2\uniaud32\lib\Debug.ACP\pci.lib (F:\src\os2\uniaud32\alsa-kernel\pci\ens1371.c)
	at offset 00000C20 00058H bytes from F:\src\os2\uniaud32\lib\Debug.ACP\ca0106.lib (F:\src\os2\uniaud32\alsa-kernel\pci\ca0106\ca0106_main.c)
	at offset 00000C78 00020H bytes from F:\src\os2\uniaud32\lib\Debug.ACP\ca0106.lib (F:\src\os2\uniaud32\alsa-kernel\pci\ca0106\ca0106_mixer.c)
	at offset 00000C98 00108H bytes from F:\src\os2\uniaud32\lib\Debug.ACP\hda.lib (F:\src\os2\uniaud32\alsa-kernel\pci\hda\patch_conexant.c)
	at offset 00000DA0 00068H bytes from F:\src\os2\uniaud32\lib\Debug.ACP\hda.lib (F:\src\os2\uniaud32\alsa-kernel\pci\hda\patch_realtek.c)
	at offset 00000E08 00428H bytes from F:\src\os2\uniaud32\lib\Debug.ACP\hda.lib (F:\src\os2\uniaud32\alsa-kernel\pci\hda\hda_intel.c)
	at offset 00001230 00070H bytes from F:\src\os2\uniaud32\lib\Debug.ACP\cs46xx.lib (F:\src\os2\uniaud32\alsa-kernel\pci\cs46xx\cs46xx.c)
	at offset 000012A0 00054H bytes from F:\src\os2\uniaud32\lib\Debug.ACP\cs5535audio.lib (F:\src\os2\uniaud32\alsa-kernel\pci\cs5535audio\cs5535audio.c)
	at offset 000012F4 00070H bytes from F:\src\os2\uniaud32\lib\Debug.ACP\emu10k1.lib (F:\src\os2\uniaud32\alsa-kernel\pci\emu10k1\emu10k1.c)
	at offset 00001364 00010H bytes from F:\src\os2\uniaud32\lib\Debug.ACP\emu10k1.lib (F:\src\os2\uniaud32\alsa-kernel\pci\emu10k1\p16v.c)
	at offset 00001374 00814H bytes from F:\src\os2\uniaud32\lib\Debug.ACP\emu10k1.lib (F:\src\os2\uniaud32\alsa-kernel\pci\emu10k1\emufx.c)
	at offset 00001B88 00010H bytes from F:\src\os2\uniaud32\lib\Debug.ACP\emu10k1.lib (F:\src\os2\uniaud32\alsa-kernel\pci\emu10k1\emumixer.c)
	at offset 00001B98 000C4H bytes from F:\src\os2\uniaud32\lib\Debug.ACP\ymfpci.lib (F:\src\os2\uniaud32\alsa-kernel\pci\ymfpci\ymfpci.c)
	at offset 00001C5C 00010H bytes from F:\src\os2\uniaud32\lib\Debug.ACP\ymfpci.lib (F:\src\os2\uniaud32\alsa-kernel\pci\ymfpci\ymfpci_main.c)
	at offset 00001C6C 00038H bytes from F:\src\os2\uniaud32\lib\Debug.ACP\ali5451.lib (F:\src\os2\uniaud32\alsa-kernel\pci\ali5451\ali5451.c)
	at offset 00001CA4 00070H bytes from F:\src\os2\uniaud32\lib\Debug.ACP\trident.lib (F:\src\os2\uniaud32\alsa-kernel\pci\trident\trident.c)
	at offset 00001D14 00020H bytes from F:\src\os2\uniaud32\lib\Debug.ACP\trident.lib (F:\src\os2\uniaud32\alsa-kernel\pci\trident\trident_main.c)
	at offset 00001D34 00070H bytes from F:\src\os2\uniaud32\lib\Debug.ACP\nm256.lib (F:\src\os2\uniaud32\alsa-kernel\pci\nm256\nm256.c)
	at offset 00001DA4 00018H bytes from F:\src\os2\uniaud32\lib\Debug.ACP\ac97.lib (F:\src\os2\uniaud32\alsa-kernel\pci\ac97\ac97_pcm.c)
	at offset 00001DBC 049A6H bytes from F:\src\os2\uniaud32\lib\Debug.ACP\ac97.lib (F:\src\os2\uniaud32\alsa-kernel\pci\ac97\ac97_codec.c)

 0005:0007F534 000000004H LASTDATA32             DATA 32-bit
	at offset 00000000 00004H bytes from F:\src\os2\uniaud32\drv32\bin\Debug.ACP\end.obj (end.asm)

 0005:0007F538 000000000H XIB                    DATA 32-bit

 0005:0007F538 000000006H XI                     DATA 32-bit
	at offset 00000000 00006H bytes from E:\watcom\lib386\os2\clib3r.lib (mbislead.c)

 0005:0007F53E 000000000H XIE                    DATA 32-bit

 0005:0007F53E 000000000H TIB                    DATA 32-bit

 0005:0007F53E 000000000H TI                     DATA 32-bit

 0005:0007F53E 000000000H TIE                    DATA 32-bit

 0005:0007F53E 000000000H YIB                    DATA 32-bit

 0005:0007F53E 000000000H YI                     DATA 32-bit

 0005:0007F53E 000000000H YIE                    DATA 32-bit

 0005:0007F53E 000000000H DATA                   DATA 32-bit

 0005:0007F540 000000000H CONST32                CONST 32-bit

 0005:0007F540 000000045H CONST32_RO             CONST 32-bit
	at offset 00000000 00045H bytes from F:\acpi\lib\acpidrv.lib (acpi)

 0005:0007F590 000000004H _NULL                  BEGDATA 32-bit
	at offset 00000000 00004H bytes from E:\watcom\lib386\os2\clib3r.lib (segdefns)

 0005:0007F594 000000000H _AFTERNULL             BEGDATA 32-bit

 0005:0007F5A0 000010000H STACK                  STACK 32-bit
	at offset 00000000 10000H bytes from E:\watcom\lib386\os2\clib3r.lib (segdefns)


 Origin   Group
 0000:0   FLAT
 0003:0   CGROUP
 0005:0   DGROUP


 Address         Publics by Name
 0003:000D5EE0       ACPIFindPCIDevice
 0003:0000A067       AddBaseAddress_
 0003:00003ED1       add_timer_
 0003:00010351       add_wait_queue_
 0003:0001036D       add_wait_queue_exclusive_
 0003:0000A74B       alloc_pages_
 0003:00007681       ALSAToOSSDataType_
 0003:00007776       ALSAToOSSRateFlags_
 0003:00003409       ALSA_FreeIrq_
 0003:00001672       ALSA_IDC
 0003:00003451       ALSA_Interrupt
 0003:00003326       ALSA_SetIrq_
 0003:00000656       ALSA_STRATEGY
 0003:00003D6C       ALSA_TIMER_
 0005:00001754       BootCode
 0003:000049DF       cancel_delayed_work_
 0003:000573C2       ca_midi_init_
 0003:00009B43       CharOut_
 0003:00091AB8       client_init_data_
 0003:00005A5C       ConvertVolume_
 0003:0000A996       copy_from_user_
 0003:000D7002       copy_from_user_toio_
 0003:0000A8F1       copy_to_user_
 0003:000D6F52       copy_to_user_fromio_
 0003:000042F6       create_proc_entry_
 0003:000046BD       create_workqueue_
 0003:0000A01D       DbgPrintIrq_
 0001:0000004C       DbgU32IntCnt
 0001:00000048       DbgU32TimerCnt
 0003:00009861       DecLongToASCII_
 0003:00003EEC       del_timer_
 0003:00004747       destroy_workqueue_
 0005:000017F0       DevHelp32
 0001:0000003C       DevHelpInit
 0003:00000010       DevHlp
 0003:00000030       DevHlp_ModifiedDS
 0003:0000445F       disable_dma_
 0003:0000CD4E       disable_irq_
 0000:00000000  Imp  DOS32FLATDS          (DOSCALLS.370)
 0000:00000000  Imp  DOSCLOSE             (DOSCALLS.59)
 0000:00000000  Imp  DosExit              (DOSCALLS.234)
 0000:00000000  Imp  DOSIODELAYCNT        (DOSCALLS.427)
 0000:00000000  Imp  DOSOPEN              (DOSCALLS.70)
 0000:00000000  Imp  DosQueryCp           (DOSCALLS.291)
 0000:00000000  Imp  DosQueryDBCSEnv      (NLS.6)
 0000:00000000  Imp  DosQuerySysInfo      (DOSCALLS.348)
 0000:00000000  Imp  DOSWRITE             (DOSCALLS.138)
 0000:00000000  Imp  DosWrite             (DOSCALLS.282)
 0003:000D6348       down_
 0003:000D63AC       down_interruptible_
 0003:00003E85       do_gettimeofday_
 0003:00004444       enable_dma_
 0003:0000CBA6       eoi_irq_
 0003:000043BE       fasync_helper_
 0001:0000046D       FileName
 0003:0000B5FC       FillCaps_
 0003:000D6070       FindAddress
 0003:00004650       flush_workqueue_
 0001:00000040       fOpen
 0003:00004429       free_dma_
 0003:0000CA9B       free_irq_
 0003:0000A63D       free_pages_
 0003:00004B1D       gcd_
 0003:0000A0CB       GetBaseAddress_
 0003:0000AFD1       GetMaxChannels_
 0003:0000AE57       GetNumberOfCards_
 0003:0000AE7A       GetNumberOfPcm_
 0003:00001513       GetParms_
 0003:0000AEEF       GetPcmForChannels_
 0003:00001624       GetTKSSBase
 0003:0000B940       GetUniaudCardInfo_
 0003:0000BEF2       GetUniaudControlInfo_
 0003:0000BA8C       GetUniaudControlNum_
 0003:0000BC81       GetUniaudControls_
 0003:0000C063       GetUniaudControlValueGet_
 0003:0000C1D4       GetUniaudControlValuePut_
 0003:0000B0BA       GetUniaudPcmCaps1_
 0003:0000B692       GetUniaudPcmCaps_
 0001:00000000       help_header
 0002:00000000       help_stub_strategy
 0003:000099CE       HexLongToASCII_
 0003:0000425C       hweight32_
 0003:000000E0       IDC_
 0003:0008CC07       ilog2_
 0003:000D5F82       InitACPICall
 0001:00000046       InitPktOff
 0001:00000044       InitPktSeg
 0003:000D62DC       init_MUTEX_
 0003:000D6312       init_MUTEX_LOCKED_
 0003:00010434       init_waitqueue_entry_
 0003:00010336       init_waitqueue_head_
 0003:000103D8       interruptible_sleep_on_
 0003:000103A4       interruptible_sleep_on_timeout_
 0005:000017F4       intSwitchStack
 0003:0000CD2B       in_interrupt_
 0003:00001664       iodelay32_
 0003:0005400E       ioport_map_
 0003:0005404A       ioport_unmap_
 0003:00053EB0       ioread16_
 0003:00053EFE       ioread32_
 0003:00053E64       ioread8_
 0003:0000A84C       iounmap_
 0003:00053F86       iowrite16_
 0003:00053FCB       iowrite32_
 0003:00053F43       iowrite8_
 0003:0000A87E       is_access_ok_
 0003:000E8E40       itoa_
 0003:0000AB9A       kcalloc_
 0000:00000000  Imp  KernLinToPageList    (KEE.64)
 0000:00000000  Imp  KernSelToFlat        (KEE.66)
 0000:00000000  Imp  KernThunkStackTo16   (KEE.40)
 0000:00000000  Imp  KernThunkStackTo32   (KEE.41)
 0000:00000000  Imp  KernVMAlloc          (KEE.60)
 0000:00000000  Imp  KernVMFree           (KEE.61)
 0000:00000000  Imp  KernVMLock           (KEE.62)
 0003:000043E6       kill_fasync_
 0003:0000476A       kstrdup_
 0003:0000AB54       kzalloc_
 0003:000E8DC0       lltoa_
 0003:000E8D20       ltoa_
 0003:000E8BF0       mbtowc_
 0003:00003E51       mdelay_
 0003:00004960       memdup_user_
 0003:000E6A60       memmove_
 0003:000E6A40       memset_
 0003:000047DC       mod_firmware_load_
 0003:00003F11       mod_timer_
 0003:00003F2D       msleep_
 0003:0000506D       MyDevBlock_
 0002:000003DA       MY_DEVHELP_ATTACHDD
 0003:00003625       os2gettimemsec_
 0003:00003602       os2gettimesec_
 0003:0000F6C4       OSS32_APMResume_
 0003:0000F771       OSS32_APMSuspend_
 0003:00005041       OSS32_CloseUNI16_
 0003:000050BF       OSS32_DebugString_
 0003:00004C83       OSS32_Initialize_
 0003:000055AD       OSS32_MidiClose_
 0003:00005879       OSS32_MidiCommand_
 0003:000050F6       OSS32_MidiOpen_
 0003:00005841       OSS32_MidiQueryCaps_
 0003:0000578D       OSS32_MidiRead_
 0003:00005755       OSS32_MidiWrite_
 0003:00006191       OSS32_MixClose_
 0003:00006C03       OSS32_MixGetProperty_
 0003:00006221       OSS32_MixGetVolume_
 0003:00005AA9       OSS32_MixOpen_
 0003:00006DD3       OSS32_MixQueryCaps_
 0003:00006EB9       OSS32_MixQueryName_
 0003:0000675D       OSS32_MixSetProperty_
 0003:00006272       OSS32_MixSetVolume_
 0003:00004FE5       OSS32_ProcessIRQ_
 0003:00005011       OSS32_ProcessMIDIIRQ_
 0003:00007865       OSS32_QueryDevCaps_
 0003:00007017       OSS32_QueryNames_
 0003:000040B6       OSS32_SetFileId_
 0003:00004F48       OSS32_Shutdown_
 0003:000091B9       OSS32_WaveAddBuffer_
 0003:000080EA       OSS32_WaveClose_
 0003:00009657       OSS32_WaveGetHwPtr_
 0003:000094C8       OSS32_WaveGetPosition_
 0003:000095A9       OSS32_WaveGetSpace_
 0003:000096FD       OSS32_WaveGetStatus_
 0003:00007E0D       OSS32_WaveOpen_
 0003:00008437       OSS32_WavePause_
 0003:00008271       OSS32_WavePrepare_
 0003:000084C5       OSS32_WaveResume_
 0003:00008556       OSS32_WaveSetHwParams_
 0003:0000979D       OSS32_WaveSetVolume_
 0003:0000831B       OSS32_WaveStart_
 0003:000083A9       OSS32_WaveStop_
 0003:00006C54       OSSToALSAVolume_
 0003:0000F831       PciAdjustInterrupts_
 0003:0000D86F       pcibios_present_
 0003:0000D022       pcidev_activate_
 0003:0000D059       pcidev_deactivate_
 0003:0000CFEB       pcidev_prepare_
 0003:0000E08C       pci_alloc_consistent_
 0003:0000E4ED       pci_disable_device_
 0003:0000D8DB       pci_dma_supported_
 0003:0000DB94       pci_enable_device_
 0003:0000D90F       pci_find_capability_
 0003:0000D591       pci_find_device_
 0003:0000D89F       pci_find_slot_
 0003:0000E1BA       pci_free_consistent_
 0003:0000E253       pci_get_dma_mask_
 0003:0000E21A       pci_get_driver_data_
 0003:0000D821       pci_get_flags_
 0003:00054065       pci_iomap_
 0003:00054295       pci_iounmap_
 0003:0000F4CE       pci_match_device_
 0003:0000DDF8       pci_module_init_
 0003:0000E341       pci_orig_restore_state_
 0003:0000E2E9       pci_orig_save_state_
 0003:0000CD7B       pci_read_config_byte_
 0003:0000CE55       pci_read_config_dword_
 0003:0000CDE7       pci_read_config_word_
 0003:0000DBFC       pci_register_driver_
 0003:0000F493       pci_release_regions_
 0003:0000EF93       pci_release_region_
 0003:0000F424       pci_request_regions_
 0003:0000E537       pci_request_region_
 0003:0000E469       pci_restore_state_
 0003:0000E3E8       pci_save_state_
 0003:0000E1EC       pci_set_driver_data_
 0003:0000E2B1       pci_set_latency_time_
 0003:0000DF8E       pci_set_master_
 0003:0000D9C7       pci_set_power_state_
 0003:0000DE36       pci_unregister_driver_
 0003:0000CEBA       pci_write_config_byte_
 0003:0000CF8B       pci_write_config_dword_
 0003:0000CF22       pci_write_config_word_
 0003:0001ED76       pcm_info_
 0003:0001EE5B       pcm_instances_
 0005:00001774       PDDName
 0001:00000466       pddname16
 0003:0000A1EB       phys_to_virt_
 0003:0000DFEA       pm_register_
 0003:0000E01F       pm_unregister_
 0003:00004218       poll_wait_
 0003:0000CBD2       process_interrupt_
 0003:00004372       proc_register_
 0003:00004398       proc_unregister_
 0003:00085712       query_amp_caps_
 0003:0008FC52       queueptr_
 0003:00004A9A       queue_delayed_work_
 0003:0000453B       queue_work_
 0003:0000720D       register_chrdev_
 0003:0000447A       register_reboot_notifier_
 0003:00007384       register_sound_dsp_
 0003:00007332       register_sound_midi_
 0003:000072E0       register_sound_mixer_
 0003:0000728E       register_sound_special_
 0003:000073D6       register_sound_synth_
 0003:000D6E5F       release_and_free_resource_
 0003:0000492C       release_firmware_
 0003:0000E28C       release_resource_
 0003:0000A771       remap_page_range_
 0003:00004356       remove_proc_entry_
 0003:00010388       remove_wait_queue_
 0003:00004403       request_dma_
 0003:00004882       request_firmware_
 0003:0000C8C2       request_irq_
 0005:00001778       RMAllocResource1632
 0005:00001798       RMCreateAdapter1632
 0005:00001790       RMCreateDevice1632
 0005:000017A0       RMCreateDriver1632
 0003:00002DB4       RMDeallocateIRQ_
 0005:00001788       RMDeallocResource1632
 0005:000017A8       RMDestroyDriver1632
 0005:000017B8       RMDevIDToHandleList1632
 0003:00002E2D       RMDone_
 0005:000017B0       RMGetNodeInfo1632
 0005:000017C0       RMHandleToResourceHandleList1632
 0003:000028EC       RMInit_
 0005:00001780       RMModifyResources1632
 0003:00002A9B       RMRequestIO_
 0003:00002C6E       RMRequestIRQ_
 0003:00002B8B       RMRequestMem_
 0003:000032FA       RMSetHandles_
 0003:00004200       schedule_
 0003:00003DCA       schedule_timeout_
 0003:00004A2B       schedule_work_
 0003:0000AEA3       SetPCMInstance_
 0003:000E1900       snd_ac97_bus_
 0003:000E5217       snd_ac97_bus_proc_done_
 0003:000E518D       snd_ac97_bus_proc_init_
 0003:000E15C2       snd_ac97_get_name_
 0003:000E179A       snd_ac97_get_short_name_
 0003:000E19EC       snd_ac97_mixer_
 0003:000D7A11       snd_ac97_pcm_assign_
 0003:000D81BD       snd_ac97_pcm_close_
 0003:000D83AE       snd_ac97_pcm_double_rate_rules_
 0003:000D7E62       snd_ac97_pcm_open_
 0003:000E5148       snd_ac97_proc_done_
 0003:000E4FB3       snd_ac97_proc_init_
 0003:000DE39C       snd_ac97_read_
 0003:000E2ABC       snd_ac97_resume_
 0003:000D73AD       snd_ac97_set_rate_
 0003:000E2939       snd_ac97_suspend_
 0003:000E3600       snd_ac97_tune_hardware_
 0003:000DE510       snd_ac97_update_
 0003:000DE5DF       snd_ac97_update_bits_
 0003:000DE654       snd_ac97_update_bits_nolock_
 0003:000DE322       snd_ac97_write_
 0003:000DE485       snd_ac97_write_cache_
 0003:0001F3FE       snd_add_device_sysfs_file_
 0003:0008A690       snd_array_free_
 0003:0008A586       snd_array_new_
 0003:000544EC       snd_ca0106_i2c_write_
 0003:000586F7       snd_ca0106_mixer_
 0003:000589EC       snd_ca0106_mixer_resume_
 0003:0005898D       snd_ca0106_mixer_suspend_
 0003:000596A2       snd_ca0106_proc_init_
 0003:0005430B       snd_ca0106_ptr_read_
 0003:00054371       snd_ca0106_ptr_write_
 0003:000543CF       snd_ca0106_spi_write_
 0003:0002CEE4       snd_card_create_
 0003:0002D4A1       snd_card_disconnect_
 0003:0002DF8F       snd_card_file_add_
 0003:0002E05F       snd_card_file_remove_
 0003:0002D7C7       snd_card_free_
 0003:0002D709       snd_card_free_when_closed_
 0003:0002DE55       snd_card_info_done_
 0003:0002DD9C       snd_card_info_init_
 0003:0002DCAC       snd_card_info_read_oss_
 0003:0002D257       snd_card_locked_
 0003:00020D81       snd_card_proc_new_
 0003:0002DB0A       snd_card_register_
 0003:0002DAC4       snd_card_set_id_
 0003:0002DE8B       snd_component_add_
 0003:000A13CC       snd_cs46xx_create_
 0003:0009DF4D       snd_cs46xx_download_
 0003:0009DFDA       snd_cs46xx_download_image_
 0003:000A028E       snd_cs46xx_gameport_
 0003:000A01AF       snd_cs46xx_midi_
 0003:0009FAC0       snd_cs46xx_mixer_
 0003:0009F695       snd_cs46xx_pcm_
 0003:000A1235       snd_cs46xx_resume_
 0003:000A0BA6       snd_cs46xx_start_dsp_
 0003:000A10E1       snd_cs46xx_suspend_
 0003:000A3031       snd_cs5535audio_pcm_
 0003:000A245B       snd_cs5535audio_resume_
 0003:000A2351       snd_cs5535audio_suspend_
 0003:0002A10D       snd_ctl_add_
 0003:0002C5BD       snd_ctl_boolean_mono_info_
 0003:0002C60B       snd_ctl_boolean_stereo_info_
 0003:0002C569       snd_ctl_create_
 0003:0002A5EB       snd_ctl_find_id_
 0003:0002A55E       snd_ctl_find_numid_
 0003:00029F7D       snd_ctl_free_one_
 0003:000D6D3D       snd_ctl_make_virtual_master_
 0003:00029E13       snd_ctl_new1_
 0003:00029BFD       snd_ctl_notify_
 0003:0002C187       snd_ctl_register_ioctl_
 0003:0002A2A0       snd_ctl_remove_
 0003:0002A36C       snd_ctl_remove_id_
 0003:0002A4C4       snd_ctl_rename_id_
 0003:0002C278       snd_ctl_unregister_ioctl_
 0003:0002937E       snd_device_disconnect_
 0003:000295D4       snd_device_disconnect_all_
 0003:00029253       snd_device_free_
 0003:00029659       snd_device_free_all_
 0003:00029186       snd_device_new_
 0003:00029451       snd_device_register_
 0003:0002952D       snd_device_register_all_
 0003:0002C870       snd_dma_alloc_pages_
 0003:0002C981       snd_dma_alloc_pages_fallback_
 0003:0002CA1E       snd_dma_free_pages_
 0003:0002CAA4       snd_dma_get_reserved_buf_
 0003:0002CBC9       snd_dma_reserve_buf_
 0003:000B8DCC       snd_emu1010_fpga_link_dst_src_write_
 0003:000B8D2B       snd_emu1010_fpga_read_
 0003:000B8C65       snd_emu1010_fpga_write_
 0003:000B945E       snd_emu10k1_ac97_read_
 0003:000B94C7       snd_emu10k1_ac97_write_
 0003:000BA125       snd_emu10k1_alloc_pages_
 0003:000B4C0D       snd_emu10k1_audigy_midi_
 0003:000B6A4A       snd_emu10k1_create_
 0003:000B56E4       snd_emu10k1_done_
 0003:000ACC24       snd_emu10k1_efx_alloc_pm_buffer_
 0003:000ACD5B       snd_emu10k1_efx_free_pm_buffer_
 0003:000A575E       snd_emu10k1_efx_read_
 0003:000ACF53       snd_emu10k1_efx_resume_
 0003:000ACDAE       snd_emu10k1_efx_suspend_
 0003:000ABF40       snd_emu10k1_free_efx_
 0003:000BA2F2       snd_emu10k1_free_pages_
 0003:000ACB4E       snd_emu10k1_fx8010_new_
 0003:000A53F1       snd_emu10k1_fx8010_register_irq_handler_
 0003:000ABFB0       snd_emu10k1_fx8010_tram_setup_
 0003:000A54DF       snd_emu10k1_fx8010_unregister_irq_handler_
 0003:000B8AF1       snd_emu10k1_i2c_write_
 0003:000ABED2       snd_emu10k1_init_efx_
 0003:000BA941       snd_emu10k1_interrupt_
 0003:000B8E9C       snd_emu10k1_intr_disable_
 0003:000B8E42       snd_emu10k1_intr_enable_
 0003:000B9FE5       snd_emu10k1_memblk_map_
 0003:000B4B7E       snd_emu10k1_midi_
 0003:000AF7AA       snd_emu10k1_mixer_
 0003:000B320B       snd_emu10k1_pcm_
 0003:000B4044       snd_emu10k1_pcm_efx_
 0003:000B34AF       snd_emu10k1_pcm_mic_
 0003:000B3386       snd_emu10k1_pcm_multi_
 0003:000B8373       snd_emu10k1_proc_init_
 0003:000B88C1       snd_emu10k1_ptr20_read_
 0003:000B892E       snd_emu10k1_ptr20_write_
 0003:000B8673       snd_emu10k1_ptr_read_
 0003:000B8784       snd_emu10k1_ptr_write_
 0003:000B9528       snd_emu10k1_rate_to_pitch_
 0003:000B7520       snd_emu10k1_resume_init_
 0003:000B75A8       snd_emu10k1_resume_regs_
 0003:000B8993       snd_emu10k1_spi_write_
 0003:000B7423       snd_emu10k1_suspend_regs_
 0003:000BA33D       snd_emu10k1_synth_alloc_
 0003:000BA7BD       snd_emu10k1_synth_bzero_
 0003:000BA873       snd_emu10k1_synth_copy_from_user_
 0003:000BA3E5       snd_emu10k1_synth_free_
 0003:000A4E73       snd_emu10k1_timer_
 0003:000B97A9       snd_emu10k1_voice_alloc_
 0003:000B9336       snd_emu10k1_voice_clear_loop_stop_
 0003:000B9917       snd_emu10k1_voice_free_
 0003:000B920E       snd_emu10k1_voice_half_loop_intr_ack_
 0003:000B9168       snd_emu10k1_voice_half_loop_intr_disable_
 0003:000B90C6       snd_emu10k1_voice_half_loop_intr_enable_
 0003:000B4D0C       snd_emu10k1_voice_init_
 0003:000B9040       snd_emu10k1_voice_intr_ack_
 0003:000B8F9A       snd_emu10k1_voice_intr_disable_
 0003:000B8EF8       snd_emu10k1_voice_intr_enable_
 0003:000B9294       snd_emu10k1_voice_set_loop_stop_
 0003:000B93DC       snd_emu10k1_wait_
 0003:0002C80D       snd_free_dev_pages_
 0003:0002C748       snd_free_pages_
 0003:0002E30E       snd_free_sgbuf_pages_
 0003:00083881       snd_hda_add_codec_preset_
 0003:00089001       snd_hda_add_new_ctls_
 0003:00086574       snd_hda_add_nid_
 0003:00084A1C       snd_hda_add_pincfg_
 0003:0008698E       snd_hda_add_vmaster_
 0003:00087FFB       snd_hda_build_controls_
 0003:00088CD7       snd_hda_build_pcms_
 0003:00084293       snd_hda_bus_new_
 0003:000894D3       snd_hda_bus_reboot_notify_
 0003:0008810E       snd_hda_calc_stream_format_
 0003:00088ECE       snd_hda_check_board_codec_sid_config_
 0003:00088D3F       snd_hda_check_board_config_
 0003:00089158       snd_hda_ch_mode_get_
 0003:000890DB       snd_hda_ch_mode_info_
 0003:000891B4       snd_hda_ch_mode_put_
 0003:00085BB6       snd_hda_codec_amp_read_
 0003:00085D46       snd_hda_codec_amp_stereo_
 0003:00085C45       snd_hda_codec_amp_update_
 0003:0008809A       snd_hda_codec_build_controls_
 0003:00088BA1       snd_hda_codec_build_pcms_
 0003:000854DF       snd_hda_codec_cleanup_stream_
 0003:0008530B       snd_hda_codec_configure_
 0003:00084B29       snd_hda_codec_get_pincfg_
 0003:00084E46       snd_hda_codec_new_
 0003:0008E65C       snd_hda_codec_proc_new_
 0003:00083BFD       snd_hda_codec_read_
 0003:00086723       snd_hda_codec_reset_
 0003:00085DCA       snd_hda_codec_resume_amp_
 0003:00087C6A       snd_hda_codec_resume_cache_
 0003:00085453       snd_hda_codec_setup_stream_
 0003:00084AEC       snd_hda_codec_set_pincfg_
 0003:00087BAF       snd_hda_codec_update_cache_
 0003:00083C4F       snd_hda_codec_write_
 0003:00087AFE       snd_hda_codec_write_cache_
 0003:0008AAC1       snd_hda_create_hwdep_
 0003:00087A04       snd_hda_create_spdif_in_ctls_
 0003:00087648       snd_hda_create_spdif_out_ctls_
 0003:0008780D       snd_hda_create_spdif_share_sw_
 0003:00086605       snd_hda_ctls_clear_
 0003:000864A0       snd_hda_ctl_add_
 0003:000838E2       snd_hda_delete_codec_preset_
 0003:00086471       snd_hda_find_mixer_ctl_
 0003:00083D6E       snd_hda_get_connections_
 0003:000839D7       snd_hda_get_jack_connectivity_
 0003:0008394C       snd_hda_get_jack_location_
 0003:00083A0A       snd_hda_get_jack_type_
 0003:00083D07       snd_hda_get_sub_nodes_
 0003:00089246       snd_hda_input_mux_info_
 0003:000892E4       snd_hda_input_mux_put_
 0003:000886A1       snd_hda_is_supported_format_
 0003:000859DE       snd_hda_jack_detect_
 0003:00086B5E       snd_hda_mixer_amp_switch_get_
 0003:00086AEC       snd_hda_mixer_amp_switch_info_
 0003:00086C4C       snd_hda_mixer_amp_switch_put_
 0003:00086229       snd_hda_mixer_amp_tlv_
 0003:0008605C       snd_hda_mixer_amp_volume_get_
 0003:00085EB0       snd_hda_mixer_amp_volume_info_
 0003:00086137       snd_hda_mixer_amp_volume_put_
 0003:00086F1D       snd_hda_mixer_bind_ctls_get_
 0003:00086EA7       snd_hda_mixer_bind_ctls_info_
 0003:00086F94       snd_hda_mixer_bind_ctls_put_
 0003:00086D5D       snd_hda_mixer_bind_switch_get_
 0003:00086DD3       snd_hda_mixer_bind_switch_put_
 0003:00087054       snd_hda_mixer_bind_tlv_
 0003:00089A3C       snd_hda_multi_out_analog_cleanup_
 0003:0008968C       snd_hda_multi_out_analog_open_
 0003:0008983D       snd_hda_multi_out_analog_prepare_
 0003:000895F1       snd_hda_multi_out_dig_cleanup_
 0003:00089642       snd_hda_multi_out_dig_close_
 0003:00089532       snd_hda_multi_out_dig_open_
 0003:00089596       snd_hda_multi_out_dig_prepare_
 0003:000857EE       snd_hda_override_amp_caps_
 0003:0008CAD9       snd_hda_parse_generic_codec_
 0003:00089C62       snd_hda_parse_pin_def_config_
 0003:00085968       snd_hda_pin_sense_
 0003:00085927       snd_hda_query_pin_caps_
 0003:00084076       snd_hda_queue_unsol_event_
 0003:0008A52F       snd_hda_resume_
 0003:00083CBB       snd_hda_sequence_write_
 0003:00087CF2       snd_hda_sequence_write_cache_
 0003:00086360       snd_hda_set_vmaster_tlv_
 0003:00084C5C       snd_hda_shutup_pins_
 0003:0008A4D8       snd_hda_suspend_
 0003:00010FC1       snd_hwdep_new_
 0003:00020678       snd_info_card_create_
 0003:00020802       snd_info_card_disconnect_
 0003:00020894       snd_info_card_free_
 0003:00020792       snd_info_card_id_change_
 0003:0002072C       snd_info_card_register_
 0003:0001F797       snd_info_check_reserved_words_
 0003:00020BF9       snd_info_create_card_entry_
 0003:00020BB0       snd_info_create_module_entry_
 0003:000205F6       snd_info_done_
 0003:00020E0A       snd_info_free_entry_
 0003:000208E3       snd_info_get_line_
 0003:000209ED       snd_info_get_str_
 0003:000204EA       snd_info_init_
 0003:00028A01       snd_info_minor_register_
 0003:00028A7F       snd_info_minor_unregister_
 0003:00020E76       snd_info_register_
 0003:0001A52D       snd_interval_div_
 0003:0001B01B       snd_interval_list_
 0003:0001A682       snd_interval_muldivk_
 0003:0001A7BF       snd_interval_mulkdiv_
 0003:0001A3D1       snd_interval_mul_
 0003:0001A91B       snd_interval_ratnum_
 0003:0001A0F2       snd_interval_refine_
 0003:00009D11       snd_iprintf_
 0003:0001EF31       snd_lookup_minor_data_
 0003:00028AB5       snd_lookup_oss_minor_data_
 0003:0002C798       snd_malloc_dev_pages_
 0003:0002C6DC       snd_malloc_pages_
 0003:0002E38A       snd_malloc_sgbuf_pages_
 0003:000E61F4       snd_midi_channel_alloc_set_
 0003:000E6294       snd_midi_channel_free_set_
 0003:000E5A80       snd_midi_channel_set_clear_
 0003:000E5247       snd_midi_process_event_
 0003:0001F61C       snd_minor_info_done_
 0003:0001F5B3       snd_minor_info_init_
 0003:0002911B       snd_minor_info_oss_done_
 0003:000290AE       snd_minor_info_oss_init_
 0003:0009C306       snd_mpu401_uart_interrupt_
 0003:0009C349       snd_mpu401_uart_interrupt_tx_
 0003:0009CD24       snd_mpu401_uart_new_
 0003:0009A18F       snd_opl3_calc_volume_
 0003:0009BAAB       snd_opl3_clear_patches_
 0003:0009B302       snd_opl3_control_
 0003:000998E2       snd_opl3_create_
 0003:0009A08F       snd_opl3_drum_switch_
 0003:0009B9C1       snd_opl3_find_patch_
 0003:00099B33       snd_opl3_hwdep_new_
 0003:0009982E       snd_opl3_init_
 0003:00099642       snd_opl3_interrupt_
 0003:0009B431       snd_opl3_ioctl_
 0003:0009B0FC       snd_opl3_key_press_
 0003:00099FFF       snd_opl3_load_drums_
 0003:0009B7C1       snd_opl3_load_patch_
 0003:00099770       snd_opl3_new_
 0003:0009B0AA       snd_opl3_note_off_
 0003:0009A6BD       snd_opl3_note_on_
 0003:0009B3C2       snd_opl3_nrpn_
 0003:0009B40B       snd_opl3_open_
 0003:0009B66B       snd_opl3_release_
 0003:0009BB1B       snd_opl3_reset_
 0003:00098AD9       snd_opl3_synth_cleanup_
 0003:000989D2       snd_opl3_synth_setup_
 0003:0009899E       snd_opl3_synth_use_dec_
 0003:0009895D       snd_opl3_synth_use_inc_
 0003:0009B3E5       snd_opl3_sysex_
 0003:0009B120       snd_opl3_terminate_note_
 0003:0009A54B       snd_opl3_timer_func_
 0003:00099AAD       snd_opl3_timer_new_
 0003:0009B6A5       snd_opl3_write_
 0003:00028768       snd_oss_info_register_
 0003:000A4C02       snd_p16v_alloc_pm_buffer_
 0003:000A44A6       snd_p16v_free_
 0003:000A4C51       snd_p16v_free_pm_buffer_
 0003:000A4B8C       snd_p16v_mixer_
 0003:000A44DF       snd_p16v_pcm_
 0003:000A4CEA       snd_p16v_resume_
 0003:000A4C7A       snd_p16v_suspend_
 0003:0000F683       snd_pci_compat_get_pci_driver_
 0003:0000F5CC       snd_pci_dev_present_
 0003:000D6F13       snd_pci_quirk_lookup_
 0003:000D6E90       snd_pci_quirk_lookup_id_
 0003:0001E27A       snd_pcm_attach_substream_
 0003:0001E6B6       snd_pcm_detach_substream_
 0003:000243A8       snd_pcm_drain_done_
 0003:00018831       snd_pcm_format_big_endian_
 0003:00018799       snd_pcm_format_linear_
 0003:000187D9       snd_pcm_format_little_endian_
 0003:0001DD07       snd_pcm_format_name_
 0003:000188DB       snd_pcm_format_physical_width_
 0003:000189D2       snd_pcm_format_set_silence_
 0003:000186EE       snd_pcm_format_signed_
 0003:00018978       snd_pcm_format_silence_64_
 0003:00018932       snd_pcm_format_size_
 0003:00018746       snd_pcm_format_unsigned_
 0003:00018884       snd_pcm_format_width_
 0003:00026409       snd_pcm_hw_constraints_complete_
 0003:00025E67       snd_pcm_hw_constraints_init_
 0003:0001B468       snd_pcm_hw_constraint_integer_
 0003:0001B5CB       snd_pcm_hw_constraint_list_
 0003:0001B3C3       snd_pcm_hw_constraint_mask64_
 0003:0001B346       snd_pcm_hw_constraint_mask_
 0003:0001B4C0       snd_pcm_hw_constraint_minmax_
 0003:0001B8C4       snd_pcm_hw_constraint_msbits_
 0003:0001BA39       snd_pcm_hw_constraint_pow2_
 0003:0001B7DF       snd_pcm_hw_constraint_ratdens_
 0003:0001B6D5       snd_pcm_hw_constraint_ratnums_
 0003:0001B982       snd_pcm_hw_constraint_step_
 0003:0001C1FA       snd_pcm_hw_params_choose_
 0003:0001BFD7       snd_pcm_hw_param_first_
 0003:0001C175       snd_pcm_hw_param_last_
 0003:0001BC2A       snd_pcm_hw_param_value_
 0003:0002258D       snd_pcm_hw_refine_
 0003:0001B1CE       snd_pcm_hw_rule_add_
 0003:000223D5       snd_pcm_info_
 0003:00022510       snd_pcm_info_user_
 0003:00028194       snd_pcm_kernel_ioctl_
 0003:000215F8       snd_pcm_lib_free_pages_
 0003:00021746       snd_pcm_lib_free_vmalloc_buffer_
 0003:0001C500       snd_pcm_lib_ioctl_
 0003:000214B3       snd_pcm_lib_malloc_pages_
 0003:000211D4       snd_pcm_lib_preallocate_free_
 0003:00021201       snd_pcm_lib_preallocate_free_for_all_
 0003:000212E2       snd_pcm_lib_preallocate_pages_
 0003:00021328       snd_pcm_lib_preallocate_pages_for_all_
 0003:0001D79C       snd_pcm_lib_readv_
 0003:0001D543       snd_pcm_lib_read_
 0003:0001D01F       snd_pcm_lib_writev_
 0003:0001CD5C       snd_pcm_lib_write_
 0003:00018B92       snd_pcm_limit_hw_rates_
 0003:0001DFA9       snd_pcm_new_
 0003:0001DD34       snd_pcm_new_stream_
 0003:0001EAF1       snd_pcm_notify_
 0003:00026772       snd_pcm_open_substream_
 0003:000D29DF       snd_pcm_oss_read3_
 0003:000D2BD8       snd_pcm_oss_readv3_
 0003:000D290E       snd_pcm_oss_write3_
 0003:000D2B07       snd_pcm_oss_writev3_
 0003:0001C582       snd_pcm_period_elapsed_
 0003:000195C0       snd_pcm_playback_silence_
 0003:00018C47       snd_pcm_rate_to_rate_bit_
 0003:000266D1       snd_pcm_release_substream_
 0003:00019E7A       snd_pcm_set_ops_
 0003:00019ECC       snd_pcm_set_sync_
 0003:0002140F       snd_pcm_sgbuf_get_chunk_size_
 0003:000213AE       snd_pcm_sgbuf_ops_page_
 0003:00024218       snd_pcm_start_
 0003:000237A6       snd_pcm_status_
 0003:00024376       snd_pcm_stop_
 0003:00024727       snd_pcm_suspend_
 0003:0002479D       snd_pcm_suspend_all_
 0003:00021ADF       snd_pcm_timer_done_
 0003:000219C4       snd_pcm_timer_init_
 0003:000217AD       snd_pcm_timer_resolution_change_
 0003:00019E4F       snd_pcm_update_hw_ptr_
 0003:00019A89       snd_pcm_update_state_
 0003:0002E1BA       snd_power_wait_
 0003:0008A74F       snd_print_pcm_bits_
 0003:0008A6D3       snd_print_pcm_rates_
 0003:00015B15       snd_rawmidi_drain_input_
 0003:00015A41       snd_rawmidi_drain_output_
 0003:000159C8       snd_rawmidi_drop_output_
 0003:0001666D       snd_rawmidi_info_select_
 0003:0001697D       snd_rawmidi_input_params_
 0003:00015E49       snd_rawmidi_kernel_open_
 0003:00016F40       snd_rawmidi_kernel_read_
 0003:0001646A       snd_rawmidi_kernel_release_
 0003:000176C4       snd_rawmidi_kernel_write_
 0003:00017D64       snd_rawmidi_new_
 0003:00016832       snd_rawmidi_output_params_
 0003:00016B88       snd_rawmidi_receive_
 0003:00018591       snd_rawmidi_set_ops_
 0003:0001745C       snd_rawmidi_transmit_
 0003:0001735B       snd_rawmidi_transmit_ack_
 0003:0001716A       snd_rawmidi_transmit_empty_
 0003:000171F4       snd_rawmidi_transmit_peek_
 0003:0001F1B8       snd_register_device_for_dev_
 0003:00028CBF       snd_register_oss_device_
 0003:000CEECE       snd_sbdsp_command_
 0003:000CF369       snd_sbdsp_create_
 0003:000CEF4D       snd_sbdsp_get_byte_
 0003:000CEFC9       snd_sbdsp_reset_
 0003:000CE879       snd_sbmixer_add_ctl_
 0003:000CEA27       snd_sbmixer_new_
 0003:000CDAA0       snd_sbmixer_read_
 0003:000CEDF7       snd_sbmixer_resume_
 0003:000CED20       snd_sbmixer_suspend_
 0003:000CDA55       snd_sbmixer_write_
 0003:00095725       snd_sequencer_device_done_
 0003:000956AC       snd_sequencer_device_init_
 0003:000917AD       snd_sequencer_memory_done_
 0003:0009178B       snd_sequencer_memory_init_
 0003:00090F0F       snd_seq_cell_free_
 0003:0008FD1F       snd_seq_check_queue_
 0003:000936D7       snd_seq_client_notify_subscription_
 0003:000919D2       snd_seq_client_use_ptr_
 0003:00090918       snd_seq_control_queue_
 0003:00094CE7       snd_seq_create_kernel_client_
 0003:00095A01       snd_seq_create_port_
 0003:00095F8D       snd_seq_delete_all_ports_
 0003:00094E29       snd_seq_delete_kernel_client_
 0003:00095E9A       snd_seq_delete_port_
 0003:0008E8B8       snd_seq_device_load_drivers_
 0003:0008E8D0       snd_seq_device_new_
 0003:0008EC2B       snd_seq_device_register_driver_
 0003:0008EE18       snd_seq_device_unregister_driver_
 0003:000927F8       snd_seq_dispatch_event_
 0003:00090BFD       snd_seq_dump_var_event_
 0003:0008FEA8       snd_seq_enqueue_event_
 0003:000911B4       snd_seq_event_dup_
 0003:00096B45       snd_seq_event_port_attach_
 0003:00096C01       snd_seq_event_port_detach_
 0003:00090DD6       snd_seq_expand_var_event_
 0003:000986A6       snd_seq_fifo_cell_out_
 0003:000987B6       snd_seq_fifo_cell_putback_
 0003:000984FA       snd_seq_fifo_clear_
 0003:00098454       snd_seq_fifo_delete_
 0003:00098553       snd_seq_fifo_event_in_
 0003:00098371       snd_seq_fifo_new_
 0003:0009880C       snd_seq_fifo_poll_wait_
 0003:0009885C       snd_seq_fifo_resize_
 0003:0009624B       snd_seq_get_port_info_
 0003:000954D4       snd_seq_info_clients_read_
 0003:0008F40B       snd_seq_info_done_
 0003:0008F3AD       snd_seq_info_init_
 0003:000917C5       snd_seq_info_pool_
 0003:000909B5       snd_seq_info_queues_read_
 0003:0009781B       snd_seq_info_timer_read_
 0003:00095097       snd_seq_kernel_client_ctl_
 0003:00094FEA       snd_seq_kernel_client_dispatch_
 0003:00094F6E       snd_seq_kernel_client_enqueue_
 0003:00094FA9       snd_seq_kernel_client_enqueue_blocking_
 0003:00095101       snd_seq_kernel_client_write_poll_
 0003:00091736       snd_seq_pool_delete_
 0003:00091559       snd_seq_pool_done_
 0003:00091435       snd_seq_pool_init_
 0003:00091689       snd_seq_pool_new_
 0003:000913C2       snd_seq_pool_poll_wait_
 0003:000965CF       snd_seq_port_connect_
 0003:0009690E       snd_seq_port_disconnect_
 0003:00096AC5       snd_seq_port_get_subscription_
 0003:000958C3       snd_seq_port_query_nearest_
 0003:00095814       snd_seq_port_use_ptr_
 0003:00097DC5       snd_seq_prioq_avail_
 0003:00097B9C       snd_seq_prioq_cell_in_
 0003:00097D2D       snd_seq_prioq_cell_out_
 0003:00097E09       snd_seq_prioq_cell_peek_
 0003:000979E2       snd_seq_prioq_delete_
 0003:00097EF6       snd_seq_prioq_leave_
 0003:0009796A       snd_seq_prioq_new_
 0003:0009821B       snd_seq_prioq_remove_events_
 0003:0008FB28       snd_seq_queues_delete_
 0003:0008FB06       snd_seq_queues_init_
 0003:0008FB75       snd_seq_queue_alloc_
 0003:000900A7       snd_seq_queue_check_access_
 0003:0009052B       snd_seq_queue_client_leave_
 0003:000905EE       snd_seq_queue_client_leave_cells_
 0003:0009048D       snd_seq_queue_client_termination_
 0003:0008FBF2       snd_seq_queue_delete_
 0003:0008FCB5       snd_seq_queue_find_name_
 0003:0008F834       snd_seq_queue_get_cur_queues_
 0003:00090418       snd_seq_queue_is_used_
 0003:00090651       snd_seq_queue_remove_cells_
 0003:0009010D       snd_seq_queue_set_owner_
 0003:00090225       snd_seq_queue_timer_close_
 0003:000901B3       snd_seq_queue_timer_open_
 0003:0009027B       snd_seq_queue_timer_set_tempo_
 0003:00090337       snd_seq_queue_use_
 0003:000960F5       snd_seq_set_port_info_
 0003:00093F4B       snd_seq_set_queue_tempo_
 0003:0008F4CB       snd_seq_system_broadcast_
 0003:0008F720       snd_seq_system_client_done_
 0003:0008F5AA       snd_seq_system_client_init_
 0003:0008F513       snd_seq_system_notify_
 0003:00097471       snd_seq_timer_close_
 0003:000976C7       snd_seq_timer_continue_
 0003:00096E67       snd_seq_timer_defaults_
 0003:00096E07       snd_seq_timer_delete_
 0003:000977F4       snd_seq_timer_get_cur_tick_
 0003:00097756       snd_seq_timer_get_cur_time_
 0003:00096D9C       snd_seq_timer_new_
 0003:0009730B       snd_seq_timer_open_
 0003:00096F0C       snd_seq_timer_reset_
 0003:0009719F       snd_seq_timer_set_position_tick_
 0003:0009720F       snd_seq_timer_set_position_time_
 0003:000970E8       snd_seq_timer_set_ppq_
 0003:00097280       snd_seq_timer_set_skew_
 0003:00097060       snd_seq_timer_set_tempo_
 0003:00097641       snd_seq_timer_start_
 0003:000974E6       snd_seq_timer_stop_
 0003:00011D60       snd_timer_close_
 0003:000125B5       snd_timer_continue_
 0003:00013401       snd_timer_global_free_
 0003:000133AC       snd_timer_global_new_
 0003:0001342A       snd_timer_global_register_
 0003:00012880       snd_timer_interrupt_
 0003:00012D17       snd_timer_new_
 0003:0001326D       snd_timer_notify_
 0003:00011AE0       snd_timer_open_
 0003:0001267F       snd_timer_pause_
 0003:00011FF3       snd_timer_resolution_
 0003:00012301       snd_timer_start_
 0003:00012535       snd_timer_stop_
 0003:000CAFCC       snd_trident_alloc_pages_
 0003:000CA54C       snd_trident_alloc_voice_
 0003:000C9D6A       snd_trident_create_
 0003:000C943E       snd_trident_create_gameport_
 0003:000C79D7       snd_trident_foldback_pcm_
 0003:000CB030       snd_trident_free_pages_
 0003:000CA6A3       snd_trident_free_voice_
 0003:000C7821       snd_trident_pcm_
 0003:000CA9A9       snd_trident_resume_
 0003:000C7BEE       snd_trident_spdif_pcm_
 0003:000C5085       snd_trident_start_voice_
 0003:000C50DE       snd_trident_stop_voice_
 0003:000CA8DE       snd_trident_suspend_
 0003:000C52E1       snd_trident_write_voice_regs_
 0003:0001F378       snd_unregister_device_
 0003:00028E3E       snd_unregister_oss_device_
 0003:000E63B3       snd_util_memhdr_free_
 0003:000E6343       snd_util_memhdr_new_
 0003:000E65C0       snd_util_mem_alloc_
 0003:000E66D4       snd_util_mem_avail_
 0003:000E666F       snd_util_mem_free_
 0003:000C0D8A       snd_ymfpci_create_
 0003:000BAE92       snd_ymfpci_free_gameport_
 0003:000BF3F2       snd_ymfpci_mixer_
 0003:000BDF83       snd_ymfpci_pcm2_
 0003:000BDE7F       snd_ymfpci_pcm_
 0003:000BE173       snd_ymfpci_pcm_4ch_
 0003:000BE081       snd_ymfpci_pcm_spdif_
 0003:000C0BFC       snd_ymfpci_resume_
 0003:000C0A74       snd_ymfpci_suspend_
 0003:000BF8DB       snd_ymfpci_timer_
 0003:000E6A10       snprintf_
 0003:00010499       spin_lock_
 0003:000104BE       spin_lock_flag_
 0003:00010475       spin_lock_init_
 0003:000104E4       spin_trylock_
 0003:00010509       spin_unlock_
 0003:00003D2D       sprintf_
 0003:000E6940       sscanf_
 0005:00001764       stackbase
 0005:00001768       stacksel
 0003:00000080       STRATEGY_
 0003:00003F70       strcmp_
 0003:00004B7B       strict_strtoul_
 0003:00009B89       StringOut_
 0003:000E6880       strlcpy_
 0003:000D6020       StrLen
 0003:000D6040       StrNCmp
 0003:00003FCD       strncmp_
 0003:000102CF       strncpy_
 0003:000E67D0       strstr_
 0003:000E6CF0       strtol_
 0003:000E6CE0       strtoul_
 0003:000E8A20       strupr_
 0003:0000403C       tasklet_hi_schedule_
 0003:00004074       tasklet_init_
 0003:00000024       thunk1632_devhelp
 0003:00000044       thunk1632_devhelp_modified_ds
 0002:000001A0       thunk3216_devhelp
 0002:000001B2       thunk3216_devhelp_modified_ds
 0003:00000140       TIMER_
 0003:000E89C0       tolower_
 0003:000E8D50       ulltoa_
 0003:000E8CD0       ultoa_
 0003:0000C7AC       UniaudCloseAll_
 0003:0000B708       UniaudCtlGetPowerState_
 0003:0000B824       UniaudCtlSetPowerState_
 0003:0000C3C5       UniaudIoctlHWParamSet_
 0003:0000C345       UniaudIoctlHWRefine_
 0003:0000C74A       UniaudIoctlPCMDrop_
 0003:0000C622       UniaudIoctlPCMPrepare_
 0003:0000C5B0       UniaudIoctlPCMRead_
 0003:0000C684       UniaudIoctlPCMResume_
 0003:0000C6E8       UniaudIoctlPCMStart_
 0003:0000C4C5       UniaudIoctlPCMStatus_
 0003:0000C53E       UniaudIoctlPCMWrite_
 0003:0000C445       UniaudIoctlSWParamSet_
 0001:0000001E       uniaud_header
 0003:0000ABEC       uniaud_set_interrupted_substream_
 0002:0000010A       uniaud_stub_idc
 0002:00000096       uniaud_stub_strategy
 0002:00000128       uniaud_stub_timer
 0003:00007504       UNIXToOSSError_
 0003:0000724D       unregister_chrdev_
 0003:0000449F       unregister_reboot_notifier_
 0003:000074AC       unregister_sound_dsp_
 0003:00007480       unregister_sound_midi_
 0003:00007454       unregister_sound_mixer_
 0003:00007428       unregister_sound_special_
 0003:000074D8       unregister_sound_synth_
 0003:000D637A       up_
 0003:000E8DF0       utoa_
 0003:0000A707       vfree_
 0003:0000A1A1       virt_to_phys_
 0003:0000A68F       vmalloc_
 0003:0000A24A       VMAlloc_
 0003:0000A314       VMFree_
 0003:000E69B0       vsnprintf_
 0003:00003947       vsprintf_
 0003:000E6910       vsscanf_
 0003:000035A5       W?$dln(pnv)v
 0003:0000357C       W?$nwn(ui)pnv
 0003:000035C8       W?$nwn(uipnv)pnv
 0005:00000554       W?acHeap$npnuc
 0003:00004C1B       W?CallOSS16$n(ululul)ul
 0003:00001096       W?CheckCardName$n(pfa)v
 0003:0000FEF8       W?compact$n()v
 0005:00000030       W?deviceOwner$nul
 0003:0000084E       W?DevSaveMessage$n(pfai)v
 0003:00000A0D       W?DiscardableInit$n(pf$RPInit$$)ul
 0003:00001313       W?DoParm$n(apfa)i
 0003:0000F9A0       W?dumpheap$n()v
 0005:000000B0       W?fnCardExitCall$n[]pn()v
 0005:00001894       W?ForceCard$ni
 0003:0000FFC0       W?free$n(pnv)v
 0003:0000FB8D       W?HeapCheck$n(pna)v
 0003:00010227       W?HeapInit$n(ul)ul
 0003:000101D1       W?IsHeapAddr$n(ul)ul
 0003:00000FC7       W?IsWhitespace$n(a)i
 0003:0000090D       W?LockSegments$n()i
 0003:0000FD98       W?malloc$n(ul)pnv
 0003:00000E5D       W?mymemchr$n(pfaaus)pfa
 0003:0000FCA5       W?npvAllocateBlock$n(pn$_MEMBLOCK$$ulpn$1$)pnv
 0005:00000034       W?numOS2Opens$nul
 0003:000016FC       W?OSS32IDC$n(ulpn$__6ikc0pIDC32_PACKET$$)ul
 0003:0000140E       W?ParseParm$n(pfai)i
 0005:0000054C       W?pmbFree$npn$_MEMBLOCK$$
 0005:00000548       W?pmbUsed$npn$_MEMBLOCK$$
 0003:00010124       W?realloc$n(pnvul)pnv
 0003:0000FE8F       W?remove$n(pn$_MEMBLOCK$$)v
 0005:00000060       W?RMFlags$nul
 0005:00000054       W?RM_Help$npn()i
 0005:00000058       W?RM_Help0$npn()i
 0005:0000005C       W?RM_Help3$npn()i
 0003:0000FAE3       W?SignatureCheck$n(pn$_MEMBLOCK$$pna)s
 0003:00001018       W?SkipWhite$n(pfa)pfa
 0003:0000288A       W?StratClose$n(pf$RP$$)ul
 0005:00001800       W?StratDispatch$n[]pn(pf$RP$$)ul
 0003:00000544       W?StratInit$n(pf$RP$$)ul
 0003:000005AE       W?StratInitComplete$n(pf$RP$$)ul
 0003:00001CB3       W?StratIOCtl$n(pf$RP$$)ul
 0003:000004DD       W?StratOpen$n(pf$RP$$)ul
 0003:000006D8       W?StratRead$n(pf$RP$$)ul
 0003:000005E9       W?StratShutdown$n(pf$RP$$)ul
 0003:00000EDC       W?sz2us$n(pfai)us
 0003:00000E1D       W?toupper$n(i)i
 0005:0000055C       W?ulcAlloc$nul
 0005:00000568       W?ulcFree$nul
 0005:0000E9E0       W?ulcTotalHeap$nul
 0005:00000558       W?ulnAlloc$nul
 0005:00000560       W?ulnAllocCalls$nul
 0005:00000570       W?ulnCompact$nul
 0005:00000564       W?ulnFree$nul
 0005:0000056C       W?ulnFreeCalls$nul
 0005:00000550       W?uMemFree$nui
 0003:000100C2       W?_memfree$n()ui
 0003:000100E5       W?_msize$n(pnv)ui
 0003:0000AC52       WaitForControlChange_
 0003:0000ACEB       WaitForPCMInterrupt_
 0003:00010450       waitqueue_active_
 0003:000E8BC0       wctomb_
 0005:00002144       _alsa_fops
 0005:00043AC7       _auto_pin_cfg_labels
 0003:00000050       _CallPDD16
 0002:0000049A       _CallRM
 0005:00001D04       _cardcalls
 0005:0000A214       _card_id_changed
 0005:0000A210       _control_id_changed
 0005:000081D4       _CountWv
 0005:000018EC       _current
 0005:000018C8       _current_task
 0005:000000D8       _DbgInt
 0005:000000FC       _DebugLevel
 0005:0008F5A0       _edata
 0005:0008F5A0       _end
 0005:00000048       _fDebug
 0005:0000A21C       _fInInterrupt
 0005:0000D5DC       _fRewired
 0005:000000D4       _fStrategyInit
 0005:00000044       _fVerbose
 0005:000081DC       _hextab
 0005:0000004C       _idc16_PddHandler
 0005:00001CB4       _iLastError
 0005:00001A92       _iomem_resource
 0005:00001A76       _ioport_resource
 0003:000E8CB0       _ismbblead_
 0005:000017CE       _ISR00
 0005:000017D2       _ISR01
 0005:000017D6       _ISR02
 0005:000017DA       _ISR03
 0005:000017DE       _ISR04
 0005:000017E2       _ISR05
 0005:000017E6       _ISR06
 0005:000017EA       _ISR07
 0005:000018C4       _jiffies
 0000:00000000  Imp  _KernSISData         (KEE.90)
 0005:000081D8       _LockAdd
 0005:000081ED       _MAGIC_COMM_PORT
 0005:00001AAE       _mem_map
 0001:00000060       _MESSAGE_STR
 0005:00001E0C       _midi_port
 0001:00000460       _MSG_TABLE16
 0005:00001770       _MSG_TABLE32
 0005:000000D0       _nrCardsDetected
 0005:00002158       _opened_handles
 0005:00043E68       _opl3_ops
 0005:00002004       _oss_devices
 0005:0000AA9C       _pci_devices
 0005:000081F0       _pcmcaps
 0005:00002150       _pcm_device
 0005:00002148       _per_bytes
 0005:0000214C       _prev_size
 0003:00004177       _printk
 0005:00001CB8       _proc_root
 0003:0000AA5E       _put_user_
 0005:00000038       _rdOffset
 0003:0000024C       _RMAllocResource
 0002:00000204       _RMAllocResource16
 0002:000001C8       _RMAllocResourceOrg
 0003:00000358       _RMCreateAdapter
 0002:000002B6       _RMCreateAdapter16
 0002:0000027A       _RMCreateAdapterOrg
 0003:00000310       _RMCreateDevice
 0002:0000031E       _RMCreateDevice16
 0002:000002E2       _RMCreateDeviceOrg
 0003:000003A0       _RMCreateDriver
 0002:0000047A       _RMCreateDriver16
 0002:00000400       _RMCreateDriverOrg
 0003:000002D0       _RMDeallocResource
 0002:000003BA       _RMDeallocResource16
 0002:00000390       _RMDeallocResourceOrg
 0002:00000374       _RMDestroyDevice16
 0002:0000034A       _RMDestroyDeviceOrg
 0003:000003E0       _RMDestroyDriver
 0002:000004F8       _RMDestroyDriver16
 0002:000004CE       _RMDestroyDriverOrg
 0003:0000044C       _RMDevIDToHandleList
 0002:000005A8       _RMDevIDToHandleList16
 0001:0000005C       _RMFlags
 0003:0000040C       _RMGetNodeInfo
 0002:0000054C       _RMGetNodeInfo16
 0003:000004A0       _RMHandleToResourceHandleList
 0002:0000061C       _RMHandleToResourceHandleList16
 0003:0000028C       _RMModifyResources
 0002:00000252       _RMModifyResources16
 0002:00000228       _RMModifyResourcesOrg
 0001:00000050       _RM_Help0
 0001:00000054       _RM_Help1
 0001:00000058       _RM_Help3
 0005:00043C94       _seq_client_load
 0005:00043CD8       _seq_default_timer_card
 0005:00043CD0       _seq_default_timer_class
 0005:00043CDC       _seq_default_timer_device
 0005:00043CE4       _seq_default_timer_resolution
 0005:00043CD4       _seq_default_timer_sclass
 0005:00043CE0       _seq_default_timer_subdevice
 0005:00000DA8       _snd_cards
 0003:000D6A30       _snd_ctl_add_slave_
 0005:00000AA4       _snd_ecards_limit
 0005:0004380B       _snd_hda_bind_sw
 0005:000437FB       _snd_hda_bind_vol
 0005:00043A67       _snd_hda_pcm_type_name
 0005:00000AA8       _snd_major
 0005:00044098       _snd_opl3_regmap
 0005:00000AB8       _snd_oss_root
 0005:0000059C       _snd_pcm_devices_os2
 0005:0000F0B8       _snd_pcm_f_ops
 0003:0001BBB3       _snd_pcm_hw_params_any_
 0003:0001BD81       _snd_pcm_hw_param_setempty_
 0003:000D0CDC       _snd_pcm_hw_param_set_
 0005:00078F98       _snd_pcm_known_rates
 0003:00021690       _snd_pcm_lib_alloc_vmalloc_buffer_
 0005:0000EFF4       _snd_pcm_link_rwlock
 0005:00000AB4       _snd_seq_root
 0005:00008210       _substream_int
 0005:000018F0       _system_utsname
 0005:00001BB2       _szLastALSAError1
 0005:00001C33       _szLastALSAError2
 0005:00001C32       _szOverrunTest1
 0005:00001CB3       _szOverrunTest2
 0005:00000040       _szprintBuf
 0005:00001F78       _szRecSources
 0005:00001AB2       _this_module
 0005:000017C8       _TimerHandler16
 0005:000017F8       _TKSSBase
 0005:00002154       _total
 0005:00000104       _ulget_free_pagesMemUsed
 0005:0000A218       _unlock_all
 0005:00043E64       _use_internal_drums
 0005:0000003C       _wrOffset
 0005:000629D4       __AccessFHeap
 0005:000629C0       __AccessFileH
 0005:000629C8       __AccessIOB
 0005:000629D0       __AccessNHeap
 0005:000629E0       __AccessTDList
 0005:00062A4C       __amblksiz
 0005:00062A24       __ASTACKPTR
 0005:00062A20       __ASTACKSIZ
 0003:000E8A40       __Bits
 0005:00062A28       __cbyte
 0005:00062A2C       __cbyte2
 0003:00004235       __check_region_
 0005:00062A30       __child
 0003:000E8FA0       __CommonInit_
 0003:0000E048       __compat_get_order_
 0003:0000A8A5       __copy_user_
 0003:0000A955       __copy_user_zeroing_
 0005:000629FC       __curbrk
 0000:00001234  Abs  __DOSseg__
 0005:000629F8       __dynend
 0005:0007F53E       __End_XI
 0005:0007F53E       __End_YI
 0003:000E90E0       __EnterWVIDEO_
 0005:00062A36       __Envptr
 0005:00062A3A       __Envseg
 0003:000E8B76       __exit_
 0003:000E8E70       __exit_with_msg_
 0003:000E8EC0       __fatal_runtime_error_
 0003:000E89D0       __FDFS
 0003:000E8F40       __FiniRtns
 0003:00000000       __GETDS
 0003:0000A34B       __get_free_dma_pages_
 0003:0000A4D5       __get_free_pages_
 0003:0000A9FA       __get_user_
 0003:000E6795       __I8LS
 0003:000E67B0       __I8M
 0003:000E677A       __I8RS
 0003:000E8EF0       __InitRtns
 0003:0000A799       __ioremap_
 0003:000E6D00       __IsTable
 0003:0000AB0D       __kfree_
 0003:0000AAA2       __kmalloc_
 0005:00062A00       __LpCmdLine
 0005:00062A08       __LpDllName
 0005:00062A04       __LpPgmName
 0005:00062A0C       __LpwCmdLine
 0005:00062A14       __LpwDllName
 0005:00062A10       __LpwPgmName
 0003:000E8FE5       __mbinit_
 0005:00062A34       __no87
 0005:0007F590       __nullarea
 0003:00000000       __OffBeginCS32
 0005:00000000       __OffBeginDS32
 0002:000006DB       __OffFinalCS16
 0003:000E9108       __OffFinalCS32
 0001:0000048B       __OffFinalDS16
 0005:0007F534       __OffFinalDS32
 0005:0000176C       __OffsetFinalCS16
 0005:0000176E       __OffsetFinalDS16
 0003:000E8B59       __OS2Fini_
 0003:000E8B1B       __OS2Init_
 0003:000E8AAC       __OS2MainInit_
 0005:00062A3C       __osmajor
 0005:00062A3D       __osminor
 0003:000E7C90       __prtf_
 0005:000629DC       __ReleaseFHeap
 0005:000629C4       __ReleaseFileH
 0005:000629CC       __ReleaseIOB
 0005:000629D8       __ReleaseNHeap
 0005:000629E4       __ReleaseTDList
 0003:0000D7AA       __release_region_
 0003:0000D698       __request_region_
 0003:000E7A20       __scnf_
 0003:000E89B1       __set_doserrno_
 0003:000E8982       __set_EDOM_
 0003:000E899E       __set_EINVAL_
 0003:000E8990       __set_ERANGE_
 0003:000E8974       __set_errno_
 0003:000E8B61       __shutdown_stack_checking_
 0003:000E6508       __snd_util_memblk_new_
 0003:000E6427       __snd_util_mem_alloc_
 0003:000E6609       __snd_util_mem_free_
 0005:00062A18       __STACKLOW
 0005:00062A1C       __STACKTOP
 0005:0007F538       __Start_XI
 0005:0007F53E       __Start_YI
 0003:000E6E10       __STOSB
 0003:000E6E47       __STOSD
 0003:000E8AA3       __threadid_
 0003:000E8A9C       __threadstack_
 0005:000629F0       __threadstksize
 0003:000E6795       __U8LS
 0003:000E67B0       __U8M
 0003:000E6760       __U8RS
 0003:00003E1F       __udelay_
 0003:00010401       __wake_up_
 0003:000034E6       __wcpp_2_pure_error__
 0003:000034B4       __wcpp_2_undefed_cdtor__
 0003:000034CD       __wcpp_2_undefined_member_function__
 0003:000034FF       __wcpp_2_undef_vfun__
 0003:0000354A       __wcpp_4_pure_error__
 0003:00003518       __wcpp_4_undefed_cdtor__
 0003:00003531       __wcpp_4_undefined_member_function__
 0003:00003563       __wcpp_4_undef_vfun__
 0005:00076178       ___Alphabet
 0004:00000003       ___begtext
 0005:000629B0       ___EFG_printf
 0005:000629B4       ___EFG_scanf
 0005:000632A2       ___exitcall_alsa_ac97_exit
 0005:00055670       ___exitcall_alsa_card_ali_exit
 0005:0000F5E8       ___exitcall_alsa_card_als4000_exit
 0005:00010698       ___exitcall_alsa_card_atiixp_exit
 0005:000436A8       ___exitcall_alsa_card_azx_exit
 0005:0000F484       ___exitcall_alsa_card_bt87x_exit
 0005:00013B14       ___exitcall_alsa_card_ca0106_exit
 0005:00010369       ___exitcall_alsa_card_cmipci_exit
 0005:00013234       ___exitcall_alsa_card_cs4281_exit
 0005:0004418C       ___exitcall_alsa_card_cs46xx_exit
 0005:00051E14       ___exitcall_alsa_card_cs5535audio_exit
 0005:00052010       ___exitcall_alsa_card_emu10k1_exit
 0005:00013660       ___exitcall_alsa_card_ens137x_exit
 0005:00012F99       ___exitcall_alsa_card_es1938_exit
 0005:00012738       ___exitcall_alsa_card_es1968_exit
 0005:00010B04       ___exitcall_alsa_card_fm801_exit
 0005:000124F4       ___exitcall_alsa_card_intel8x0_exit
 0005:000117C4       ___exitcall_alsa_card_m3_exit
 0005:000623D4       ___exitcall_alsa_card_nm256_exit
 0005:0005573C       ___exitcall_alsa_card_trident_exit
 0005:0001117C       ___exitcall_alsa_card_via82xx_exit
 0005:00054CE8       ___exitcall_alsa_card_ymfpci_exit
 0005:0000EA48       ___exitcall_alsa_hwdep_exit
 0005:000440E0       ___exitcall_alsa_mpu401_uart_exit
 0005:00043F04       ___exitcall_alsa_opl3_exit
 0005:00043E90       ___exitcall_alsa_opl3_seq_exit
 0005:0000EF14       ___exitcall_alsa_pcm_exit
 0005:00062920       ___exitcall_alsa_pcm_oss_exit
 0005:0000EB84       ___exitcall_alsa_rawmidi_exit
 0005:000628A0       ___exitcall_alsa_sb_common_exit
 0005:00043D14       ___exitcall_alsa_seq_device_exit
 0005:00043CEC       ___exitcall_alsa_seq_exit
 0005:000633CC       ___exitcall_alsa_seq_midi_emul_exit
 0005:0000EF70       ___exitcall_alsa_sound_exit
 0005:0000EAF4       ___exitcall_alsa_timer_exit
 0005:000633D4       ___exitcall_alsa_util_mem_exit
 0005:00023834       ___exitcall_patch_analog_exit
 0005:000194E0       ___exitcall_patch_atihdmi_exit
 0005:00023FD8       ___exitcall_patch_cmedia_exit
 0005:00019380       ___exitcall_patch_conexant_exit
 0005:00043367       ___exitcall_patch_realtek_exit
 0005:0001BFD4       ___exitcall_patch_sigmatel_exit
 0005:00016B94       ___exitcall_patch_via_exit
 0005:0000F1C8       ___exitcall_snd_mem_exit
 0005:000629B8       ___FirstThreadData
 0005:00062A3E       ___FPE_handler
 0005:000629BC       ___GetThreadPtr
 0005:00001730       ___hmodule
 0005:0006329E       ___initcall_alsa_ac97_init
 0005:0005566C       ___initcall_alsa_card_ali_init
 0005:0000F5E4       ___initcall_alsa_card_als4000_init
 0005:00010694       ___initcall_alsa_card_atiixp_init
 0005:000436A4       ___initcall_alsa_card_azx_init
 0005:0000F480       ___initcall_alsa_card_bt87x_init
 0005:00013B10       ___initcall_alsa_card_ca0106_init
 0005:00010365       ___initcall_alsa_card_cmipci_init
 0005:00013230       ___initcall_alsa_card_cs4281_init
 0005:00044188       ___initcall_alsa_card_cs46xx_init
 0005:00051E10       ___initcall_alsa_card_cs5535audio_init
 0005:0005200C       ___initcall_alsa_card_emu10k1_init
 0005:0001365C       ___initcall_alsa_card_ens137x_init
 0005:00012F95       ___initcall_alsa_card_es1938_init
 0005:00012734       ___initcall_alsa_card_es1968_init
 0005:00010B00       ___initcall_alsa_card_fm801_init
 0005:000124F0       ___initcall_alsa_card_intel8x0_init
 0005:000117C0       ___initcall_alsa_card_m3_init
 0005:000623D0       ___initcall_alsa_card_nm256_init
 0005:00055738       ___initcall_alsa_card_trident_init
 0005:00011178       ___initcall_alsa_card_via82xx_init
 0005:00054CE4       ___initcall_alsa_card_ymfpci_init
 0005:0000EA44       ___initcall_alsa_hwdep_init
 0005:000440DC       ___initcall_alsa_mpu401_uart_init
 0005:00043F00       ___initcall_alsa_opl3_init
 0005:00043E8C       ___initcall_alsa_opl3_seq_init
 0005:0000EF10       ___initcall_alsa_pcm_init
 0005:0006291C       ___initcall_alsa_pcm_oss_init
 0005:0000EB80       ___initcall_alsa_rawmidi_init
 0005:0006289C       ___initcall_alsa_sb_common_init
 0005:00043D10       ___initcall_alsa_seq_device_init
 0005:00043CE8       ___initcall_alsa_seq_init
 0005:000633C8       ___initcall_alsa_seq_midi_emul_init
 0005:0000EF6C       ___initcall_alsa_sound_init
 0005:0000EAF0       ___initcall_alsa_timer_init
 0005:000633D0       ___initcall_alsa_util_mem_init
 0005:00023830       ___initcall_patch_analog_init
 0005:000194DC       ___initcall_patch_atihdmi_init
 0005:00023FD4       ___initcall_patch_cmedia_init
 0005:0001937C       ___initcall_patch_conexant_init
 0005:00043363       ___initcall_patch_realtek_init
 0005:0001BFD0       ___initcall_patch_sigmatel_init
 0005:00016B90       ___initcall_patch_via_init
 0005:0000F1C4       ___initcall_snd_mem_init
 0005:0000172C       ___IsDBCS
 0005:00001520       ___Is_DLL
 0005:00062A44       ___MBCodePage
 0005:00001628       ___MBCSIsTable
 0005:000629F4       ___process_fini
 0005:00001524       ___saved_CS
 0005:000629EC       ___sig_fini_rtn
 0005:000629E8       ___sig_init_rtn
 0005:00062A48       ___WD_Present


 Address         Publics by Value
 0000:00000000  Imp  DosQuerySysInfo      (DOSCALLS.348)
 0000:00000000  Imp  KernLinToPageList    (KEE.64)
 0000:00000000  Imp  KernSelToFlat        (KEE.66)
 0000:00000000  Imp  KernThunkStackTo32   (KEE.41)
 0000:00000000  Imp  KernThunkStackTo16   (KEE.40)
 0000:00000000  Imp  DOSOPEN              (DOSCALLS.70)
 0000:00000000  Imp  _KernSISData         (KEE.90)
 0000:00000000  Imp  DosQueryCp           (DOSCALLS.291)
 0000:00000000  Imp  KernVMFree           (KEE.61)
 0000:00000000  Imp  DosExit              (DOSCALLS.234)
 0000:00000000  Imp  DOSCLOSE             (DOSCALLS.59)
 0000:00000000  Imp  DosWrite             (DOSCALLS.282)
 0000:00000000  Imp  KernVMAlloc          (KEE.60)
 0000:00000000  Imp  DOS32FLATDS          (DOSCALLS.370)
 0000:00000000  Imp  DOSWRITE             (DOSCALLS.138)
 0000:00000000  Imp  KernVMLock           (KEE.62)
 0000:00000000  Imp  DOSIODELAYCNT        (DOSCALLS.427)
 0000:00000000  Imp  DosQueryDBCSEnv      (NLS.6)
 0000:00001234  Abs  __DOSseg__
 0001:00000000       help_header
 0001:0000001E       uniaud_header
 0001:0000003C       DevHelpInit
 0001:00000040       fOpen
 0001:00000044       InitPktSeg
 0001:00000046       InitPktOff
 0001:00000048       DbgU32TimerCnt
 0001:0000004C       DbgU32IntCnt
 0001:00000050       _RM_Help0
 0001:00000054       _RM_Help1
 0001:00000058       _RM_Help3
 0001:0000005C       _RMFlags
 0001:00000060       _MESSAGE_STR
 0001:00000460       _MSG_TABLE16
 0001:00000466       pddname16
 0001:0000046D       FileName
 0001:0000048B       __OffFinalDS16
 0002:00000000       help_stub_strategy
 0002:00000096       uniaud_stub_strategy
 0002:0000010A       uniaud_stub_idc
 0002:00000128       uniaud_stub_timer
 0002:000001A0       thunk3216_devhelp
 0002:000001B2       thunk3216_devhelp_modified_ds
 0002:000001C8       _RMAllocResourceOrg
 0002:00000204       _RMAllocResource16
 0002:00000228       _RMModifyResourcesOrg
 0002:00000252       _RMModifyResources16
 0002:0000027A       _RMCreateAdapterOrg
 0002:000002B6       _RMCreateAdapter16
 0002:000002E2       _RMCreateDeviceOrg
 0002:0000031E       _RMCreateDevice16
 0002:0000034A       _RMDestroyDeviceOrg
 0002:00000374       _RMDestroyDevice16
 0002:00000390       _RMDeallocResourceOrg
 0002:000003BA       _RMDeallocResource16
 0002:000003DA       MY_DEVHELP_ATTACHDD
 0002:00000400       _RMCreateDriverOrg
 0002:0000047A       _RMCreateDriver16
 0002:0000049A       _CallRM
 0002:000004CE       _RMDestroyDriverOrg
 0002:000004F8       _RMDestroyDriver16
 0002:0000054C       _RMGetNodeInfo16
 0002:000005A8       _RMDevIDToHandleList16
 0002:0000061C       _RMHandleToResourceHandleList16
 0002:000006DB       __OffFinalCS16
 0003:00000000       __GETDS
 0003:00000000       __OffBeginCS32
 0003:00000010       DevHlp
 0003:00000024       thunk1632_devhelp
 0003:00000030       DevHlp_ModifiedDS
 0003:00000044       thunk1632_devhelp_modified_ds
 0003:00000050       _CallPDD16
 0003:00000080       STRATEGY_
 0003:000000E0       IDC_
 0003:00000140       TIMER_
 0003:0000024C       _RMAllocResource
 0003:0000028C       _RMModifyResources
 0003:000002D0       _RMDeallocResource
 0003:00000310       _RMCreateDevice
 0003:00000358       _RMCreateAdapter
 0003:000003A0       _RMCreateDriver
 0003:000003E0       _RMDestroyDriver
 0003:0000040C       _RMGetNodeInfo
 0003:0000044C       _RMDevIDToHandleList
 0003:000004A0       _RMHandleToResourceHandleList
 0003:000004DD       W?StratOpen$n(pf$RP$$)ul
 0003:00000544       W?StratInit$n(pf$RP$$)ul
 0003:000005AE       W?StratInitComplete$n(pf$RP$$)ul
 0003:000005E9       W?StratShutdown$n(pf$RP$$)ul
 0003:00000656       ALSA_STRATEGY
 0003:000006D8       W?StratRead$n(pf$RP$$)ul
 0003:0000084E       W?DevSaveMessage$n(pfai)v
 0003:0000090D       W?LockSegments$n()i
 0003:00000A0D       W?DiscardableInit$n(pf$RPInit$$)ul
 0003:00000E1D       W?toupper$n(i)i
 0003:00000E5D       W?mymemchr$n(pfaaus)pfa
 0003:00000EDC       W?sz2us$n(pfai)us
 0003:00000FC7       W?IsWhitespace$n(a)i
 0003:00001018       W?SkipWhite$n(pfa)pfa
 0003:00001096       W?CheckCardName$n(pfa)v
 0003:00001313       W?DoParm$n(apfa)i
 0003:0000140E       W?ParseParm$n(pfai)i
 0003:00001513       GetParms_
 0003:00001624       GetTKSSBase
 0003:00001664       iodelay32_
 0003:00001672       ALSA_IDC
 0003:000016FC       W?OSS32IDC$n(ulpn$__6ikc0pIDC32_PACKET$$)ul
 0003:00001CB3       W?StratIOCtl$n(pf$RP$$)ul
 0003:0000288A       W?StratClose$n(pf$RP$$)ul
 0003:000028EC       RMInit_
 0003:00002A9B       RMRequestIO_
 0003:00002B8B       RMRequestMem_
 0003:00002C6E       RMRequestIRQ_
 0003:00002DB4       RMDeallocateIRQ_
 0003:00002E2D       RMDone_
 0003:000032FA       RMSetHandles_
 0003:00003326       ALSA_SetIrq_
 0003:00003409       ALSA_FreeIrq_
 0003:00003451       ALSA_Interrupt
 0003:000034B4       __wcpp_2_undefed_cdtor__
 0003:000034CD       __wcpp_2_undefined_member_function__
 0003:000034E6       __wcpp_2_pure_error__
 0003:000034FF       __wcpp_2_undef_vfun__
 0003:00003518       __wcpp_4_undefed_cdtor__
 0003:00003531       __wcpp_4_undefined_member_function__
 0003:0000354A       __wcpp_4_pure_error__
 0003:00003563       __wcpp_4_undef_vfun__
 0003:0000357C       W?$nwn(ui)pnv
 0003:000035A5       W?$dln(pnv)v
 0003:000035C8       W?$nwn(uipnv)pnv
 0003:00003602       os2gettimesec_
 0003:00003625       os2gettimemsec_
 0003:00003947       vsprintf_
 0003:00003D2D       sprintf_
 0003:00003D6C       ALSA_TIMER_
 0003:00003DCA       schedule_timeout_
 0003:00003E1F       __udelay_
 0003:00003E51       mdelay_
 0003:00003E85       do_gettimeofday_
 0003:00003ED1       add_timer_
 0003:00003EEC       del_timer_
 0003:00003F11       mod_timer_
 0003:00003F2D       msleep_
 0003:00003F70       strcmp_
 0003:00003FCD       strncmp_
 0003:0000403C       tasklet_hi_schedule_
 0003:00004074       tasklet_init_
 0003:000040B6       OSS32_SetFileId_
 0003:00004177       _printk
 0003:00004200       schedule_
 0003:00004218       poll_wait_
 0003:00004235       __check_region_
 0003:0000425C       hweight32_
 0003:000042F6       create_proc_entry_
 0003:00004356       remove_proc_entry_
 0003:00004372       proc_register_
 0003:00004398       proc_unregister_
 0003:000043BE       fasync_helper_
 0003:000043E6       kill_fasync_
 0003:00004403       request_dma_
 0003:00004429       free_dma_
 0003:00004444       enable_dma_
 0003:0000445F       disable_dma_
 0003:0000447A       register_reboot_notifier_
 0003:0000449F       unregister_reboot_notifier_
 0003:0000453B       queue_work_
 0003:00004650       flush_workqueue_
 0003:000046BD       create_workqueue_
 0003:00004747       destroy_workqueue_
 0003:0000476A       kstrdup_
 0003:000047DC       mod_firmware_load_
 0003:00004882       request_firmware_
 0003:0000492C       release_firmware_
 0003:00004960       memdup_user_
 0003:000049DF       cancel_delayed_work_
 0003:00004A2B       schedule_work_
 0003:00004A9A       queue_delayed_work_
 0003:00004B1D       gcd_
 0003:00004B7B       strict_strtoul_
 0003:00004C1B       W?CallOSS16$n(ululul)ul
 0003:00004C83       OSS32_Initialize_
 0003:00004F48       OSS32_Shutdown_
 0003:00004FE5       OSS32_ProcessIRQ_
 0003:00005011       OSS32_ProcessMIDIIRQ_
 0003:00005041       OSS32_CloseUNI16_
 0003:0000506D       MyDevBlock_
 0003:000050BF       OSS32_DebugString_
 0003:000050F6       OSS32_MidiOpen_
 0003:000055AD       OSS32_MidiClose_
 0003:00005755       OSS32_MidiWrite_
 0003:0000578D       OSS32_MidiRead_
 0003:00005841       OSS32_MidiQueryCaps_
 0003:00005879       OSS32_MidiCommand_
 0003:00005A5C       ConvertVolume_
 0003:00005AA9       OSS32_MixOpen_
 0003:00006191       OSS32_MixClose_
 0003:00006221       OSS32_MixGetVolume_
 0003:00006272       OSS32_MixSetVolume_
 0003:0000675D       OSS32_MixSetProperty_
 0003:00006C03       OSS32_MixGetProperty_
 0003:00006C54       OSSToALSAVolume_
 0003:00006DD3       OSS32_MixQueryCaps_
 0003:00006EB9       OSS32_MixQueryName_
 0003:00007017       OSS32_QueryNames_
 0003:0000720D       register_chrdev_
 0003:0000724D       unregister_chrdev_
 0003:0000728E       register_sound_special_
 0003:000072E0       register_sound_mixer_
 0003:00007332       register_sound_midi_
 0003:00007384       register_sound_dsp_
 0003:000073D6       register_sound_synth_
 0003:00007428       unregister_sound_special_
 0003:00007454       unregister_sound_mixer_
 0003:00007480       unregister_sound_midi_
 0003:000074AC       unregister_sound_dsp_
 0003:000074D8       unregister_sound_synth_
 0003:00007504       UNIXToOSSError_
 0003:00007681       ALSAToOSSDataType_
 0003:00007776       ALSAToOSSRateFlags_
 0003:00007865       OSS32_QueryDevCaps_
 0003:00007E0D       OSS32_WaveOpen_
 0003:000080EA       OSS32_WaveClose_
 0003:00008271       OSS32_WavePrepare_
 0003:0000831B       OSS32_WaveStart_
 0003:000083A9       OSS32_WaveStop_
 0003:00008437       OSS32_WavePause_
 0003:000084C5       OSS32_WaveResume_
 0003:00008556       OSS32_WaveSetHwParams_
 0003:000091B9       OSS32_WaveAddBuffer_
 0003:000094C8       OSS32_WaveGetPosition_
 0003:000095A9       OSS32_WaveGetSpace_
 0003:00009657       OSS32_WaveGetHwPtr_
 0003:000096FD       OSS32_WaveGetStatus_
 0003:0000979D       OSS32_WaveSetVolume_
 0003:00009861       DecLongToASCII_
 0003:000099CE       HexLongToASCII_
 0003:00009B43       CharOut_
 0003:00009B89       StringOut_
 0003:00009D11       snd_iprintf_
 0003:0000A01D       DbgPrintIrq_
 0003:0000A067       AddBaseAddress_
 0003:0000A0CB       GetBaseAddress_
 0003:0000A1A1       virt_to_phys_
 0003:0000A1EB       phys_to_virt_
 0003:0000A24A       VMAlloc_
 0003:0000A314       VMFree_
 0003:0000A34B       __get_free_dma_pages_
 0003:0000A4D5       __get_free_pages_
 0003:0000A63D       free_pages_
 0003:0000A68F       vmalloc_
 0003:0000A707       vfree_
 0003:0000A74B       alloc_pages_
 0003:0000A771       remap_page_range_
 0003:0000A799       __ioremap_
 0003:0000A84C       iounmap_
 0003:0000A87E       is_access_ok_
 0003:0000A8A5       __copy_user_
 0003:0000A8F1       copy_to_user_
 0003:0000A955       __copy_user_zeroing_
 0003:0000A996       copy_from_user_
 0003:0000A9FA       __get_user_
 0003:0000AA5E       _put_user_
 0003:0000AAA2       __kmalloc_
 0003:0000AB0D       __kfree_
 0003:0000AB54       kzalloc_
 0003:0000AB9A       kcalloc_
 0003:0000ABEC       uniaud_set_interrupted_substream_
 0003:0000AC52       WaitForControlChange_
 0003:0000ACEB       WaitForPCMInterrupt_
 0003:0000AE57       GetNumberOfCards_
 0003:0000AE7A       GetNumberOfPcm_
 0003:0000AEA3       SetPCMInstance_
 0003:0000AEEF       GetPcmForChannels_
 0003:0000AFD1       GetMaxChannels_
 0003:0000B0BA       GetUniaudPcmCaps1_
 0003:0000B5FC       FillCaps_
 0003:0000B692       GetUniaudPcmCaps_
 0003:0000B708       UniaudCtlGetPowerState_
 0003:0000B824       UniaudCtlSetPowerState_
 0003:0000B940       GetUniaudCardInfo_
 0003:0000BA8C       GetUniaudControlNum_
 0003:0000BC81       GetUniaudControls_
 0003:0000BEF2       GetUniaudControlInfo_
 0003:0000C063       GetUniaudControlValueGet_
 0003:0000C1D4       GetUniaudControlValuePut_
 0003:0000C345       UniaudIoctlHWRefine_
 0003:0000C3C5       UniaudIoctlHWParamSet_
 0003:0000C445       UniaudIoctlSWParamSet_
 0003:0000C4C5       UniaudIoctlPCMStatus_
 0003:0000C53E       UniaudIoctlPCMWrite_
 0003:0000C5B0       UniaudIoctlPCMRead_
 0003:0000C622       UniaudIoctlPCMPrepare_
 0003:0000C684       UniaudIoctlPCMResume_
 0003:0000C6E8       UniaudIoctlPCMStart_
 0003:0000C74A       UniaudIoctlPCMDrop_
 0003:0000C7AC       UniaudCloseAll_
 0003:0000C8C2       request_irq_
 0003:0000CA9B       free_irq_
 0003:0000CBA6       eoi_irq_
 0003:0000CBD2       process_interrupt_
 0003:0000CD2B       in_interrupt_
 0003:0000CD4E       disable_irq_
 0003:0000CD7B       pci_read_config_byte_
 0003:0000CDE7       pci_read_config_word_
 0003:0000CE55       pci_read_config_dword_
 0003:0000CEBA       pci_write_config_byte_
 0003:0000CF22       pci_write_config_word_
 0003:0000CF8B       pci_write_config_dword_
 0003:0000CFEB       pcidev_prepare_
 0003:0000D022       pcidev_activate_
 0003:0000D059       pcidev_deactivate_
 0003:0000D591       pci_find_device_
 0003:0000D698       __request_region_
 0003:0000D7AA       __release_region_
 0003:0000D821       pci_get_flags_
 0003:0000D86F       pcibios_present_
 0003:0000D89F       pci_find_slot_
 0003:0000D8DB       pci_dma_supported_
 0003:0000D90F       pci_find_capability_
 0003:0000D9C7       pci_set_power_state_
 0003:0000DB94       pci_enable_device_
 0003:0000DBFC       pci_register_driver_
 0003:0000DDF8       pci_module_init_
 0003:0000DE36       pci_unregister_driver_
 0003:0000DF8E       pci_set_master_
 0003:0000DFEA       pm_register_
 0003:0000E01F       pm_unregister_
 0003:0000E048       __compat_get_order_
 0003:0000E08C       pci_alloc_consistent_
 0003:0000E1BA       pci_free_consistent_
 0003:0000E1EC       pci_set_driver_data_
 0003:0000E21A       pci_get_driver_data_
 0003:0000E253       pci_get_dma_mask_
 0003:0000E28C       release_resource_
 0003:0000E2B1       pci_set_latency_time_
 0003:0000E2E9       pci_orig_save_state_
 0003:0000E341       pci_orig_restore_state_
 0003:0000E3E8       pci_save_state_
 0003:0000E469       pci_restore_state_
 0003:0000E4ED       pci_disable_device_
 0003:0000E537       pci_request_region_
 0003:0000EF93       pci_release_region_
 0003:0000F424       pci_request_regions_
 0003:0000F493       pci_release_regions_
 0003:0000F4CE       pci_match_device_
 0003:0000F5CC       snd_pci_dev_present_
 0003:0000F683       snd_pci_compat_get_pci_driver_
 0003:0000F6C4       OSS32_APMResume_
 0003:0000F771       OSS32_APMSuspend_
 0003:0000F831       PciAdjustInterrupts_
 0003:0000F9A0       W?dumpheap$n()v
 0003:0000FAE3       W?SignatureCheck$n(pn$_MEMBLOCK$$pna)s
 0003:0000FB8D       W?HeapCheck$n(pna)v
 0003:0000FCA5       W?npvAllocateBlock$n(pn$_MEMBLOCK$$ulpn$1$)pnv
 0003:0000FD98       W?malloc$n(ul)pnv
 0003:0000FE8F       W?remove$n(pn$_MEMBLOCK$$)v
 0003:0000FEF8       W?compact$n()v
 0003:0000FFC0       W?free$n(pnv)v
 0003:000100C2       W?_memfree$n()ui
 0003:000100E5       W?_msize$n(pnv)ui
 0003:00010124       W?realloc$n(pnvul)pnv
 0003:000101D1       W?IsHeapAddr$n(ul)ul
 0003:00010227       W?HeapInit$n(ul)ul
 0003:000102CF       strncpy_
 0003:00010336       init_waitqueue_head_
 0003:00010351       add_wait_queue_
 0003:0001036D       add_wait_queue_exclusive_
 0003:00010388       remove_wait_queue_
 0003:000103A4       interruptible_sleep_on_timeout_
 0003:000103D8       interruptible_sleep_on_
 0003:00010401       __wake_up_
 0003:00010434       init_waitqueue_entry_
 0003:00010450       waitqueue_active_
 0003:00010475       spin_lock_init_
 0003:00010499       spin_lock_
 0003:000104BE       spin_lock_flag_
 0003:000104E4       spin_trylock_
 0003:00010509       spin_unlock_
 0003:00010FC1       snd_hwdep_new_
 0003:00011AE0       snd_timer_open_
 0003:00011D60       snd_timer_close_
 0003:00011FF3       snd_timer_resolution_
 0003:00012301       snd_timer_start_
 0003:00012535       snd_timer_stop_
 0003:000125B5       snd_timer_continue_
 0003:0001267F       snd_timer_pause_
 0003:00012880       snd_timer_interrupt_
 0003:00012D17       snd_timer_new_
 0003:0001326D       snd_timer_notify_
 0003:000133AC       snd_timer_global_new_
 0003:00013401       snd_timer_global_free_
 0003:0001342A       snd_timer_global_register_
 0003:000159C8       snd_rawmidi_drop_output_
 0003:00015A41       snd_rawmidi_drain_output_
 0003:00015B15       snd_rawmidi_drain_input_
 0003:00015E49       snd_rawmidi_kernel_open_
 0003:0001646A       snd_rawmidi_kernel_release_
 0003:0001666D       snd_rawmidi_info_select_
 0003:00016832       snd_rawmidi_output_params_
 0003:0001697D       snd_rawmidi_input_params_
 0003:00016B88       snd_rawmidi_receive_
 0003:00016F40       snd_rawmidi_kernel_read_
 0003:0001716A       snd_rawmidi_transmit_empty_
 0003:000171F4       snd_rawmidi_transmit_peek_
 0003:0001735B       snd_rawmidi_transmit_ack_
 0003:0001745C       snd_rawmidi_transmit_
 0003:000176C4       snd_rawmidi_kernel_write_
 0003:00017D64       snd_rawmidi_new_
 0003:00018591       snd_rawmidi_set_ops_
 0003:000186EE       snd_pcm_format_signed_
 0003:00018746       snd_pcm_format_unsigned_
 0003:00018799       snd_pcm_format_linear_
 0003:000187D9       snd_pcm_format_little_endian_
 0003:00018831       snd_pcm_format_big_endian_
 0003:00018884       snd_pcm_format_width_
 0003:000188DB       snd_pcm_format_physical_width_
 0003:00018932       snd_pcm_format_size_
 0003:00018978       snd_pcm_format_silence_64_
 0003:000189D2       snd_pcm_format_set_silence_
 0003:00018B92       snd_pcm_limit_hw_rates_
 0003:00018C47       snd_pcm_rate_to_rate_bit_
 0003:000195C0       snd_pcm_playback_silence_
 0003:00019A89       snd_pcm_update_state_
 0003:00019E4F       snd_pcm_update_hw_ptr_
 0003:00019E7A       snd_pcm_set_ops_
 0003:00019ECC       snd_pcm_set_sync_
 0003:0001A0F2       snd_interval_refine_
 0003:0001A3D1       snd_interval_mul_
 0003:0001A52D       snd_interval_div_
 0003:0001A682       snd_interval_muldivk_
 0003:0001A7BF       snd_interval_mulkdiv_
 0003:0001A91B       snd_interval_ratnum_
 0003:0001B01B       snd_interval_list_
 0003:0001B1CE       snd_pcm_hw_rule_add_
 0003:0001B346       snd_pcm_hw_constraint_mask_
 0003:0001B3C3       snd_pcm_hw_constraint_mask64_
 0003:0001B468       snd_pcm_hw_constraint_integer_
 0003:0001B4C0       snd_pcm_hw_constraint_minmax_
 0003:0001B5CB       snd_pcm_hw_constraint_list_
 0003:0001B6D5       snd_pcm_hw_constraint_ratnums_
 0003:0001B7DF       snd_pcm_hw_constraint_ratdens_
 0003:0001B8C4       snd_pcm_hw_constraint_msbits_
 0003:0001B982       snd_pcm_hw_constraint_step_
 0003:0001BA39       snd_pcm_hw_constraint_pow2_
 0003:0001BBB3       _snd_pcm_hw_params_any_
 0003:0001BC2A       snd_pcm_hw_param_value_
 0003:0001BD81       _snd_pcm_hw_param_setempty_
 0003:0001BFD7       snd_pcm_hw_param_first_
 0003:0001C175       snd_pcm_hw_param_last_
 0003:0001C1FA       snd_pcm_hw_params_choose_
 0003:0001C500       snd_pcm_lib_ioctl_
 0003:0001C582       snd_pcm_period_elapsed_
 0003:0001CD5C       snd_pcm_lib_write_
 0003:0001D01F       snd_pcm_lib_writev_
 0003:0001D543       snd_pcm_lib_read_
 0003:0001D79C       snd_pcm_lib_readv_
 0003:0001DD07       snd_pcm_format_name_
 0003:0001DD34       snd_pcm_new_stream_
 0003:0001DFA9       snd_pcm_new_
 0003:0001E27A       snd_pcm_attach_substream_
 0003:0001E6B6       snd_pcm_detach_substream_
 0003:0001EAF1       snd_pcm_notify_
 0003:0001ED76       pcm_info_
 0003:0001EE5B       pcm_instances_
 0003:0001EF31       snd_lookup_minor_data_
 0003:0001F1B8       snd_register_device_for_dev_
 0003:0001F378       snd_unregister_device_
 0003:0001F3FE       snd_add_device_sysfs_file_
 0003:0001F5B3       snd_minor_info_init_
 0003:0001F61C       snd_minor_info_done_
 0003:0001F797       snd_info_check_reserved_words_
 0003:000204EA       snd_info_init_
 0003:000205F6       snd_info_done_
 0003:00020678       snd_info_card_create_
 0003:0002072C       snd_info_card_register_
 0003:00020792       snd_info_card_id_change_
 0003:00020802       snd_info_card_disconnect_
 0003:00020894       snd_info_card_free_
 0003:000208E3       snd_info_get_line_
 0003:000209ED       snd_info_get_str_
 0003:00020BB0       snd_info_create_module_entry_
 0003:00020BF9       snd_info_create_card_entry_
 0003:00020D81       snd_card_proc_new_
 0003:00020E0A       snd_info_free_entry_
 0003:00020E76       snd_info_register_
 0003:000211D4       snd_pcm_lib_preallocate_free_
 0003:00021201       snd_pcm_lib_preallocate_free_for_all_
 0003:000212E2       snd_pcm_lib_preallocate_pages_
 0003:00021328       snd_pcm_lib_preallocate_pages_for_all_
 0003:000213AE       snd_pcm_sgbuf_ops_page_
 0003:0002140F       snd_pcm_sgbuf_get_chunk_size_
 0003:000214B3       snd_pcm_lib_malloc_pages_
 0003:000215F8       snd_pcm_lib_free_pages_
 0003:00021690       _snd_pcm_lib_alloc_vmalloc_buffer_
 0003:00021746       snd_pcm_lib_free_vmalloc_buffer_
 0003:000217AD       snd_pcm_timer_resolution_change_
 0003:000219C4       snd_pcm_timer_init_
 0003:00021ADF       snd_pcm_timer_done_
 0003:000223D5       snd_pcm_info_
 0003:00022510       snd_pcm_info_user_
 0003:0002258D       snd_pcm_hw_refine_
 0003:000237A6       snd_pcm_status_
 0003:00024218       snd_pcm_start_
 0003:00024376       snd_pcm_stop_
 0003:000243A8       snd_pcm_drain_done_
 0003:00024727       snd_pcm_suspend_
 0003:0002479D       snd_pcm_suspend_all_
 0003:00025E67       snd_pcm_hw_constraints_init_
 0003:00026409       snd_pcm_hw_constraints_complete_
 0003:000266D1       snd_pcm_release_substream_
 0003:00026772       snd_pcm_open_substream_
 0003:00028194       snd_pcm_kernel_ioctl_
 0003:00028768       snd_oss_info_register_
 0003:00028A01       snd_info_minor_register_
 0003:00028A7F       snd_info_minor_unregister_
 0003:00028AB5       snd_lookup_oss_minor_data_
 0003:00028CBF       snd_register_oss_device_
 0003:00028E3E       snd_unregister_oss_device_
 0003:000290AE       snd_minor_info_oss_init_
 0003:0002911B       snd_minor_info_oss_done_
 0003:00029186       snd_device_new_
 0003:00029253       snd_device_free_
 0003:0002937E       snd_device_disconnect_
 0003:00029451       snd_device_register_
 0003:0002952D       snd_device_register_all_
 0003:000295D4       snd_device_disconnect_all_
 0003:00029659       snd_device_free_all_
 0003:00029BFD       snd_ctl_notify_
 0003:00029E13       snd_ctl_new1_
 0003:00029F7D       snd_ctl_free_one_
 0003:0002A10D       snd_ctl_add_
 0003:0002A2A0       snd_ctl_remove_
 0003:0002A36C       snd_ctl_remove_id_
 0003:0002A4C4       snd_ctl_rename_id_
 0003:0002A55E       snd_ctl_find_numid_
 0003:0002A5EB       snd_ctl_find_id_
 0003:0002C187       snd_ctl_register_ioctl_
 0003:0002C278       snd_ctl_unregister_ioctl_
 0003:0002C569       snd_ctl_create_
 0003:0002C5BD       snd_ctl_boolean_mono_info_
 0003:0002C60B       snd_ctl_boolean_stereo_info_
 0003:0002C6DC       snd_malloc_pages_
 0003:0002C748       snd_free_pages_
 0003:0002C798       snd_malloc_dev_pages_
 0003:0002C80D       snd_free_dev_pages_
 0003:0002C870       snd_dma_alloc_pages_
 0003:0002C981       snd_dma_alloc_pages_fallback_
 0003:0002CA1E       snd_dma_free_pages_
 0003:0002CAA4       snd_dma_get_reserved_buf_
 0003:0002CBC9       snd_dma_reserve_buf_
 0003:0002CEE4       snd_card_create_
 0003:0002D257       snd_card_locked_
 0003:0002D4A1       snd_card_disconnect_
 0003:0002D709       snd_card_free_when_closed_
 0003:0002D7C7       snd_card_free_
 0003:0002DAC4       snd_card_set_id_
 0003:0002DB0A       snd_card_register_
 0003:0002DCAC       snd_card_info_read_oss_
 0003:0002DD9C       snd_card_info_init_
 0003:0002DE55       snd_card_info_done_
 0003:0002DE8B       snd_component_add_
 0003:0002DF8F       snd_card_file_add_
 0003:0002E05F       snd_card_file_remove_
 0003:0002E1BA       snd_power_wait_
 0003:0002E30E       snd_free_sgbuf_pages_
 0003:0002E38A       snd_malloc_sgbuf_pages_
 0003:00053E64       ioread8_
 0003:00053EB0       ioread16_
 0003:00053EFE       ioread32_
 0003:00053F43       iowrite8_
 0003:00053F86       iowrite16_
 0003:00053FCB       iowrite32_
 0003:0005400E       ioport_map_
 0003:0005404A       ioport_unmap_
 0003:00054065       pci_iomap_
 0003:00054295       pci_iounmap_
 0003:0005430B       snd_ca0106_ptr_read_
 0003:00054371       snd_ca0106_ptr_write_
 0003:000543CF       snd_ca0106_spi_write_
 0003:000544EC       snd_ca0106_i2c_write_
 0003:000573C2       ca_midi_init_
 0003:000586F7       snd_ca0106_mixer_
 0003:0005898D       snd_ca0106_mixer_suspend_
 0003:000589EC       snd_ca0106_mixer_resume_
 0003:000596A2       snd_ca0106_proc_init_
 0003:00083881       snd_hda_add_codec_preset_
 0003:000838E2       snd_hda_delete_codec_preset_
 0003:0008394C       snd_hda_get_jack_location_
 0003:000839D7       snd_hda_get_jack_connectivity_
 0003:00083A0A       snd_hda_get_jack_type_
 0003:00083BFD       snd_hda_codec_read_
 0003:00083C4F       snd_hda_codec_write_
 0003:00083CBB       snd_hda_sequence_write_
 0003:00083D07       snd_hda_get_sub_nodes_
 0003:00083D6E       snd_hda_get_connections_
 0003:00084076       snd_hda_queue_unsol_event_
 0003:00084293       snd_hda_bus_new_
 0003:00084A1C       snd_hda_add_pincfg_
 0003:00084AEC       snd_hda_codec_set_pincfg_
 0003:00084B29       snd_hda_codec_get_pincfg_
 0003:00084C5C       snd_hda_shutup_pins_
 0003:00084E46       snd_hda_codec_new_
 0003:0008530B       snd_hda_codec_configure_
 0003:00085453       snd_hda_codec_setup_stream_
 0003:000854DF       snd_hda_codec_cleanup_stream_
 0003:00085712       query_amp_caps_
 0003:000857EE       snd_hda_override_amp_caps_
 0003:00085927       snd_hda_query_pin_caps_
 0003:00085968       snd_hda_pin_sense_
 0003:000859DE       snd_hda_jack_detect_
 0003:00085BB6       snd_hda_codec_amp_read_
 0003:00085C45       snd_hda_codec_amp_update_
 0003:00085D46       snd_hda_codec_amp_stereo_
 0003:00085DCA       snd_hda_codec_resume_amp_
 0003:00085EB0       snd_hda_mixer_amp_volume_info_
 0003:0008605C       snd_hda_mixer_amp_volume_get_
 0003:00086137       snd_hda_mixer_amp_volume_put_
 0003:00086229       snd_hda_mixer_amp_tlv_
 0003:00086360       snd_hda_set_vmaster_tlv_
 0003:00086471       snd_hda_find_mixer_ctl_
 0003:000864A0       snd_hda_ctl_add_
 0003:00086574       snd_hda_add_nid_
 0003:00086605       snd_hda_ctls_clear_
 0003:00086723       snd_hda_codec_reset_
 0003:0008698E       snd_hda_add_vmaster_
 0003:00086AEC       snd_hda_mixer_amp_switch_info_
 0003:00086B5E       snd_hda_mixer_amp_switch_get_
 0003:00086C4C       snd_hda_mixer_amp_switch_put_
 0003:00086D5D       snd_hda_mixer_bind_switch_get_
 0003:00086DD3       snd_hda_mixer_bind_switch_put_
 0003:00086EA7       snd_hda_mixer_bind_ctls_info_
 0003:00086F1D       snd_hda_mixer_bind_ctls_get_
 0003:00086F94       snd_hda_mixer_bind_ctls_put_
 0003:00087054       snd_hda_mixer_bind_tlv_
 0003:00087648       snd_hda_create_spdif_out_ctls_
 0003:0008780D       snd_hda_create_spdif_share_sw_
 0003:00087A04       snd_hda_create_spdif_in_ctls_
 0003:00087AFE       snd_hda_codec_write_cache_
 0003:00087BAF       snd_hda_codec_update_cache_
 0003:00087C6A       snd_hda_codec_resume_cache_
 0003:00087CF2       snd_hda_sequence_write_cache_
 0003:00087FFB       snd_hda_build_controls_
 0003:0008809A       snd_hda_codec_build_controls_
 0003:0008810E       snd_hda_calc_stream_format_
 0003:000886A1       snd_hda_is_supported_format_
 0003:00088BA1       snd_hda_codec_build_pcms_
 0003:00088CD7       snd_hda_build_pcms_
 0003:00088D3F       snd_hda_check_board_config_
 0003:00088ECE       snd_hda_check_board_codec_sid_config_
 0003:00089001       snd_hda_add_new_ctls_
 0003:000890DB       snd_hda_ch_mode_info_
 0003:00089158       snd_hda_ch_mode_get_
 0003:000891B4       snd_hda_ch_mode_put_
 0003:00089246       snd_hda_input_mux_info_
 0003:000892E4       snd_hda_input_mux_put_
 0003:000894D3       snd_hda_bus_reboot_notify_
 0003:00089532       snd_hda_multi_out_dig_open_
 0003:00089596       snd_hda_multi_out_dig_prepare_
 0003:000895F1       snd_hda_multi_out_dig_cleanup_
 0003:00089642       snd_hda_multi_out_dig_close_
 0003:0008968C       snd_hda_multi_out_analog_open_
 0003:0008983D       snd_hda_multi_out_analog_prepare_
 0003:00089A3C       snd_hda_multi_out_analog_cleanup_
 0003:00089C62       snd_hda_parse_pin_def_config_
 0003:0008A4D8       snd_hda_suspend_
 0003:0008A52F       snd_hda_resume_
 0003:0008A586       snd_array_new_
 0003:0008A690       snd_array_free_
 0003:0008A6D3       snd_print_pcm_rates_
 0003:0008A74F       snd_print_pcm_bits_
 0003:0008AAC1       snd_hda_create_hwdep_
 0003:0008CAD9       snd_hda_parse_generic_codec_
 0003:0008CC07       ilog2_
 0003:0008E65C       snd_hda_codec_proc_new_
 0003:0008E8B8       snd_seq_device_load_drivers_
 0003:0008E8D0       snd_seq_device_new_
 0003:0008EC2B       snd_seq_device_register_driver_
 0003:0008EE18       snd_seq_device_unregister_driver_
 0003:0008F3AD       snd_seq_info_init_
 0003:0008F40B       snd_seq_info_done_
 0003:0008F4CB       snd_seq_system_broadcast_
 0003:0008F513       snd_seq_system_notify_
 0003:0008F5AA       snd_seq_system_client_init_
 0003:0008F720       snd_seq_system_client_done_
 0003:0008F834       snd_seq_queue_get_cur_queues_
 0003:0008FB06       snd_seq_queues_init_
 0003:0008FB28       snd_seq_queues_delete_
 0003:0008FB75       snd_seq_queue_alloc_
 0003:0008FBF2       snd_seq_queue_delete_
 0003:0008FC52       queueptr_
 0003:0008FCB5       snd_seq_queue_find_name_
 0003:0008FD1F       snd_seq_check_queue_
 0003:0008FEA8       snd_seq_enqueue_event_
 0003:000900A7       snd_seq_queue_check_access_
 0003:0009010D       snd_seq_queue_set_owner_
 0003:000901B3       snd_seq_queue_timer_open_
 0003:00090225       snd_seq_queue_timer_close_
 0003:0009027B       snd_seq_queue_timer_set_tempo_
 0003:00090337       snd_seq_queue_use_
 0003:00090418       snd_seq_queue_is_used_
 0003:0009048D       snd_seq_queue_client_termination_
 0003:0009052B       snd_seq_queue_client_leave_
 0003:000905EE       snd_seq_queue_client_leave_cells_
 0003:00090651       snd_seq_queue_remove_cells_
 0003:00090918       snd_seq_control_queue_
 0003:000909B5       snd_seq_info_queues_read_
 0003:00090BFD       snd_seq_dump_var_event_
 0003:00090DD6       snd_seq_expand_var_event_
 0003:00090F0F       snd_seq_cell_free_
 0003:000911B4       snd_seq_event_dup_
 0003:000913C2       snd_seq_pool_poll_wait_
 0003:00091435       snd_seq_pool_init_
 0003:00091559       snd_seq_pool_done_
 0003:00091689       snd_seq_pool_new_
 0003:00091736       snd_seq_pool_delete_
 0003:0009178B       snd_sequencer_memory_init_
 0003:000917AD       snd_sequencer_memory_done_
 0003:000917C5       snd_seq_info_pool_
 0003:000919D2       snd_seq_client_use_ptr_
 0003:00091AB8       client_init_data_
 0003:000927F8       snd_seq_dispatch_event_
 0003:000936D7       snd_seq_client_notify_subscription_
 0003:00093F4B       snd_seq_set_queue_tempo_
 0003:00094CE7       snd_seq_create_kernel_client_
 0003:00094E29       snd_seq_delete_kernel_client_
 0003:00094F6E       snd_seq_kernel_client_enqueue_
 0003:00094FA9       snd_seq_kernel_client_enqueue_blocking_
 0003:00094FEA       snd_seq_kernel_client_dispatch_
 0003:00095097       snd_seq_kernel_client_ctl_
 0003:00095101       snd_seq_kernel_client_write_poll_
 0003:000954D4       snd_seq_info_clients_read_
 0003:000956AC       snd_sequencer_device_init_
 0003:00095725       snd_sequencer_device_done_
 0003:00095814       snd_seq_port_use_ptr_
 0003:000958C3       snd_seq_port_query_nearest_
 0003:00095A01       snd_seq_create_port_
 0003:00095E9A       snd_seq_delete_port_
 0003:00095F8D       snd_seq_delete_all_ports_
 0003:000960F5       snd_seq_set_port_info_
 0003:0009624B       snd_seq_get_port_info_
 0003:000965CF       snd_seq_port_connect_
 0003:0009690E       snd_seq_port_disconnect_
 0003:00096AC5       snd_seq_port_get_subscription_
 0003:00096B45       snd_seq_event_port_attach_
 0003:00096C01       snd_seq_event_port_detach_
 0003:00096D9C       snd_seq_timer_new_
 0003:00096E07       snd_seq_timer_delete_
 0003:00096E67       snd_seq_timer_defaults_
 0003:00096F0C       snd_seq_timer_reset_
 0003:00097060       snd_seq_timer_set_tempo_
 0003:000970E8       snd_seq_timer_set_ppq_
 0003:0009719F       snd_seq_timer_set_position_tick_
 0003:0009720F       snd_seq_timer_set_position_time_
 0003:00097280       snd_seq_timer_set_skew_
 0003:0009730B       snd_seq_timer_open_
 0003:00097471       snd_seq_timer_close_
 0003:000974E6       snd_seq_timer_stop_
 0003:00097641       snd_seq_timer_start_
 0003:000976C7       snd_seq_timer_continue_
 0003:00097756       snd_seq_timer_get_cur_time_
 0003:000977F4       snd_seq_timer_get_cur_tick_
 0003:0009781B       snd_seq_info_timer_read_
 0003:0009796A       snd_seq_prioq_new_
 0003:000979E2       snd_seq_prioq_delete_
 0003:00097B9C       snd_seq_prioq_cell_in_
 0003:00097D2D       snd_seq_prioq_cell_out_
 0003:00097DC5       snd_seq_prioq_avail_
 0003:00097E09       snd_seq_prioq_cell_peek_
 0003:00097EF6       snd_seq_prioq_leave_
 0003:0009821B       snd_seq_prioq_remove_events_
 0003:00098371       snd_seq_fifo_new_
 0003:00098454       snd_seq_fifo_delete_
 0003:000984FA       snd_seq_fifo_clear_
 0003:00098553       snd_seq_fifo_event_in_
 0003:000986A6       snd_seq_fifo_cell_out_
 0003:000987B6       snd_seq_fifo_cell_putback_
 0003:0009880C       snd_seq_fifo_poll_wait_
 0003:0009885C       snd_seq_fifo_resize_
 0003:0009895D       snd_opl3_synth_use_inc_
 0003:0009899E       snd_opl3_synth_use_dec_
 0003:000989D2       snd_opl3_synth_setup_
 0003:00098AD9       snd_opl3_synth_cleanup_
 0003:00099642       snd_opl3_interrupt_
 0003:00099770       snd_opl3_new_
 0003:0009982E       snd_opl3_init_
 0003:000998E2       snd_opl3_create_
 0003:00099AAD       snd_opl3_timer_new_
 0003:00099B33       snd_opl3_hwdep_new_
 0003:00099FFF       snd_opl3_load_drums_
 0003:0009A08F       snd_opl3_drum_switch_
 0003:0009A18F       snd_opl3_calc_volume_
 0003:0009A54B       snd_opl3_timer_func_
 0003:0009A6BD       snd_opl3_note_on_
 0003:0009B0AA       snd_opl3_note_off_
 0003:0009B0FC       snd_opl3_key_press_
 0003:0009B120       snd_opl3_terminate_note_
 0003:0009B302       snd_opl3_control_
 0003:0009B3C2       snd_opl3_nrpn_
 0003:0009B3E5       snd_opl3_sysex_
 0003:0009B40B       snd_opl3_open_
 0003:0009B431       snd_opl3_ioctl_
 0003:0009B66B       snd_opl3_release_
 0003:0009B6A5       snd_opl3_write_
 0003:0009B7C1       snd_opl3_load_patch_
 0003:0009B9C1       snd_opl3_find_patch_
 0003:0009BAAB       snd_opl3_clear_patches_
 0003:0009BB1B       snd_opl3_reset_
 0003:0009C306       snd_mpu401_uart_interrupt_
 0003:0009C349       snd_mpu401_uart_interrupt_tx_
 0003:0009CD24       snd_mpu401_uart_new_
 0003:0009DF4D       snd_cs46xx_download_
 0003:0009DFDA       snd_cs46xx_download_image_
 0003:0009F695       snd_cs46xx_pcm_
 0003:0009FAC0       snd_cs46xx_mixer_
 0003:000A01AF       snd_cs46xx_midi_
 0003:000A028E       snd_cs46xx_gameport_
 0003:000A0BA6       snd_cs46xx_start_dsp_
 0003:000A10E1       snd_cs46xx_suspend_
 0003:000A1235       snd_cs46xx_resume_
 0003:000A13CC       snd_cs46xx_create_
 0003:000A2351       snd_cs5535audio_suspend_
 0003:000A245B       snd_cs5535audio_resume_
 0003:000A3031       snd_cs5535audio_pcm_
 0003:000A44A6       snd_p16v_free_
 0003:000A44DF       snd_p16v_pcm_
 0003:000A4B8C       snd_p16v_mixer_
 0003:000A4C02       snd_p16v_alloc_pm_buffer_
 0003:000A4C51       snd_p16v_free_pm_buffer_
 0003:000A4C7A       snd_p16v_suspend_
 0003:000A4CEA       snd_p16v_resume_
 0003:000A4E73       snd_emu10k1_timer_
 0003:000A53F1       snd_emu10k1_fx8010_register_irq_handler_
 0003:000A54DF       snd_emu10k1_fx8010_unregister_irq_handler_
 0003:000A575E       snd_emu10k1_efx_read_
 0003:000ABED2       snd_emu10k1_init_efx_
 0003:000ABF40       snd_emu10k1_free_efx_
 0003:000ABFB0       snd_emu10k1_fx8010_tram_setup_
 0003:000ACB4E       snd_emu10k1_fx8010_new_
 0003:000ACC24       snd_emu10k1_efx_alloc_pm_buffer_
 0003:000ACD5B       snd_emu10k1_efx_free_pm_buffer_
 0003:000ACDAE       snd_emu10k1_efx_suspend_
 0003:000ACF53       snd_emu10k1_efx_resume_
 0003:000AF7AA       snd_emu10k1_mixer_
 0003:000B320B       snd_emu10k1_pcm_
 0003:000B3386       snd_emu10k1_pcm_multi_
 0003:000B34AF       snd_emu10k1_pcm_mic_
 0003:000B4044       snd_emu10k1_pcm_efx_
 0003:000B4B7E       snd_emu10k1_midi_
 0003:000B4C0D       snd_emu10k1_audigy_midi_
 0003:000B4D0C       snd_emu10k1_voice_init_
 0003:000B56E4       snd_emu10k1_done_
 0003:000B6A4A       snd_emu10k1_create_
 0003:000B7423       snd_emu10k1_suspend_regs_
 0003:000B7520       snd_emu10k1_resume_init_
 0003:000B75A8       snd_emu10k1_resume_regs_
 0003:000B8373       snd_emu10k1_proc_init_
 0003:000B8673       snd_emu10k1_ptr_read_
 0003:000B8784       snd_emu10k1_ptr_write_
 0003:000B88C1       snd_emu10k1_ptr20_read_
 0003:000B892E       snd_emu10k1_ptr20_write_
 0003:000B8993       snd_emu10k1_spi_write_
 0003:000B8AF1       snd_emu10k1_i2c_write_
 0003:000B8C65       snd_emu1010_fpga_write_
 0003:000B8D2B       snd_emu1010_fpga_read_
 0003:000B8DCC       snd_emu1010_fpga_link_dst_src_write_
 0003:000B8E42       snd_emu10k1_intr_enable_
 0003:000B8E9C       snd_emu10k1_intr_disable_
 0003:000B8EF8       snd_emu10k1_voice_intr_enable_
 0003:000B8F9A       snd_emu10k1_voice_intr_disable_
 0003:000B9040       snd_emu10k1_voice_intr_ack_
 0003:000B90C6       snd_emu10k1_voice_half_loop_intr_enable_
 0003:000B9168       snd_emu10k1_voice_half_loop_intr_disable_
 0003:000B920E       snd_emu10k1_voice_half_loop_intr_ack_
 0003:000B9294       snd_emu10k1_voice_set_loop_stop_
 0003:000B9336       snd_emu10k1_voice_clear_loop_stop_
 0003:000B93DC       snd_emu10k1_wait_
 0003:000B945E       snd_emu10k1_ac97_read_
 0003:000B94C7       snd_emu10k1_ac97_write_
 0003:000B9528       snd_emu10k1_rate_to_pitch_
 0003:000B97A9       snd_emu10k1_voice_alloc_
 0003:000B9917       snd_emu10k1_voice_free_
 0003:000B9FE5       snd_emu10k1_memblk_map_
 0003:000BA125       snd_emu10k1_alloc_pages_
 0003:000BA2F2       snd_emu10k1_free_pages_
 0003:000BA33D       snd_emu10k1_synth_alloc_
 0003:000BA3E5       snd_emu10k1_synth_free_
 0003:000BA7BD       snd_emu10k1_synth_bzero_
 0003:000BA873       snd_emu10k1_synth_copy_from_user_
 0003:000BA941       snd_emu10k1_interrupt_
 0003:000BAE92       snd_ymfpci_free_gameport_
 0003:000BDE7F       snd_ymfpci_pcm_
 0003:000BDF83       snd_ymfpci_pcm2_
 0003:000BE081       snd_ymfpci_pcm_spdif_
 0003:000BE173       snd_ymfpci_pcm_4ch_
 0003:000BF3F2       snd_ymfpci_mixer_
 0003:000BF8DB       snd_ymfpci_timer_
 0003:000C0A74       snd_ymfpci_suspend_
 0003:000C0BFC       snd_ymfpci_resume_
 0003:000C0D8A       snd_ymfpci_create_
 0003:000C5085       snd_trident_start_voice_
 0003:000C50DE       snd_trident_stop_voice_
 0003:000C52E1       snd_trident_write_voice_regs_
 0003:000C7821       snd_trident_pcm_
 0003:000C79D7       snd_trident_foldback_pcm_
 0003:000C7BEE       snd_trident_spdif_pcm_
 0003:000C943E       snd_trident_create_gameport_
 0003:000C9D6A       snd_trident_create_
 0003:000CA54C       snd_trident_alloc_voice_
 0003:000CA6A3       snd_trident_free_voice_
 0003:000CA8DE       snd_trident_suspend_
 0003:000CA9A9       snd_trident_resume_
 0003:000CAFCC       snd_trident_alloc_pages_
 0003:000CB030       snd_trident_free_pages_
 0003:000CDA55       snd_sbmixer_write_
 0003:000CDAA0       snd_sbmixer_read_
 0003:000CE879       snd_sbmixer_add_ctl_
 0003:000CEA27       snd_sbmixer_new_
 0003:000CED20       snd_sbmixer_suspend_
 0003:000CEDF7       snd_sbmixer_resume_
 0003:000CEECE       snd_sbdsp_command_
 0003:000CEF4D       snd_sbdsp_get_byte_
 0003:000CEFC9       snd_sbdsp_reset_
 0003:000CF369       snd_sbdsp_create_
 0003:000D0CDC       _snd_pcm_hw_param_set_
 0003:000D290E       snd_pcm_oss_write3_
 0003:000D29DF       snd_pcm_oss_read3_
 0003:000D2B07       snd_pcm_oss_writev3_
 0003:000D2BD8       snd_pcm_oss_readv3_
 0003:000D5EE0       ACPIFindPCIDevice
 0003:000D5F82       InitACPICall
 0003:000D6020       StrLen
 0003:000D6040       StrNCmp
 0003:000D6070       FindAddress
 0003:000D62DC       init_MUTEX_
 0003:000D6312       init_MUTEX_LOCKED_
 0003:000D6348       down_
 0003:000D637A       up_
 0003:000D63AC       down_interruptible_
 0003:000D6A30       _snd_ctl_add_slave_
 0003:000D6D3D       snd_ctl_make_virtual_master_
 0003:000D6E5F       release_and_free_resource_
 0003:000D6E90       snd_pci_quirk_lookup_id_
 0003:000D6F13       snd_pci_quirk_lookup_
 0003:000D6F52       copy_to_user_fromio_
 0003:000D7002       copy_from_user_toio_
 0003:000D73AD       snd_ac97_set_rate_
 0003:000D7A11       snd_ac97_pcm_assign_
 0003:000D7E62       snd_ac97_pcm_open_
 0003:000D81BD       snd_ac97_pcm_close_
 0003:000D83AE       snd_ac97_pcm_double_rate_rules_
 0003:000DE322       snd_ac97_write_
 0003:000DE39C       snd_ac97_read_
 0003:000DE485       snd_ac97_write_cache_
 0003:000DE510       snd_ac97_update_
 0003:000DE5DF       snd_ac97_update_bits_
 0003:000DE654       snd_ac97_update_bits_nolock_
 0003:000E15C2       snd_ac97_get_name_
 0003:000E179A       snd_ac97_get_short_name_
 0003:000E1900       snd_ac97_bus_
 0003:000E19EC       snd_ac97_mixer_
 0003:000E2939       snd_ac97_suspend_
 0003:000E2ABC       snd_ac97_resume_
 0003:000E3600       snd_ac97_tune_hardware_
 0003:000E4FB3       snd_ac97_proc_init_
 0003:000E5148       snd_ac97_proc_done_
 0003:000E518D       snd_ac97_bus_proc_init_
 0003:000E5217       snd_ac97_bus_proc_done_
 0003:000E5247       snd_midi_process_event_
 0003:000E5A80       snd_midi_channel_set_clear_
 0003:000E61F4       snd_midi_channel_alloc_set_
 0003:000E6294       snd_midi_channel_free_set_
 0003:000E6343       snd_util_memhdr_new_
 0003:000E63B3       snd_util_memhdr_free_
 0003:000E6427       __snd_util_mem_alloc_
 0003:000E6508       __snd_util_memblk_new_
 0003:000E65C0       snd_util_mem_alloc_
 0003:000E6609       __snd_util_mem_free_
 0003:000E666F       snd_util_mem_free_
 0003:000E66D4       snd_util_mem_avail_
 0003:000E6760       __U8RS
 0003:000E677A       __I8RS
 0003:000E6795       __I8LS
 0003:000E6795       __U8LS
 0003:000E67B0       __I8M
 0003:000E67B0       __U8M
 0003:000E67D0       strstr_
 0003:000E6880       strlcpy_
 0003:000E6910       vsscanf_
 0003:000E6940       sscanf_
 0003:000E69B0       vsnprintf_
 0003:000E6A10       snprintf_
 0003:000E6A40       memset_
 0003:000E6A60       memmove_
 0003:000E6CE0       strtoul_
 0003:000E6CF0       strtol_
 0003:000E6D00       __IsTable
 0003:000E6E10       __STOSB
 0003:000E6E47       __STOSD
 0003:000E7A20       __scnf_
 0003:000E7C90       __prtf_
 0003:000E8974       __set_errno_
 0003:000E8982       __set_EDOM_
 0003:000E8990       __set_ERANGE_
 0003:000E899E       __set_EINVAL_
 0003:000E89B1       __set_doserrno_
 0003:000E89C0       tolower_
 0003:000E89D0       __FDFS
 0003:000E8A20       strupr_
 0003:000E8A40       __Bits
 0003:000E8A9C       __threadstack_
 0003:000E8AA3       __threadid_
 0003:000E8AAC       __OS2MainInit_
 0003:000E8B1B       __OS2Init_
 0003:000E8B59       __OS2Fini_
 0003:000E8B61       __shutdown_stack_checking_
 0003:000E8B76       __exit_
 0003:000E8BC0       wctomb_
 0003:000E8BF0       mbtowc_
 0003:000E8CB0       _ismbblead_
 0003:000E8CD0       ultoa_
 0003:000E8D20       ltoa_
 0003:000E8D50       ulltoa_
 0003:000E8DC0       lltoa_
 0003:000E8DF0       utoa_
 0003:000E8E40       itoa_
 0003:000E8E70       __exit_with_msg_
 0003:000E8EC0       __fatal_runtime_error_
 0003:000E8EF0       __InitRtns
 0003:000E8F40       __FiniRtns
 0003:000E8FA0       __CommonInit_
 0003:000E8FE5       __mbinit_
 0003:000E90E0       __EnterWVIDEO_
 0003:000E9108       __OffFinalCS32
 0004:00000003       ___begtext
 0005:00000000       __OffBeginDS32
 0005:00000030       W?deviceOwner$nul
 0005:00000034       W?numOS2Opens$nul
 0005:00000038       _rdOffset
 0005:0000003C       _wrOffset
 0005:00000040       _szprintBuf
 0005:00000044       _fVerbose
 0005:00000048       _fDebug
 0005:0000004C       _idc16_PddHandler
 0005:00000054       W?RM_Help$npn()i
 0005:00000058       W?RM_Help0$npn()i
 0005:0000005C       W?RM_Help3$npn()i
 0005:00000060       W?RMFlags$nul
 0005:000000B0       W?fnCardExitCall$n[]pn()v
 0005:000000D0       _nrCardsDetected
 0005:000000D4       _fStrategyInit
 0005:000000D8       _DbgInt
 0005:000000FC       _DebugLevel
 0005:00000104       _ulget_free_pagesMemUsed
 0005:00000548       W?pmbUsed$npn$_MEMBLOCK$$
 0005:0000054C       W?pmbFree$npn$_MEMBLOCK$$
 0005:00000550       W?uMemFree$nui
 0005:00000554       W?acHeap$npnuc
 0005:00000558       W?ulnAlloc$nul
 0005:0000055C       W?ulcAlloc$nul
 0005:00000560       W?ulnAllocCalls$nul
 0005:00000564       W?ulnFree$nul
 0005:00000568       W?ulcFree$nul
 0005:0000056C       W?ulnFreeCalls$nul
 0005:00000570       W?ulnCompact$nul
 0005:0000059C       _snd_pcm_devices_os2
 0005:00000AA4       _snd_ecards_limit
 0005:00000AA8       _snd_major
 0005:00000AB4       _snd_seq_root
 0005:00000AB8       _snd_oss_root
 0005:00000DA8       _snd_cards
 0005:00001520       ___Is_DLL
 0005:00001524       ___saved_CS
 0005:00001628       ___MBCSIsTable
 0005:0000172C       ___IsDBCS
 0005:00001730       ___hmodule
 0005:00001754       BootCode
 0005:00001764       stackbase
 0005:00001768       stacksel
 0005:0000176C       __OffsetFinalCS16
 0005:0000176E       __OffsetFinalDS16
 0005:00001770       _MSG_TABLE32
 0005:00001774       PDDName
 0005:00001778       RMAllocResource1632
 0005:00001780       RMModifyResources1632
 0005:00001788       RMDeallocResource1632
 0005:00001790       RMCreateDevice1632
 0005:00001798       RMCreateAdapter1632
 0005:000017A0       RMCreateDriver1632
 0005:000017A8       RMDestroyDriver1632
 0005:000017B0       RMGetNodeInfo1632
 0005:000017B8       RMDevIDToHandleList1632
 0005:000017C0       RMHandleToResourceHandleList1632
 0005:000017C8       _TimerHandler16
 0005:000017CE       _ISR00
 0005:000017D2       _ISR01
 0005:000017D6       _ISR02
 0005:000017DA       _ISR03
 0005:000017DE       _ISR04
 0005:000017E2       _ISR05
 0005:000017E6       _ISR06
 0005:000017EA       _ISR07
 0005:000017F0       DevHelp32
 0005:000017F4       intSwitchStack
 0005:000017F8       _TKSSBase
 0005:00001800       W?StratDispatch$n[]pn(pf$RP$$)ul
 0005:00001894       W?ForceCard$ni
 0005:000018C4       _jiffies
 0005:000018C8       _current_task
 0005:000018EC       _current
 0005:000018F0       _system_utsname
 0005:00001A76       _ioport_resource
 0005:00001A92       _iomem_resource
 0005:00001AAE       _mem_map
 0005:00001AB2       _this_module
 0005:00001BB2       _szLastALSAError1
 0005:00001C32       _szOverrunTest1
 0005:00001C33       _szLastALSAError2
 0005:00001CB3       _szOverrunTest2
 0005:00001CB4       _iLastError
 0005:00001CB8       _proc_root
 0005:00001D04       _cardcalls
 0005:00001E0C       _midi_port
 0005:00001F78       _szRecSources
 0005:00002004       _oss_devices
 0005:00002144       _alsa_fops
 0005:00002148       _per_bytes
 0005:0000214C       _prev_size
 0005:00002150       _pcm_device
 0005:00002154       _total
 0005:00002158       _opened_handles
 0005:000081D4       _CountWv
 0005:000081D8       _LockAdd
 0005:000081DC       _hextab
 0005:000081ED       _MAGIC_COMM_PORT
 0005:000081F0       _pcmcaps
 0005:00008210       _substream_int
 0005:0000A210       _control_id_changed
 0005:0000A214       _card_id_changed
 0005:0000A218       _unlock_all
 0005:0000A21C       _fInInterrupt
 0005:0000AA9C       _pci_devices
 0005:0000D5DC       _fRewired
 0005:0000E9E0       W?ulcTotalHeap$nul
 0005:0000EA44       ___initcall_alsa_hwdep_init
 0005:0000EA48       ___exitcall_alsa_hwdep_exit
 0005:0000EAF0       ___initcall_alsa_timer_init
 0005:0000EAF4       ___exitcall_alsa_timer_exit
 0005:0000EB80       ___initcall_alsa_rawmidi_init
 0005:0000EB84       ___exitcall_alsa_rawmidi_exit
 0005:0000EF10       ___initcall_alsa_pcm_init
 0005:0000EF14       ___exitcall_alsa_pcm_exit
 0005:0000EF6C       ___initcall_alsa_sound_init
 0005:0000EF70       ___exitcall_alsa_sound_exit
 0005:0000EFF4       _snd_pcm_link_rwlock
 0005:0000F0B8       _snd_pcm_f_ops
 0005:0000F1C4       ___initcall_snd_mem_init
 0005:0000F1C8       ___exitcall_snd_mem_exit
 0005:0000F480       ___initcall_alsa_card_bt87x_init
 0005:0000F484       ___exitcall_alsa_card_bt87x_exit
 0005:0000F5E4       ___initcall_alsa_card_als4000_init
 0005:0000F5E8       ___exitcall_alsa_card_als4000_exit
 0005:00010365       ___initcall_alsa_card_cmipci_init
 0005:00010369       ___exitcall_alsa_card_cmipci_exit
 0005:00010694       ___initcall_alsa_card_atiixp_init
 0005:00010698       ___exitcall_alsa_card_atiixp_exit
 0005:00010B00       ___initcall_alsa_card_fm801_init
 0005:00010B04       ___exitcall_alsa_card_fm801_exit
 0005:00011178       ___initcall_alsa_card_via82xx_init
 0005:0001117C       ___exitcall_alsa_card_via82xx_exit
 0005:000117C0       ___initcall_alsa_card_m3_init
 0005:000117C4       ___exitcall_alsa_card_m3_exit
 0005:000124F0       ___initcall_alsa_card_intel8x0_init
 0005:000124F4       ___exitcall_alsa_card_intel8x0_exit
 0005:00012734       ___initcall_alsa_card_es1968_init
 0005:00012738       ___exitcall_alsa_card_es1968_exit
 0005:00012F95       ___initcall_alsa_card_es1938_init
 0005:00012F99       ___exitcall_alsa_card_es1938_exit
 0005:00013230       ___initcall_alsa_card_cs4281_init
 0005:00013234       ___exitcall_alsa_card_cs4281_exit
 0005:0001365C       ___initcall_alsa_card_ens137x_init
 0005:00013660       ___exitcall_alsa_card_ens137x_exit
 0005:00013B10       ___initcall_alsa_card_ca0106_init
 0005:00013B14       ___exitcall_alsa_card_ca0106_exit
 0005:00016B90       ___initcall_patch_via_init
 0005:00016B94       ___exitcall_patch_via_exit
 0005:0001937C       ___initcall_patch_conexant_init
 0005:00019380       ___exitcall_patch_conexant_exit
 0005:000194DC       ___initcall_patch_atihdmi_init
 0005:000194E0       ___exitcall_patch_atihdmi_exit
 0005:0001BFD0       ___initcall_patch_sigmatel_init
 0005:0001BFD4       ___exitcall_patch_sigmatel_exit
 0005:00023830       ___initcall_patch_analog_init
 0005:00023834       ___exitcall_patch_analog_exit
 0005:00023FD4       ___initcall_patch_cmedia_init
 0005:00023FD8       ___exitcall_patch_cmedia_exit
 0005:00043363       ___initcall_patch_realtek_init
 0005:00043367       ___exitcall_patch_realtek_exit
 0005:000436A4       ___initcall_alsa_card_azx_init
 0005:000436A8       ___exitcall_alsa_card_azx_exit
 0005:000437FB       _snd_hda_bind_vol
 0005:0004380B       _snd_hda_bind_sw
 0005:00043A67       _snd_hda_pcm_type_name
 0005:00043AC7       _auto_pin_cfg_labels
 0005:00043C94       _seq_client_load
 0005:00043CD0       _seq_default_timer_class
 0005:00043CD4       _seq_default_timer_sclass
 0005:00043CD8       _seq_default_timer_card
 0005:00043CDC       _seq_default_timer_device
 0005:00043CE0       _seq_default_timer_subdevice
 0005:00043CE4       _seq_default_timer_resolution
 0005:00043CE8       ___initcall_alsa_seq_init
 0005:00043CEC       ___exitcall_alsa_seq_exit
 0005:00043D10       ___initcall_alsa_seq_device_init
 0005:00043D14       ___exitcall_alsa_seq_device_exit
 0005:00043E64       _use_internal_drums
 0005:00043E68       _opl3_ops
 0005:00043E8C       ___initcall_alsa_opl3_seq_init
 0005:00043E90       ___exitcall_alsa_opl3_seq_exit
 0005:00043F00       ___initcall_alsa_opl3_init
 0005:00043F04       ___exitcall_alsa_opl3_exit
 0005:00044098       _snd_opl3_regmap
 0005:000440DC       ___initcall_alsa_mpu401_uart_init
 0005:000440E0       ___exitcall_alsa_mpu401_uart_exit
 0005:00044188       ___initcall_alsa_card_cs46xx_init
 0005:0004418C       ___exitcall_alsa_card_cs46xx_exit
 0005:00051E10       ___initcall_alsa_card_cs5535audio_init
 0005:00051E14       ___exitcall_alsa_card_cs5535audio_exit
 0005:0005200C       ___initcall_alsa_card_emu10k1_init
 0005:00052010       ___exitcall_alsa_card_emu10k1_exit
 0005:00054CE4       ___initcall_alsa_card_ymfpci_init
 0005:00054CE8       ___exitcall_alsa_card_ymfpci_exit
 0005:0005566C       ___initcall_alsa_card_ali_init
 0005:00055670       ___exitcall_alsa_card_ali_exit
 0005:00055738       ___initcall_alsa_card_trident_init
 0005:0005573C       ___exitcall_alsa_card_trident_exit
 0005:000623D0       ___initcall_alsa_card_nm256_init
 0005:000623D4       ___exitcall_alsa_card_nm256_exit
 0005:0006289C       ___initcall_alsa_sb_common_init
 0005:000628A0       ___exitcall_alsa_sb_common_exit
 0005:0006291C       ___initcall_alsa_pcm_oss_init
 0005:00062920       ___exitcall_alsa_pcm_oss_exit
 0005:000629B0       ___EFG_printf
 0005:000629B4       ___EFG_scanf
 0005:000629B8       ___FirstThreadData
 0005:000629BC       ___GetThreadPtr
 0005:000629C0       __AccessFileH
 0005:000629C4       __ReleaseFileH
 0005:000629C8       __AccessIOB
 0005:000629CC       __ReleaseIOB
 0005:000629D0       __AccessNHeap
 0005:000629D4       __AccessFHeap
 0005:000629D8       __ReleaseNHeap
 0005:000629DC       __ReleaseFHeap
 0005:000629E0       __AccessTDList
 0005:000629E4       __ReleaseTDList
 0005:000629E8       ___sig_init_rtn
 0005:000629EC       ___sig_fini_rtn
 0005:000629F0       __threadstksize
 0005:000629F4       ___process_fini
 0005:000629F8       __dynend
 0005:000629FC       __curbrk
 0005:00062A00       __LpCmdLine
 0005:00062A04       __LpPgmName
 0005:00062A08       __LpDllName
 0005:00062A0C       __LpwCmdLine
 0005:00062A10       __LpwPgmName
 0005:00062A14       __LpwDllName
 0005:00062A18       __STACKLOW
 0005:00062A1C       __STACKTOP
 0005:00062A20       __ASTACKSIZ
 0005:00062A24       __ASTACKPTR
 0005:00062A28       __cbyte
 0005:00062A2C       __cbyte2
 0005:00062A30       __child
 0005:00062A34       __no87
 0005:00062A36       __Envptr
 0005:00062A3A       __Envseg
 0005:00062A3C       __osmajor
 0005:00062A3D       __osminor
 0005:00062A3E       ___FPE_handler
 0005:00062A44       ___MBCodePage
 0005:00062A48       ___WD_Present
 0005:00062A4C       __amblksiz
 0005:0006329E       ___initcall_alsa_ac97_init
 0005:000632A2       ___exitcall_alsa_ac97_exit
 0005:000633C8       ___initcall_alsa_seq_midi_emul_init
 0005:000633CC       ___exitcall_alsa_seq_midi_emul_exit
 0005:000633D0       ___initcall_alsa_util_mem_init
 0005:000633D4       ___exitcall_alsa_util_mem_exit
 0005:00076178       ___Alphabet
 0005:00078F98       _snd_pcm_known_rates
 0005:0007F534       __OffFinalDS32
 0005:0007F538       __Start_XI
 0005:0007F53E       __Start_YI
 0005:0007F53E       __End_XI
 0005:0007F53E       __End_YI
 0005:0007F590       __nullarea
 0005:0008F5A0       _edata
 0005:0008F5A0       _end
